:100000000C949B080C94EA080C94EA080C94EA08F7
:100010000C94EA080C94EA080C94EA080C94EA0898
:100020000C94EA080C94451C0C94EA080C94EA0819
:100030000C94E5350C94EA080C94EA080C94EA0850
:100040000C94EA080C94EA080C940C180C94EA0836
:100050000C943A0E0C94EA080C94040E0C94EA08E2
:100060000C94DE1E0C94EA080C946B310C94EA0894
:100070000C94F08C0C94EA080C94E2850C94EA0839
:100080000C94EA080C94EA080C94EA08051F0A1F6D
:100090000F1F181F2F1F461F561F661FA11F562117
:1000A000461FFE1F0F203E205C207920E0204821C3
:1000B0007C234924D8245825902533263A28A4287F
:1000C0001E296729B129DF290C2A6F2AB92A032B97
:1000D000FC2B8A31BE31013271328932CA3281330E
:1000E0004834483448344834483448344834483430
:1000F000483448344834FD33FF3304341C341E3450
:10010000EF7788780D796F79C3792C7A8181AD7A10
:10011000D17AD57AD57AD57AD57AD57AD57AD57A6B
:10012000D57A037B7E7B137C387C7B7CD77C627D9D
:100130004B7EA47EA87EA87EA87EA87EA87EA87EF0
:10014000A87EA87EE07EFE7E237F7F7FBB7F2A8005
:100150005780F78057815C815C815C815C815C8128
:100160005C815C815C81438B468B468B468B4F8BDD
:10017000528B558B678B648B0A0D3D3D3D3D3D3D5C
:100180003D3D3D3D3D3D3D3D3D3D3D3D3D3D3D3D9F
:100190003D3D3D3D3D3D3D3D3D3D3D3D3D000A0D2F
:1001A000426174743A002025642043656C6C7320AE
:1001B000004C6F772042617474206C6576656C3AF0
:1001C0002025642E2564000A0D466F756E6420425A
:1001D0004C2D4374726C3A20002564000A0D0A0D00
:1001E0002121204D495353494E4720424C2D435421
:1001F000524C3A202564202121000A0D43616C2EC7
:100200002070726573737572652073656E736F729B
:10021000004F4B0A0D000A0D466C696768742D7417
:10022000696D65202575206D696E20546F74616C51
:100230003A2575206D696E000A0D4143432D4848EB
:100240002056657273696F6E2070726F67616D6D95
:100250006564206279204D617274696E520A0D00E6
:10026000416E676C654E69636B2020202020202042
:10027000416E676C65526F6C6C202020202020201E
:100280004163634E69636B202020202020202020C2
:10029000416363526F6C6C2020202020202020209E
:1002A0005961774779726F2020202020202020205C
:1002B0004865696768742056616C75652020202048
:1002C0004163635A2020202020202020202020204D
:1002D0004761732020202020202020202020202063
:1002E000436F6D706173732056616C7565202020BB
:1002F000566F6C74616765205B302E31565D20202F
:100300005265636569766572204C6576656C202060
:100310004779726F20436F6D7061737320202020C6
:100320004D6F746F7220312020202020202020204B
:100330004D6F746F7220322020202020202020203A
:100340004D6F746F72203320202020202020202029
:100350004D6F746F72203420202020202020202018
:100360004D6F746F72203520202020202020202007
:100370004D6F746F722036202020202020202020F6
:100380006E6320616C74207370656564202020208A
:100390003139202020202020202020202020202033
:1003A000536572766F2020202020202020202020DE
:1003B000486F7665726761732020202020202020FE
:1003C00043757272656E74205B302E31415D202062
:1003D0004361706163697479205B6D41685D2020C1
:1003E000486967687420536574706F696E74202063
:1003F0004D6F746F72203720202020202020202075
:100400004D6F746F72203820202020202020202063
:10041000436F6D7061737320536574706F696E7490
:100420004932432D4572726F7220202020202020F7
:10043000424C204C696D697420202020202020200F
:100440004750535F4E69636B2020202020202020DE
:100450004750535F526F6C6C2020202020202020BA
:1004600021212120494E434F4D50415449424C4592
:1004700020212121002A002E000A0D204441432082
:100480006F7220493243204552524F522120436817
:1004900065636B204932432C2033567265662C20ED
:1004A00044414320616E6420424C2D4374726C00C1
:1004B0005B25695D005B25695D002B204D696B72D2
:1004C0006F4B6F70746572202B0048573A56256445
:1004D0002E25642053573A25642E25642563005346
:1004E000657474696E673A2564202573004D6978D8
:1004F0006572204572726F72210045525225326436
:100500003A004861726477617265204572726F7259
:1005100020313A2564202121004D697373696E678B
:1005200020424C2D4374726C3A25642121004932DB
:1005300043204552524F5221212100486569676886
:10054000743A202025356900536574706F696E74A4
:100550003A2535690050726573737572653A2535B1
:1005600069004F66667365743A2020253569004836
:10057000656967687420636F6E74726F6C004449BC
:100580005341424C4544006163742E2062656172A0
:10059000696E67004E69636B3A2020202020202579
:1005A000356900526F6C6C3A2020202020202535C0
:1005B0006900436F6D706173733A2020202535699F
:1005C000004B25693A25346920204B25693A2534AA
:1005D0006920004E693A2534692020526F3A25344B
:1005E00069200047733A253469202047693A253449
:1005F00069200050313A253469202050323A2534A0
:1006000069200050333A253469202050343A25348B
:100610006920004779726F202D2053656E736F72C9
:10062000004E69636B25346920282533692E2569BE
:100630002900526F6C6C25346920282533692E25DA
:10064000692900476965722534692028253369299D
:10065000004E69636B2025346920282533692E25D7
:10066000782900526F6C6C20253469202825336965
:100670002E257829005961772020253469202825E6
:10068000336929004E69636B20253469202825339E
:100690006929282533692900526F6C6C202534693B
:1006A00020282533692928253369290059617720B5
:1006B0002025346920282533692928253369290014
:1006C000414343202D2053656E736F72004E696362
:1006D0006B2025346920282533692900526F6C6C02
:1006E00020253469202825336929005A202020201C
:1006F00025346920282533692900566F6C74616799
:10070000653A2020202533692E253169560043752E
:100710007272656E743A2020202533692E25316966
:100720004100506F7765723A2020202020253469DF
:1007300057004469736368617267653A20253569BB
:100740006D41680052656365697665720052432D9C
:10075000525353493A202020202534690052432D1A
:100760005175616C6974793A202534690052432DC2
:100770004368616E6E656C733A25346900436F6D32
:1007800070617373004D61676E65743A2020202597
:100790003569004779726F3A20202020202535697D
:1007A00000536574706F696E743A20253569005086
:1007B0006F746925693A202025336900506F746988
:1007C00025693A202025336900536572766F202011
:1007D00000536574706F696E742020253369005072
:1007E0006F736974696F6E3A202533690052616EC8
:1007F00067653A2533692D25336900424C2D4374D2
:10080000726C204572726F7273200025336420254C
:10081000336420253364202533642000424C205467
:10082000656D70657261747572650025336420258D
:10083000336420253364202533642000424C2D434B
:1008400074726C20666F756E642000202563202012
:1008500020256320202025632020202563200020E0
:1008600025632020202563202020256320202025AB
:100870006320002025632020202D2020202D2020F3
:10088000202D2000313000313100313200466C69BA
:100890006768742D54696D65202000546F74616C15
:1008A0003A2535756D696E004163743A202025350F
:1008B000756D696E0028726573657429000A0D47AD
:1008C000656E65726174696E672064656661756CDA
:1008D0007420506172616D65746572205365742077
:1008E0002564000A0D5573696E6720506172616D51
:1008F0006574657220536574202564000A0D476590
:100900006E65726174696E672064656661756C748A
:10091000204D69786572205461626C65000A0D4D46
:10092000697865722D436F6E6669673A2027257373
:100930002720282575204D6F746F727329000A0DCA
:10094000414343206E6F742063616C69627261740D
:100950006564210D0A0000008F001E01AD013B02FD
:10096000CA025803E603740402058F051B06A70696
:100970003307BE074808D2085B09E3096B0AF20A8D
:10098000780BFD0B810C040D860D070E870E060FEC
:10099000840F00107B10F5106E11E5115B12CF1261
:1009A0004213B31323149214FE146A15D3153B1685
:1009B000A11605176717C81727188318DE183719E7
:1009C0008E19E319361A871AD61A231B6E1BB61B0B
:1009D000FD1B411C831CC31C001D3C1D751DAB1D54
:1009E000E01D121E421E6F1E9A1EC31EE91E0D1F21
:1009F0002E1F4D1F691F841F9B1FB01FC31FD31FB6
:100A0000E11FEC1FF51FFB1FFF1F00203E25336970
:100A10003D53657269616C706F7431003E253369B6
:100A20003D53657269616C706F7432004E6F204582
:100A300072726F722020202020202020004E6F74C0
:100A400020636F6D70617469626C652020004D4B8E
:100A5000334D6167206E6F7420636F6D7061004E5F
:100A60006F20464320636F6D6D756E69636174001E
:100A70004D4B334D616720636F6D6D756E696361BA
:100A80000047505320636F6D6D756E6963617469C3
:100A90006F00636F6D706173732076616C75652094
:100AA0002020005243205369676E616C206C6F7385
:100AB000742020004643207370692072782065728C
:100AC000726F7220004E6F204E4320636F6D6D7504
:100AD0006E69636174004643204E69636B204779F9
:100AE000726F2020202000464320526F6C6C2047FC
:100AF00079726F20202020004643205961772047DB
:100B000079726F2020202020004643204E69636BBD
:100B100020414343202020202000464320526F6C78
:100B20006C204143432020202020004643205A2DA2
:100B30004143432020202020202020005072657354
:100B4000737572652073656E736F7220004932434E
:100B50002046432D3E424C2D4374726C2000426C63
:100B6000204D697373696E67202020202020004D7E
:100B700069786572204572726F72202020202000F3
:100B80004361726566726565204572726F722020DE
:100B90000047505320466978206C6F7374202020E2
:100BA00020004D61676E6574204572726F7220205F
:100BB0002020004D6F746F722072657374617274BF
:100BC00020202000424C204C696D69746174696F6B
:100BD0006E202020004750532052616E6765202010
:100BE0002020202020004E6F2053442D436172644A
:100BF0002020202020200053442D4C6F6767696E11
:100C000067206572726F7200466C79696E67207238
:100C1000616E676521202020004D617820416C7451
:100C20006974756465212020200020202020202068
:100C300020202020202020202020202020202000D4
:100C400020202532692E25316956202000202025BC
:100C500032692E25316956202000414C543A253402
:100C6000696D20256300414C543A2534696D20207C
:100C700000414C543A2D2D2D2D2000202025326985
:100C80003A2530326920200020202532693A25306B
:100C900032692020004449523A20253364256300FC
:100CA0004300200020202535692020002020253504
:100CB00069202000493A2532692E253169412000FA
:100CC0003A003A003A002D2D2D2D2D2D2D2D2D2BB6
:100CD0002D2D2D2D2D2D2D2D2D2D2D002D2D2D2D71
:100CE0002D2D2D2D2D2D2D2D2D2D2D2D2D2D2D2D34
:100CF0002D003A005341543A2532642000444953B0
:100D0000543A2533646D004420003344002121000F
:100D10004D41473A25337525252000484D3A253366
:100D200064256320256300696E636C3A253264256F
:100D300063282532692900202020202532756D2F57
:100D4000733A2020484D3A253364256320256300FB
:100D50004552523A202532642021004552523A2011
:100D600000207777772E4D696B726F4B6F707465CB
:100D7000722E6465202000202532693A25303269C0
:100D800020202532692E25316956202534696D4190
:100D90006800202532693A253032692020253269E1
:100DA0002E25316956202534696D41680044495229
:100DB0003A253364256300414C543A2534696D006B
:100DC000414C543A2534696D00414C543A2D2D2D37
:100DD0002D2000256300484D3A25336425632020EB
:100DE000444953543A2533646D20256300505752CB
:100DF0003A2532692E253169412028256957292055
:100E0000004346002020004750533A2532756D2F8D
:100E100073205341543A256420002020334420009D
:100E20004E4F464958004447505320002020204E42
:100E30006F204E6176694374726C20202020202040
:100E400020002532692E2569202532692E2569204A
:100E50002532692E2569202532692E256941002514
:100E600033692025336920253369202533692563BB
:100E700043002532692E2569202532692E256941D6
:100E8000002532692E2569202532692E2569202505
:100E900032692E2569202532692E256941002533C6
:100EA000692025336925634320202020202020202D
:100EB00000253369202533692025336920253369CE
:100EC000256343004552523A2025326420210045D3
:100ED00052523A2000207777772E4D696B726F4B14
:100EE0006F707465722E6465202000536574746998
:100EF0006E673A257520257320004D696E3A2532BC
:100F0000692E253169562025732000414C543A0042
:100F1000504F54493A2533752000284F4E29202040
:100F200000284F46462920004C494D49540056415F
:100F300052494F0044495341424C45440043463ACC
:100F40000044495341424C45440020284F4E29203B
:100F50000020284F46462900205445414348004779
:100F600050533A0044495341424C454400284652AC
:100F70004545290028484F4D452900284149442925
:100F8000200028484F4C4429002046533A257573C9
:100F9000656B2000484F4D4520414C543A00257563
:100FA0006D00484F4C4420004E693A253469205268
:100FB0006F3A25346920433A2533690047733A254F
:100FC00034692059613A253469200050313A25347A
:100FD000692050323A25346920333A25336900506C
:100FE000343A2534692050353A25346920363A257B
:100FF000336900434F55504C494E47204F464621D8
:1010000020004C4F4F50494E472120004848212096
:1010100000434F4D50415353204F46462120000A74
:101020000D7777772E4D696B726F4B6F70746572A9
:101030002E64652028632920486953797374656D8F
:101040007320476D6248000A0D74686520757365EA
:10105000206F66207468697320736F66747761729D
:1010600065206973206F6E6C79207065726D69748C
:10107000746564200A0D6F6E206F726967696E6116
:101080006C204D696B726F4B6F707465722D486187
:10109000726477617265005573657200486F5454CD
:1010A000205633004143542044534C004A65746930
:1010B000005370656B7472756D0050504D000A0DD1
:1010C00052656365697665723A2000532E427573E6
:1010D00000756E6B6E6F776E2E205573696E67208C
:1010E00050504D2E2E2E006E6F7420737570706FE1
:1010F00072746564206279206861726477617265D8
:1011000021000A0D466C69676874436F6E74726FD4
:101110006C0A0D48617264776172653A25642E2508
:10112000640A0D536F6674776172653A5625642EB2
:1011300025642563200011241FBECFEFD0E4DEBF5D
:10114000CDBF11E0A0E0B1E0EEE9FFE101E00BBFAF
:1011500002C007900D92A63DB107D9F71AE0A6ED9F
:10116000B1E001C01D92A03AB107E1F77AEAE2E0EE
:10117000F0E081E280935700D4907E010894E11C56
:10118000F11C20EF37EF41E050E087016FE0DA011A
:10119000C9012F5F3F4F4F4F5F4FABBFFC0187919E
:1011A000F80181938F01615067FFF1CFF7016EE085
:1011B000819178277095615067FFFACF88897817F9
:1011C00029F0F7E9DF1611F40000FECF0E94BD09F7
:1011D0000C94CE8F0C94000088E791E09F938F933E
:1011E00080EF94E19F938F93E0914C04F0914D0434
:1011F00009950F900F900F900F900895809194068D
:10120000E82FFF27EE0FFF1FEA53F84F80819181EF
:101210008D5E9F4F14F010920301808191818A5B53
:101220009F4FCCF4809103018823A9F481E080933F
:101230000301809181048F5F80938104853038F0B1
:1012400088EE93E090930D0280930C0204C066E94F
:1012500070E00E94A139809181049927909319062A
:101260008093180608951F93CF93DF93182F882338
:1012700089F08EE991E09F938F9380EF94E19F93A3
:101280008F93E0914C04F0914D0409950F900F90CD
:101290000F900F908091B706823308F044C084EF1E
:1012A00091E00E94FF18EC01112329F0CE010E9469
:1012B00008198823D9F3C2E0D0E026E530E0809118
:1012C0002001909121018217930730F02196255D2E
:1012D0003F4FC730D10598F38091B7069927C89F33
:1012E0009001C99F300DD89F300D1124209300012B
:1012F0001123D9F068EC70E08C2F0E94A139DF93A4
:10130000CF9386EA91E09F938F9380EF94E19F9330
:101310008F93E0914C04F0914D0409958DB79EB7E1
:1013200006968DBF02C080930001112311F18091B8
:1013300000016AE00E94218F892F99279F938F9344
:10134000809100010E94218F99279F938F9381EBB9
:1013500091E09F938F9380EF94E19F938F93E0911F
:101360004C04F0914D0409952DB73EB7285F3F4FCF
:101370002DBFDF91CF911F910895CFEFD0E4DEBF55
:10138000CDBF8824992414B815B8B7EEEB2EB3E07E
:10139000FB2E2EEC3FEFE20EF31EF7FEFACF85E1B7
:1013A0008093020181E887B93E9A8FEF88B98BE17B
:1013B00084B911E015B98EE38AB987E48BB9469AEE
:1013C00084B7877F84BF80916000886180936000CC
:1013D0001092600084EC99E090930D0280930C02CF
:1013E00010921B0310921A031092CB071092CA0797
:1013F00010921D0310921C0310921F0310921E03E3
:1014000084EC94E0A0E0B0E0809345019093460125
:10141000A0934701B093480128980E9468190E9440
:1014200039190E94F8140E94BC350E946F1D812F4B
:101430000E941F310E942B6A0E94BB8B8091020187
:101440008C3010F4299A01C0299878940E943E307B
:101450000E94E27380915202826080935202109245
:1014600055020E94F54484EF91E00E94FF187C0130
:101470008091520280FD05C0C7010E94081988238F
:10148000B9F387EC91E09F938F93A0EFAA2EA4E18C
:10149000BA2EBF92AF92E0914C04F0914D040995A1
:1014A00080EA9FE00E94FF187C0100E010E00F90AE
:1014B0000F900F900F90C8E6D7E0FCE1CF2EF7E039
:1014C000DF2E0E94F5448091520280FD05C0C701C5
:1014D0000E9408198823B9F3F60180811816A4F434
:1014E0000BC00E94F5448091520280FD05C0C701E7
:1014F0000E9408198823B9F3C7010E94081988239C
:1015000019F4888188236CF7888187FF1BC00F5FDF
:101510001F4F1F930F930150104089ED91E09F934F
:101520008F93BF92AF92E0914C04F0914D040995D6
:101530008091D7018F5F8093D7012DB73EB72A5F87
:101540003F4F2DBF0F5F1F4F84E090E0C80ED91EA4
:1015500028960C30110508F4B4CF00E010E0C5E681
:10156000D7E0ECE1EE2EE7E0FE2E8B8187FD1FC079
:10157000F70180811816DCF40F5F1F4F1F930F9344
:10158000015010408CED91E09F938F9380EF94E198
:101590009F938F93E0914C04F0914D04099582E064
:1015A00080930A022DB73EB72A5F3F4F2DBF8B8134
:1015B00080788B830F5F1F4F84E090E0E80EF91E68
:1015C00028960C30110588F20E94EC089091920642
:1015D0008091D701981728F48091670480618093E7
:1015E00067048AEF91E09F938F93C0EFD4E1DF937C
:1015F000CF93E0914C04F0914D04099588EE93E06F
:101600000E94FF187C010E94751D0F900F900F9093
:101610000F90C7010E9408198823D9F381E192E055
:101620009F938F93DF93CF93E0914C04F0914D04FF
:10163000099580E00E94703A809102010F900F900E
:101640000F900F908A3011F0843110F0289801C06B
:10165000289A80ED97E090930D0280930C0285E527
:10166000809383048EE090E00E94622E9927182FC9
:1016700000278FE090E00E94622E080F111D10934A
:10168000DD010093DC018AE090E00E94622E992740
:10169000182F00278BE090E00E94622E080F111D8A
:1016A0001093DB010093DA010F5F1F4F39F0809137
:1016B000DC019091DD018F5F9F4F41F41092DD01BD
:1016C0001092DC011092DB011092DA018091DA01B4
:1016D0009091DB019F938F938091DC019091DD01CC
:1016E0009F938F9386E192E09F938F93DF93CF93A5
:1016F000E0914C04F0914D0409950E94EE2288E897
:1017000093E19093400180933F01C1E0C093820434
:101710008C2F0E9433098091BA060E94078B0E9489
:10172000EC0880ED97E00E94FF187C018AEF90E0C2
:101730000E94FF1883E08093F0051092D6018091FB
:1017400000072DB73EB7285F3F4F2DBF84FF02C073
:10175000C093DE0188E392E09F938F9380EF94E142
:101760009F938F93E0914C04F0914D0409950F9055
:101770000F900F900F908091E001882311F047980F
:10178000FECF80911002882309F436C280911201A5
:10179000882309F431C210921002809181048823B9
:1017A00019F00E94FE0802C00E9447480E94F544BA
:1017B000209102012A3011F0243110F0289801C044
:1017C000289A80910E03882331F080910E03815076
:1017D00080930E030EC080916F00806280936F0033
:1017E0001092C7071092C6078091670488608093A3
:1017F000670480913F0190914001019790934001CF
:1018000080933F0180913F0190914001892B21F00D
:10181000809153028823C9F180913F01909140014A
:10182000892BD9F40E94493185E090E090934001E2
:1018300080933F0180912A0690912B060196909308
:101840002B0680932A068091670481608093670449
:101850008091F10582608093F1058091080190915B
:1018600009018F5F9F4FC1F480910D038823A1F080
:1018700088EA91E690930D0280930C0280E890E054
:10188000909309018093080107C02A3011F0243198
:1018900010F0289801C0289A0E94738C8091100241
:1018A000882309F0A9C180912904882319F00E9496
:1018B0000582A2C180911001882311F00E947F1936
:1018C0000E943C150E948A10C7010E9408198823B3
:1018D00009F48EC184E190E0E80EF91E8091BA0609
:1018E000863011F40E94B37780915302882349F027
:1018F000809167048260809367048091F105826023
:101900000FC080910C0290910D02892B59F48091A7
:101910003F0190914001079728F08091F1058D7F5C
:101920008093F1058091DE01882361F080910E03A0
:10193000873940F01092DE0188E893E190930D0220
:1019400080930C0280910501882321F081508093BF
:1019500005012EC080938D041092E2021092E102E4
:101960001092E0021092DF021092DE021092DD026D
:1019700080910E038823E1F4809108019091090180
:101980008F5F9F4FA9F42091DE01223089F088E912
:101990009AE390930D0280930C0280E09CE0909378
:1019A000090180930801222319F082E08093DE016F
:1019B0008091CC01893C48F081508093CC0180918A
:1019C00067048B7F809367043FC08091B4088823AD
:1019D000F9F08091670484608093670489E08093C4
:1019E000F90380910801909109018F5F9F4F81F465
:1019F00080910D03882361F088E99AE390930D02AA
:101A000080930C0280E098EA90930901809308018A
:101A10001092EB031092EA031092E9031092E8038C
:101A20001092E7031092A7081092E6081092E508BA
:101A30001092E8081092E7088FEF9FEF9093E40868
:101A40008093E3081092CC0180910001282F332766
:101A5000809120019091210182179307CCF480910D
:101A6000D20280628093D202809108019091090194
:101A70008F5F9F4FC1F480E797E190930D028093B1
:101A80000C0280E093E090930901809308010BC061
:101A900080910C0290910D02892B29F48091D20241
:101AA0008F7D8093D2020E94ED6E84E080930B02C2
:101AB0008091DF018F5F8093DF01813309F04FC098
:101AC0001092DF018091D20281FF0AC08091D8017B
:101AD0009091D90101969093D9018093D8013FC08C
:101AE0005AEA852E55E0952E80913706909138065A
:101AF0009C01442737FD4095542F80911801909107
:101B00001901A0911A01B0911B01281739074A0742
:101B10005B0734F4809137069091380601961BC01C
:101B200080913706909138069C01442737FD4095F7
:101B3000542F8091180190911901A0911A01B09130
:101B40001B0182179307A407B5074CF48091370651
:101B50009091380601979093380680933706089441
:101B6000811C911C32E783163BE0930609F040C0CC
:101B7000882499242091DC013091DD012F5F3F4FB3
:101B80003093DD012093DC018091DA019091DB013B
:101B900001969093DB018093DA01832F9927682FB8
:101BA0008EE090E00E946A2E8091DC019091DD0130
:101BB0009070682F8FE090E00E946A2E8091DA0189
:101BC0009091DB01892F9927682F8AE090E00E948D
:101BD0006A2E8091DA019091DB019070682F8BE082
:101BE00090E00E946A2E84E190E00E94FF187C0140
:101BF0000E943D6F0E94F97380910B02882309F0C7
:101C0000BACD0E944C6AB7CD1F920F920FB60F92B9
:101C100011248F939F93EF93FF9380910701882363
:101C2000E1F48091FA019091FB0101969093FB0100
:101C30008093FA01FC01EF5BFA4FE081ED3019F07F
:101C40008F3A910539F41092FB011092FA0181E06C
:101C500080930701E093C60004C01092FB0110922C
:101C6000FA01FF91EF919F918F910F900FBE0F900E
:101C70001F9018951F920F920FB60F9211242F9359
:101C80003F934F935F936F937F938F939F93AF9304
:101C9000BF93CF93EF93FF9390E08091E001813069
:101CA00029F48091C6008093CE00CCC08091E001E1
:101CB000823029F48091C60080939004C3C0809143
:101CC000C6008093F201509100025F3A10F09093A9
:101CD00001028091F2018D3009F065C0809101020E
:101CE000823009F060C090930102852F99278057B8
:101CF0009B4FFC01329740812091FC013091FD0106
:101D0000241B3109DC0111978C91281B3109C90171
:101D10009F709093FD018093FC0146E09695879516
:101D20004A95E1F7982F935C9093FE012F733070E2
:101D3000235C2093FF018081981729F48C91281748
:101D400011F491E006C090E08091EF018F5F8093E5
:101D5000EF01C091F101CC2309F074C0992309F47B
:101D600071C081E08093F101580F5093EE01515002
:101D7000E52FFF27E057FB4F8DE080838091920491
:101D8000823509F05FC00E94EE2288E190E02CE0ED
:101D90000FB6F894A895809360000FBE2093600062
:101DA000C0930A024FC020910102822F99278130EF
:101DB0009105F9F0823091051CF4892B21F040C087
:101DC000029711F13DC08091F201833239F4809184
:101DD000F101882319F481E0809301028091F201DE
:101DE0008093900481E0809300028091F201992712
:101DF00022C02F5F20930102E52FFF27E057FB4F02
:101E00008091F201808309C0E52FFF27E057FB4F47
:101E10008091F20180835F3A20F45F5F509300026B
:101E200002C0109201022091F2018091FC01909178
:101E3000FD01820F911D9093FD018093FC0102C072
:101E400010920102FF91EF91CF91BF91AF919F91BD
:101E50008F917F916F915F914F913F912F910F9053
:101E60000FBE0F901F901895AC01A0E0B0E09D014F
:101E7000A817B90748F4E1E4F5E08191280F311D76
:101E80001196A417B507C8F33F70FD01EF5BFA4F39
:101E9000C90156E0969587955A95E1F7835C808352
:101EA0001196FD01EF5BFA4F2F733070822F835C28
:101EB0008083AE5BBA4F8DE08C93109207018091C6
:101EC00041058093C6000895A0E0B0E0EAE6FFE097
:101ED0000C949A8F2C859D850E85BB2483E280937C
:101EE00041059F59909342052093430533E0E32E2B
:101EF000F12C002309F49EC0CF84D888BE016D5E0A
:101F00007F4FA989BA890150109709F493C010979F
:101F1000B9F0F601EB0DF11DB3949081119791F496
:101F2000002349F1FB016E5F7F4FDB01C080D18050
:101F30006E5F7F4F0D90BC91A02DBB24015002C05D
:101F400090E019C01097B9F0F601EB0DF11DB394B4
:101F50004081119791F4002341F1FB016E5F7F4FA7
:101F6000DB01C080D1806E5F7F4F0D90BC91A02DB2
:101F7000BB24015002C040E018C01097B1F0F60138
:101F8000EB0DF11DB3941081119781F4002371F0D2
:101F9000FB013296DB01CD90DC90BF016E5F7F4F7D
:101FA000A081B181BB24015001C010E0F701EF5BBB
:101FB000FA4F892F86958695835C80830894E11C6F
:101FC000F11CF701EF5BFA4F892F9927837090700E
:101FD00024E0880F991F2A95E1F755279A0194E08C
:101FE000369527959A95E1F7822B835C8083089438
:101FF000E11CF11CF701EF5BFA4F4F705070440F7A
:10200000551F440F551F812F992726E096958795D8
:102010002A95E1F7842B835C80830894E11CF11CF2
:10202000F701EF5BFA4F1F73135C10830894E11CF8
:10203000F11C6ACFC7010E94340FE9E00C94B68FFF
:10204000A3E07A2F4091EE014650442309F458C092
:10205000E72FFF27E057FB4F80818D537F5FE72FEE
:10206000FF27E057FB4F20812D537F5FE72FFF278E
:10207000E057FB4F30813D537F5FE72FFF27E0574D
:10208000FB4F60816D537F5F9927880F991F880FE1
:10209000991F522F52955F70582B822F99278F705E
:1020A0009070F4E0880F991FFA95E1F7232F269599
:1020B0002695282B832F992783709070E6E0880F50
:1020C000991FEA95E1F7682B41504F3FC9F0EA2F7D
:1020D000FF27E057FB4F5083AF5F41504F3F81F0E8
:1020E000EA2FFF27E057FB4F2083AF5F41504F3F60
:1020F00039F0EA2FFF27E057FB4F6083AF5FA5CF92
:1021000083E994E09093ED018093EC01A350A093B8
:10211000EB010895A2E0B0E0E0E9F0E10C94A08FBB
:102120008091F101882309F457C40E942010809106
:102130009104823609F023C3809192049927803755
:10214000910509F4AFC081379105C4F48A36910531
:1021500009F480C28B36910544F48B34910571F1FA
:102160008636910509F45FC10AC38D36910509F4DD
:1021700069C08E36910509F44DC001C384379105BD
:1021800041F1853791054CF48137910509F491C0EF
:102190008337910509F4DFC0F2C28737910509F44E
:1021A0001BC2883791052CF48537910509F4D7C1F6
:1021B000E6C28937910509F46DC1E1C2E091EC01F5
:1021C000F091ED01808191819093B3018093B201F0
:1021D000D6C28091EE01A091EC01B091ED01853164
:1021E00040F080E1EBE6F4E00D9001928A95E1F792
:1021F0000DC08D919D910D90BC91A02D80936B048D
:1022000090936C04A0936D04B0936E0480EF809360
:10221000E9014BC0809107018823E1F38DE490E050
:102220009F938F938FE097E09F938F9381E08F939D
:102230008F938EE48F930E94640F8DB79EB707969D
:102240008DBF9DC2A091EC01B091ED011C911130A8
:1022500081F48DE4EFE0F7E00D9001928A95E1F7CB
:102260000E947B2F1983809167048F7E809367047F
:1022700001C01982809107018823E1F381E090E099
:102280009F938F93CE0101969F938F9381E08F93BD
:102290008F938DE48F930E94640FADB7BEB71796EE
:1022A000ADBF6DC281E08093F4018FEF8093050193
:1022B00066C2E091EC01F091ED01E0818E2F8A5031
:1022C0008A3058F48983882311F481E003C0863072
:1022D00010F085E0898361E00EC08E2F84518A3032
:1022E00070F48983882311F481E003C0863010F0F4
:1022F00085E0898360E089810E94FB2F12C0E98319
:10230000EF3F19F40E94DE2F89838981882311F41D
:1023100081E003C0863010F085E0898389810E94C6
:10232000802E809107018823E1F38BE790E09F9353
:102330008F9383E996E09F938F9381E090E09F9342
:102340008F93CE0101969F938F9382E08F9381E0CC
:102350008F9381E577C12091EC013091ED01D90196
:102360008C918150853008F045C0F90181818A3512
:1023700009F040C080910D038823E1F52F5F3F4FA6
:102380008BE7E3E9F6E0D9010D9001928A95E1F738
:10239000F90182910E94EB2E8091D4069927AA27F9
:1023A000BB27BC01CD0124EC39E040E050E00E94A5
:1023B000028FDC01CB018093AA019093AB01A09323
:1023C000AC01B093AD018091D5069927AA27BB2710
:1023D000BC01CD010E94028FDC01CB018093A601DC
:1023E0009093A701A093A801B093A9010E94DE2FAA
:1023F000898301C01982809107018823E1F381E07C
:1024000090E09F938F93CE0101969F938F9381E0ED
:102410008F938F9383E58F930E94640F8DB79EB740
:1024200007968DBF26C0E091EC01F091ED01E081AF
:102430008E2F8150853018F48E2F0E94802E0E949E
:10244000DE2F8983809107018823E1F381E090E00A
:102450009F938F93CE0101969F938F9381E08F93EB
:102460008F9386E48F930E94640FADB7BEB7179623
:10247000ADBF80910D03882329F46EE670E0898159
:102480000E94A13980E00E9433098091BA060E941F
:10249000078B75C1E091EC01F091ED0180819927E6
:1024A00087FD90959093E1078093E00781819927BC
:1024B00087FD90959093E3078093E20782819927A7
:1024C00087FD90959093E5078093E4078381992792
:1024D00087FD90959093E7078093E607848199277D
:1024E00087FD90959093E9078093E8078581992768
:1024F00087FD90959093EB078093EA078681992753
:1025000087FD90959093ED078093EC07878199273D
:1025100087FD90959093EF078093EE07808599272C
:1025200087FD90959093F1078093F0078185992717
:1025300087FD90959093F3078093F2078285992702
:1025400087FD90959093F5078093F40783859927ED
:1025500087FD90959093F7078093F60710C1E0915F
:10256000EC01F091ED0180810E9415358A8388236A
:1025700019F481E0898301C01982809107018823C1
:10258000E1F388E090E09F938F938DE597E09F9330
:102590008F9321E030E03F932F938091EC01909155
:1025A000ED019F938F933F932F93CE0102969F93BC
:1025B0008F933F932F93CE01820F931F9F938F93FF
:1025C00084E08F9381E08F9385E58F930E94640F61
:1025D000EDB7FEB773963CC08091EB01893008F4EB
:1025E000CEC02091EC013091ED012F5F3F4F88E08C
:1025F000ADE5B7E0F90101900D928A95E1F7D901B7
:102600008E910E946B348A83882319F481E0898338
:1026100001C01982809107018823E1F321E030E0B5
:102620003F932F93CE0102969F938F933F932F93C7
:10263000CE01820F931F9F938F9382E08F9381E04F
:102640008F9387E58F930E94640FEDB7FEB73B969B
:10265000EDBF95C080910D03882309F090C00E94C2
:10266000BA8A8983823019F0843009F088C020E466
:1026700030E0F8948091C1008F738093C100809105
:10268000C9008F738093C9008091C100877E8093B9
:10269000C1008091C900877E8093C9008091C800E5
:1026A00087FF03C08091CE00F9CF8091C00087FFE3
:1026B00003C08091C600F9CFE091EC01F091ED01EB
:1026C000E081E13021F482E08093E0012EC0E43625
:1026D00011F421E830E081E08093E001832F992715
:1026E0008093CD002093CC008091CD008093C500D5
:1026F0008091CC008093C4008091CA008F7D80932C
:10270000CA008091CA008F7E8093CA008091C90060
:102710008B7F8093C9008091CA0084608093CA0037
:102720008091CA0082608093CA008091CA00877F2E
:102730008093CA008091C200877F8093C2008091FD
:10274000C9008E7F8093C9008091C1008861809309
:10275000C1008091C90088618093C9008091C10047
:1027600080688093C1008091C90080688093C9000F
:1027700010926E0010926F00109270007894809109
:10278000920499278436910509F4BBC085369105DA
:10279000ACF48136910509F46FC0823691052CF4B2
:1027A0008B34910509F45DC00FC18236910509F49F
:1027B00070C08336910509F47FC006C18C3691053F
:1027C00009F4EDC08D3691054CF48736910509F476
:1027D000F8C08836910509F4B2C0F6C08437910577
:1027E00029F08637910509F4E8C0EEC08091EE012A
:1027F000A091EC01B091ED01803140F080E1EBE679
:10280000F4E00D9001928A95E1F70DC08D919D91B4
:102810000D90BC91A02D80936B0490936C04A093B9
:102820006D04B0936E04809107018823E1F31F9239
:10283000809104018F9384E58F930E94640F8AEF47
:102840008093E9018FEF8093050180EA9FE00E9469
:10285000FF189093E2018093E1010F900F900F9089
:10286000B3C0E091EC01F091ED01808191819093F2
:10287000B3018093B201A8C0E091EC01F091ED01A9
:10288000808180930601803298F08FE18093060169
:102890000FC0A091EC01B091ED018BE0E3E8F4E012
:1028A0000D9001928A95E1F780918C048093320615
:1028B0008FEF8093050188C08091E5019091E6013A
:1028C000892B89F4E091EC01F091ED01E081EE2398
:1028D00051F08AE0E89FC00111240E94FF189093F4
:1028E0005E0480935D04E091EC01F091ED01908134
:1028F0008AE0989FC00111249093E6018093E5013E
:1029000015C08FEF80930501E091EC01F091ED018E
:1029100090818AE0989FC00111249093E8018093F0
:10292000E701892B19F081E08093F60180EA9FE0AE
:102930000E94FF189093E2018093E10145C08FEF60
:1029400080930501E091EC01F091ED01908197FDFC
:1029500008C082E08093F3011092E4011092E30139
:102960001AC0909580914B02892B80934B029181E4
:102970008AE0989FC00111249093E4018093E301C1
:1029800084E08093F30180EA9FE00E94FF18909317
:10299000E2018093E10181E08093F70115C08FEFA0
:1029A00080930501E091EC01F091ED01808180932D
:1029B0004C0281E08093F80107C081E08093F5012B
:1029C00003C081E08093F9011092F1011092ED01B2
:1029D0001092EC011092EB01E3E0CE5F0C94BC8FFF
:1029E000982F8091C00085FFFCCF9093C60008957A
:1029F0000F931F9388E18093C1008091C000826093
:102A00008093C0008091C10080688093C100809154
:102A1000C10080648093C10000E010E00093C50015
:102A20008AE290E08093C4008091E7019091E801F0
:102A30000E94FF189093600480935F048CED90E0F7
:102A40000E94FF1890938F0480938E04109261046B
:102A500088E58093620484E0809365048BE0809332
:102A60006304109264041093ED010093EC01109242
:102A7000EB011F910F910895A0E1B0E0E2E4F5E1D0
:102A80000C949D8F80910701882309F4C1C2809125
:102A9000E1019091E2010E940819882361F01092EF
:102AA000E4011092E3011092E8011092E701109204
:102AB000E6011092E5018091E3019091E401892BF8
:102AC00041F080913F05909140050E9408198823AC
:102AD00029F48091F701882309F460C080910701EF
:102AE000882309F45BC08091F30102E416E084308E
:102AF000A8F00E94042380E590E09F938F931F939A
:102B00000F9381E08F938F9388E48F930E94640FDB
:102B10002DB73EB7295F3F4F2DBF34C010924D02F5
:102B200080E694E09F938F9387EF92E29F938F9339
:102B3000E0914C04F0914D04099584E190E09F935D
:102B40008F931F930F9381E090E09F938F9383EF78
:102B500091E09F938F9382E08F9381E08F9388E43D
:102B60008F930E94640F8091F301982F8F5F809361
:102B7000F3012DB73EB7215F3F4F2DBF943010F0CA
:102B80001092F3018091E3019091E4010E94FF18FB
:102B90009093400580933F051092F7018091F801D2
:102BA000882351F180910701882331F10E94042389
:102BB00080E590E09F938F9382E496E09F938F93BC
:102BC00021E030E03F932F9382E291E09F938F9337
:102BD0003F932F938CE492E09F938F9383E08F93A6
:102BE00081E08F938CE48F930E94640F1092F80120
:102BF0008DB79EB70F968DBF8091F5018823D1F0D8
:102C0000809107018823B1F08AE090E09F938F9331
:102C100081E694E09F938F9381E08F938F9386E575
:102C20008F930E94640F1092F5012DB73EB7295F74
:102C30003F4F2DBF8091F9018823D9F08091070182
:102C40008823B9F08BE090E09F938F9383E894E022
:102C50009F938F9381E08F93809104018F9387E4FA
:102C60008F930E94640F1092F9018DB79EB707965B
:102C70008DBF80918E0490918F040E940819882343
:102C800009F461C080910701882309F45CC0809138
:102C9000AF069927880F991F880F991F7C0100277D
:102CA000F7FC0095102F8091640390916503A0912B
:102CB0006603B0916703BC01CD01A80197010E9492
:102CC000768F30937C0420937B0480915C039091F9
:102CD0005D03A0915E03B0915F03BC01CD01A8012B
:102CE00097010E94768F30937E0420937D0480911B
:102CF000EB0280937F048091EA028093800488E055
:102D000090E09F938F938BE794E09F938F9381E064
:102D10008F9383E08F938BE68F930E94640F809153
:102D200081042DB73EB7295F3F4F2DBF853018F086
:102D300086E08093810483E690E00E94FF189093E0
:102D40008F0480938E048091E7019091E801892B94
:102D500041F080915F04909160040E9408198823DB
:102D600021F48091F601882339F1809107018823AD
:102D700019F10E94693882E490E09F938F9380EF6D
:102D800095E09F938F9381E08F938F9384E48F934B
:102D90000E94640F1092F6018DB79EB707968DBF03
:102DA0008091E7019091E801009731F00E94FF18AF
:102DB0009093600480935F048091E5019091E60117
:102DC000892B09F4B8C080915D0490915E040E9443
:102DD0000819882309F4AFC080910701882309F4FA
:102DE000AAC08091AF069927880F991F880F991F55
:102DF0007C010027F7FC0095102F809164039091CF
:102E00006503A0916603B0916703BC01CD01A801E1
:102E100097010E94768F3093500420934F04809145
:102E20005C0390915D03A0915E03B0915F03BC01D0
:102E3000CD01A80197010E94768F30935204209310
:102E40005104209193083091940840919508509135
:102E50009608DA01C90163E0880F991FAA1FBB1FFA
:102E60006A95D1F7820F931FA41FB51F820F931F7E
:102E7000A41FB51F209145013091460140914701A3
:102E800050914801BC01CD010E94768F30935404CB
:102E9000209353048091300390913103A091320329
:102EA000B091330349E0B595A795979587954A95D5
:102EB000D1F78093550480912C0390912D03A0911C
:102EC0002E03B0912F0339E0B595A7959795879577
:102ED0003A95D1F78093560480913403909135034D
:102EE000A0913603B091370329E0B595A795979542
:102EF00087952A95D1F7809357048EE090E09F93B1
:102F00008F938FE494E09F938F9381E08F938F93BF
:102F100083E48F930E94640F8091E5019091E60114
:102F20000E94FF1890935E0480935D042DB73EB716
:102F3000295F3F4F2DBF809106018F3F71F1992787
:102F400004E0880F991F0A95E1F7805A9D4F40E1F0
:102F500050E0BC01CE0101960E94558D80E190E0C9
:102F60009F938F93CE0101969F938F9381E090E082
:102F70009F938F9386E091E09F938F9382E08F934E
:102F800081E08F9381E48F930E94640F8FEF809391
:102F900006018DB79EB70B968DBF809132068823B0
:102FA000D1F0809107018823B1F081E090E09F93F8
:102FB0008F9382E396E09F938F9381E08F938F931B
:102FC00082E48F930E94640F109232062DB73EB7B1
:102FD000295F3F4F2DBF8091F4018823C9F0809174
:102FE00007018823A9F084E390E09F938F9386ECF8
:102FF00097E09F938F9381E08F938F9380E58F93DA
:103000000E94640F1092F4018DB79EB707968DBF92
:10301000E6E0C05F0C94B98F1F920F920FB60F922B
:1030200011242F933F935F936F937F938F939F937D
:10303000AF93BF93EF93FF9320E080910B0288231F
:1030400029F080910B02815080930B0280910C0437
:10305000882319F0815080930C04809113028150D1
:10306000809313028F3F09F05BC089E080931302C5
:103070008091110290911202019690931202809316
:103080001102809111018F5F81708093110188235B
:1030900019F481E080931002349903C081E0809399
:1030A000140280910C0290910D02892B21F18091E4
:1030B0000C0290910D020B9750F080910C029091B0
:1030C0000D020A9790930D0280930C0204C0109297
:1030D0000D0210920C0280910C0290910D02209131
:1030E00008013091090182239323892B11F021E0FB
:1030F00008C020E006C08FEF9FEF909309018093F6
:10310000080180910201222331F08A3011F45A9A89
:1031100007C0479A05C08A3011F45A9801C04798F1
:1031200080911402882309F45AC02091CC012223F3
:1031300009F055C08091820883FF51C086B199275C
:10314000FC01E071F07084FF13C080910E02909139
:103150000F02019690930F0280930E0280910E024F
:1031600090910F02895E9340D0F12093140237C0F2
:1031700080910E0290910F02892B69F180910E02CD
:1031800090910F028A56914030F580910E029091F5
:103190000F0269E270E00E942D8F80910E029091E3
:1031A0000F02860F971F90930F0280930E0280915B
:1031B0000E0290910F020B9750F080910E029091A9
:1031C0000F020A979093B3018093B20104C0F09369
:1031D000B301E093B20110920F0210920E02FF9120
:1031E000EF91BF91AF919F918F917F916F915F917F
:1031F0003F912F910F900FBE0F901F901895209127
:10320000110230911202280F391FC9010196089549
:103210002091110230911202821B930B892F992762
:103220008695807490700895CF93DF930E94FF1865
:10323000EC01CE010E9408198823D9F3DF91CF91C8
:103240000895CF93DF930E94FF18EC0109C080918D
:103250001201882329F0909312018FEC80937A0059
:10326000CE010E940819982F882389F3DF91CF910E
:1032700008959FB7F8945F983E9A469A8091B0005F
:103280008F708093B0008091B00083608093B00015
:103290008091B1008B738093B1008091B1008B60FD
:1032A0008093B1001092B2008FEF8093B3008091B1
:1032B000B00080688093B000809170008A7F809316
:1032C0007000809170008260809370009FBF0895AD
:1032D0008AE090E00E94FF1890931A0280931902EE
:1032E00082E085BD83EA84BD17BC84EB88BD86E09F
:1032F00086BD80916E00816080936E000895A0E08D
:10330000B0E0E5E8F9E10C94978FEE24FF24870103
:10331000570168014091CA0680903408282D332750
:103320002D5730408091E40299278D579040289F77
:10333000B001299F700D389F700D1124CB0168ECEE
:1033400070E00E94418F640F711D77FF0DC020E374
:1033500030E088279927861B970BB9010E94418F7F
:10336000B901681B790B06C0CB0160E370E00E94D5
:10337000418FBC01DB01A55BBE4FFD018485282F79
:10338000332727FD3095220F331F40918008842F6B
:10339000992787FD9095281B390B2F5F3F4F37FFEB
:1033A00002C02F5F3F4F35952795420F409380080D
:1033B0008C91282F332727FD3095220F331F6091E2
:1033C0006708862F992787FD9095281B390B2F5F5B
:1033D0003F4F37FF02C02F5F3F4F35952795962E01
:1033E000920E90926708809110019091E5028130D1
:1033F00009F01CC1923308F05BC0842F992787FD28
:103400009095A92FB92F20916403309165034091C5
:10341000660350916703BC01CD010E94028F97FFA4
:1034200004C061507E4F8F4F9F4F7B018C01F9E0AC
:1034300015950795F794E794FA95D1F7892D992773
:1034400087FD9095A92FB92F20915C0330915D03E2
:1034500040915E0350915F03BC01CD010E94028F39
:1034600097FF04C061507E4F8F4F9F4FE9E09595C5
:10347000879577956795EA95D1F757016801A61A60
:10348000B70AC80AD90A8091F2039091F3039C010C
:1034900063E0220F331F6A95E1F7281B390BC9013E
:1034A000AA2797FDA095BA2FA81AB90ACA0ADB0A5B
:1034B0008091C1069927AA27BB27BC01CD01A6018F
:1034C00095010E94028F97FF04C061507E4F8F4F7D
:1034D0009F4F5B016C0159E0D594C794B794A794B2
:1034E0005A95D1F780918F01992746E0880F991F4F
:1034F0004A95E1F740910E0150910F012091C906C4
:103500003327841B950BB9010E94418F80910E01D6
:1035100090910F01860F971F90930F0180930E01DA
:103520008091FF0680FF14C080910E0190910F01E1
:1035300097FD0F9634E0959587953A95E1F7AA2780
:1035400097FDA095BA2FA80EB91ECA1EDB1E15C086
:1035500080910E0190910F0197FD0F9624E09595B3
:1035600087952A95E1F7AA2797FDA095BA2F8A1982
:103570009B09AC09BD095C016D012091FC06222369
:1035800021F133278091060290910702829FA001CA
:10359000839F500D929F500D1124CA01AA2797FDB9
:1035A000A095BA2F8A0D9B1DAC1DBD1D2F5F3F4FEF
:1035B000442737FD4095542FBC01CD010E94768FE2
:1035C000309307022093060204C0B0920702A09233
:1035D00006028091C206282F3327220F331F220FA5
:1035E000331F8091060290910702821793077CF0A7
:1035F0008091C306282F3327220F331F220F331F3A
:1036000080910602909107022817390724F430931D
:1036100007022093060280910201843108F42EC132
:10362000809110018F5F809310012AC1943608F0B9
:1036300046C0842F992787FD9095A92FB92F2091F7
:103640005C0330915D0340915E0350915F03BC01C8
:10365000CD010E94028F97FF04C061507E4F8F4FB3
:103660009F4F5B016C01C9E0D594C794B794A794B0
:10367000CA95D1F7892D992787FD9095A92FB92F44
:103680002091640330916503409166035091670374
:10369000BC01CD010E94028F97FF04C061507E4F94
:1036A0008F4F9F4F7B018C01B9E015950795F794DB
:1036B000E794BA95D1F7EA0CFB1C0C1D1D1D8091F7
:1036C000C5069927AA27BB27BC01CD01A8019701F0
:1036D0000E94028F97FF04C061507E4F8F4F9F4F13
:1036E0007B018C01A9E015950795F794E794AA95BD
:1036F000D1F780918E019927F6E0880F991FFA95EE
:10370000E1F740910C0150910D01C091C9062C2F99
:103710003327841B950BB9010E94418F80910C01C6
:1037200090910D01860F971F90930D0180930C01CE
:103730008091FF0681FF14C080910C0190910D01D2
:1037400097FD0F96E4E095958795EA95E1F7AA270E
:1037500097FDA095BA2FE80EF91E0A1F1B1F15C072
:1037600080910C0190910D0197FD0F9674E0959555
:1037700087957A95E1F7AA2797FDA095BA2F8E191C
:103780009F09A00BB10B7C018D012091FD06222326
:1037900021F133278091040290910502829FB001AC
:1037A000839F700D929F700D1124CB01AA2797FD66
:1037B000A095BA2F8E0D9F1DA01FB11F2F5F3F4FE9
:1037C000442737FD4095542FBC01CD010E94768FD0
:1037D000309305022093040204C0F0920502E092A7
:1037E00004028091C606282F3327220F331F220F91
:1037F000331F8091040290910502821793077CF099
:103800008091C706282F3327220F331F220F331F23
:1038100080910402909105022817390724F430930F
:10382000050220930402882D992746E0880F991FEE
:103830004A95E1F720910A0130910B014C2F552751
:10384000821B930BBA010E94418F80910A019091D3
:103850000B01860F971F90930B0180930A018091B3
:103860000A0190910B0197FD0F9634E0959587958D
:103870003A95E1F7909303028093020210921001AF
:10388000ECE0CDB7DEB70C94B38F1F920F920FB65A
:103890000F9211242F933F934F935F938F939F9396
:1038A000EF93FF9380910201843108F4D7C0809197
:1038B0001502882309F0D2C08091B00086FF99C01C
:1038C0008091B0008F7B8093B000E0911802EE23CE
:1038D000F1F48091C806282F33278DED96E0289FBC
:1038E000A001299F500D389F500D1124CA0120912D
:1038F000160230911702821B930B9093090280935A
:1039000008021092170210921602469AA4C089EA81
:1039100093E090930902809308028E2F99278330B9
:103920009105D9F08430910534F48130910549F046
:10393000029761F022C08430910591F00597A9F0BB
:103940001CC0809106029091070204C0809104027D
:103950009091050287559E4F1FC080915C0807C05B
:103960008091020290910302F5CF8091650899271A
:10397000880F991F880F991FEDCFFF27EE0FFF1FAC
:10398000EA53F84F20813181220F331F80910802C2
:1039900090910902820F931F90930902809308026D
:1039A000809108029091090255E08D3D950718F02D
:1039B0008CED95E005C08757914030F487E791E0A2
:1039C0009093090280930802209108023091090225
:1039D0002C5B30403093090220930802809116023C
:1039E00090911702820F931F9093170280931602F3
:1039F00032C08091B00080648093B0008CEB90E086
:103A00009093090280930802809116029091170208
:103A100084549F4F909317028093160280910A025C
:103A2000882321F080910E03882321F480910A02DB
:103A3000823011F4469801C0469A809118028F5F37
:103A4000809318029091C806981728F481E080931B
:103A500010011092180281E0809315022091080253
:103A60003091090241E02F37340730F08FEF809317
:103A7000B3002F5F30400FC02F3F3105C9F0C0F0B9
:103A8000A9014F5F50404F37510550F480E88093B3
:103A9000B30020583040309309022093080212C02E
:103AA0008FEF8093B30050930902409308020AC03D
:103AB000809108028093B3001092090210920802CC
:103AC00010921502FF91EF919F918F915F914F910D
:103AD0003F912F910F900FBE0F901F90189510924D
:103AE0007C008FEC80937A000895CF93DF9310923F
:103AF0001F0286E987BD83E090E00E94622EC82FF6
:103B0000863E08F4C65FC8BD84E690E00E94211995
:103B100080911601909117018152934010F0C0EFEF
:103B200002C0C530F8F0C8BD82E390E00E942119C0
:103B300085E794E09F938F9380EF94E19F938F9319
:103B4000E0914C04F0914D040995809116019091FB
:103B500017010F900F900F900F908152934010F427
:103B6000C550DFCF6C2F83E090E00E946A2ECF30EB
:103B700018F0CCE8D0E002C0C0E0D0E0CA3FD105E8
:103B8000F8F4C7BD82E390E00E94211987E794E032
:103B90009F938F9380EF94E19F938F93E0914C04D8
:103BA000F0914D04099580911601909117010F90A5
:103BB0000F900F900F908052934010F02196DECF1F
:103BC000C0933F068091A00680FF09C08C2F8A50C9
:103BD0008B3E28F080916604806480936604C7BDA4
:103BE0008CE291E00E942119DF91CF910895EF922C
:103BF000FF921F93CF9310E080ED97E00E94FF1893
:103C00007C01CCE8133019F4CB3008F0C9E010E0A7
:103C100080912E0290912F028C5F934024F480912A
:103C2000150181500AC080912E0290912F02875079
:103C3000944034F0809115018F5F8093150101C08D
:103C400011E080912C0290912D028C5F934024F41E
:103C50008091140181500AC080912C0290912D0214
:103C60008750944034F0809114018F5F8093140149
:103C700001C01F5F80912A0290912B028C5F9340BC
:103C800024F48091130181500AC080912A029091FE
:103C90002B0287509440C4F0809113018F5F809372
:103CA000130113C089E794E09F938F9380EF94E111
:103CB0009F938F93E0914C04F0914D0409950F90E0
:103CC0000F900F900F905FC01F5F82E180935802AA
:103CD000809152028E7F8093520285EA8093BC00CD
:103CE000809115018A3040F4809166048160809350
:103CF00066048AE08093150180911501863F40F0AB
:103D00008091660481608093660485EF809315013D
:103D1000809114018A3040F480916604826080931F
:103D200066048AE08093140180911401863F40F07C
:103D30008091660482608093660485EF809314010D
:103D4000809113018A3040F48091660484608093EE
:103D500066048AE08093130180911301863F40F04E
:103D60008091660484608093660485EF80931301DC
:103D700080915802882339F0C7010E9408198823CE
:103D800009F090CFF5CF109212018FEC80937A005A
:103D9000809112018823E1F3CA3020F48AE090E098
:103DA0000E942119C15009F02DCF86E490E00E94B5
:103DB0002119CF911F91FF90EF9008951F920F92BC
:103DC0000FB60F921124EF92FF920F931F932F9330
:103DD0003F934F935F936F937F938F939F93AF9393
:103DE000BF93EF93FF9380913702282F3327442707
:103DF00055278F5F80933702F9012231310508F092
:103E0000C8C3EA5BFF4F0C94C88F809178009091F3
:103E1000790046C08091780090917900F9C0809136
:103E2000780090917900909339028093380224C1F0
:103E300080916D0390916E0320917800309179000C
:103E4000821B930B90933406809333068091330644
:103E50009091340690934302809342022BC180914B
:103E600078009091790020916F0330917003821B4C
:103E7000930B90933E0680933D0680913D06909172
:103E80003E06909345028093440285C380913C0294
:103E900090913D022091780030917900820F931F1C
:103EA00090933D0280933C0281E076C380913A0278
:103EB00090913B022091780030917900820F931FFE
:103EC00090933B0280933A0284E066C3809100079E
:103ED00083FF1AC080912001909121019C01220F43
:103EE000331F280F391F40917800509179008BE0E3
:103EF00090E0489FB001499F700D589F700D1124AC
:103F0000CB016EE170E00FC0809120019091210102
:103F10009C01220F331F280F391F80917800909148
:103F2000790063E070E00E942D8F260F371F3695D1
:103F3000279536952795309321012093200185E020
:103F40002BC3809178009091790020916903309182
:103F50006A03821B930B9093250280932402809125
:103F60007800909179009093360680933506809181
:103F70002402909125029C01442737FD4095542F3F
:103F80008091280390912903A0912A03B0912B03DB
:103F9000820F931FA41FB51F8093280390932903BA
:103FA000A0932A03B0932B03209128033091290377
:103FB00040912A0350912B0357FF04C021503C4FDE
:103FC0004F4F5F4F7AE055954795379527957A95EE
:103FD000D1F78091280390912903A0912A03B091F1
:103FE0002B03821B930BA40BB50B80932803909398
:103FF0002903A0932A03B0932B0348C180913A026E
:1040000090913B022091780030917900820F931FAC
:1040100090933B0280933A0210923602BFC2809185
:1040200002018A3071F4809178009091790020919A
:10403000380230913902820F931F01969695879529
:1040400017C04091380250913902843158F02091C4
:10405000780030917900240F351F8FEF97E0821B95
:10406000930B06C08091780090917900840F951F82
:1040700090932B0280932A0286E08EC280916D037A
:1040800090916E032091780030917900821B930B00
:1040900090933406809333068091330690913406D2
:1040A0002091420230914302820F931F9093290284
:1040B0008093280287E070C2809178009091790007
:1040C00020916F0330917003821B930B90933E06F7
:1040D00080933D0680913D0690913E0620914402DA
:1040E00030914502820F931F9093270280932602FE
:1040F00052C220913C0230913D0280917800909113
:104100007900280F391F30933D0220933C028091A3
:1041100002018A3019F4220F331F04C0220F331F0B
:10412000220F331F30933D0220933C0220913C022A
:1041300030913D02C90137FD079643E0959587957B
:104140004A95E1F790932F0280932E0280913E02D0
:1041500090913F02820F931F97FD01969595879549
:1041600090933F0280933E022091790330917A032D
:10417000821B930B9C012C5F3F4F37FF03C09C01B8
:10418000255F3F4F83E0359527958A95E1F730937A
:104190001F0120931E01209134023091350280913D
:1041A0001E0190911F01280F391F37FF02C02F5F9A
:1041B0003F4F35952795309335022093340274CEC6
:1041C00020913A0230913B028091780090917900E1
:1041D000280F391F30933B0220933A02809102014D
:1041E0008A3019F4220F331F04C0220F331F220F0D
:1041F000331F30933B0220933A0220913A023091D0
:104200003B02C90137FD0796B3E095958795BA95AE
:10421000E1F790932D0280932C02809140029091BF
:104220004102820F931F97FD019695958795909374
:104230004102809340022091770330917803821BE2
:10424000930B9C012C5F3F4F37FF03C09C01255F00
:104250003F4FF3E035952795FA95E1F730931D012F
:1042600020931C01209132023091330280911C0175
:1042700090911D01280F391F37FF02C02F5F3F4F5C
:1042800035952795309333022093320283E084C121
:104290001092370281E08093120180911B0290916D
:1042A0001C02019690931C0280931B028091E802ED
:1042B000282F33278091240290912502289FA00166
:1042C000299F500D389F500D11249A0157FF02C0AD
:1042D00021503F4F232F330F330B80917800909163
:1042E0007900820F931F909317018093160180919C
:1042F000160190911701AA27BB2720914602309101
:1043000047024091480250914902280F391F4A1F25
:104310005B1F20934602309347024093480250931C
:10432000490280914A028F5F80934A02803108F4EB
:1043300032C18091180190911901A0911A01B09198
:104340001B017C018D0163E0EE0CFF1C001F111F9F
:104350006A95D1F7E81AF90A0A0B1B0BE20EF31E55
:10436000041F151F80911F02992787FD9095A92F83
:10437000B92FBC01CD0120EB30E240E050E00E94BB
:10438000028FDC01CB01E81AF90A0A0B1B0BD801DA
:10439000C7010496A11DB11DB7FF05C0D801C70113
:1043A0000B96A11DB11D23E0B595A795979587950F
:1043B0002A95D1F78093180190931901A0931A01BF
:1043C000B0931B0180913706909138067C0100273D
:1043D000F7FC0095102F8091180190911901A09180
:1043E0001A01B0911B01E81AF90A0A0B1B0BE092A3
:1043F0000803F092090300930A0310930B03209122
:10440000200230912102409122025091230257FF55
:1044100004C0215F3F4F4F4F5F4F84E05595479554
:10442000379527958A95D1F78091200290912102A6
:10443000A0912202B0912302821B930BA40BB50B17
:104440008093200290932102A0932202B093230232
:104450008091200290912102A0912202B09123022A
:104460008E0D9F1DA01FB11F8093200290932102EB
:10447000A0932202B0932302809120029091210206
:10448000A0912202B0912302B7FF03C00F96A11D95
:10449000B11D14E0B595A795979587951A95D1F715
:1044A0002091080330910903281B390B54E0213077
:1044B00035071CF020E034E006C06CEF20303607F2
:1044C00014F420E03CEF80911D0290911E02809137
:1044D0001D0290911E0297FF03C0909581959F4FFA
:1044E000A901F3E0440F551FFA95E1F78D5B924067
:1044F000C4F080911D0290911E029C01E4E0220F05
:10450000331FEA95E1F7281B390B240F351F37FFBE
:1045100002C0215F3F4F74E0359527957A95E1F70A
:1045200017C080911D0290911E029C0165E0220F30
:10453000331F6A95E1F7281B390B240F351F37FF0E
:1045400002C0215E3F4F45E0359527954A95E1F73A
:1045500030931E0220931D028091460290914702E3
:10456000A0914802B0914902B7FF03C00196A11D76
:10457000B11DB595A7959795879580934602909321
:104580004702A0934802B093490288E080934A0210
:1045900002C01092370282E0809336028091360288
:1045A00080937C0080913702882319F08FEC8093F0
:1045B0007A00FF91EF91BF91AF919F918F917F9181
:1045C0006F915F914F913F912F911F910F91FF90AC
:1045D000EF900F900FBE0F901F90189590E2E2E4BD
:1045E000F6E08FE49193815087FFFCCF089590917E
:1045F0004D02903540F4E92FFF27EE5BF94F8083A1
:104600009F5F90934D020895AF92BF92CF92DF9239
:10461000FF920F931F93CF93DF9320914B0220FFC4
:104620000AC080914C02882311F0815002C0809111
:10463000220180934C0221FF0CC090914C0280918A
:104640002201981719F410924C0203C09F5F9093B7
:104650004C02822F992780FF04C081FF02C0109274
:104660004C020E94EE2280914C02282F332797EFB4
:10467000C92E92E2D92EC0914C04D0914D048A30BB
:1046800098F481E180934D023F932F9380EB94E067
:104690009F938F93DF92CF92FE0109952DB73EB77E
:1046A0002A5F3F4F2DBF11C080E180934D023F93A1
:1046B0002F9385EB94E09F938F93DF92CF92FE012F
:1046C00009958DB79EB706968DBF20914C02822F1B
:1046D0009927AA27BB27FC01419710F00C945C2C6A
:1046E000E85AFF4F07EFC02E02E2D02EC0914C04D3
:1046F000D0914D040C94C88F10924D028AEB94E037
:104700009F938F9307EF12E2DF92CF92FE010995FC
:1047100084E180934D020F900F900F900F9085E6EB
:1047200090E09F938F9388E590E09F938F931F92E3
:104730001F92809102016AE00E94218F892F9927A0
:104740009F938F93809102010E94218F99279F93BD
:104750008F938AEC94E09F938F93DF92CF92E091B6
:104760004C04F0914D04099588E280934D02EDB719
:10477000FEB73E96EDBF80E197E09F938F930E9436
:10478000DE2F99279F938F938FED94E09F938F93C4
:10479000DF92CF92E0914C04F0914D040995809105
:1047A000670499272DB73EB7285F3F4F2DBFEC0117
:1047B000C071D07084FF06C08CE380934D028DEEF3
:1047C00094E0F1C09091F903992349F18CE380932F
:1047D0004D02892F99279F938F938AEF94E09F939F
:1047E0008F931F930F93E0914C04F0914D04099522
:1047F000DF93CF939091F90381E1989FC001112439
:10480000845D954F9F938F931F930F93E0914C047A
:10481000F0914D0409958DB79EB70C9647C19091C4
:1048200066049923B1F08CE380934D02892F992778
:104830009F938F9382E095E09F938F931F930F93A5
:10484000E0914C04F0914D040995EDB7FEB7369612
:1048500079C490915302992371F08CE380934D02B7
:10486000892F99279F938F9389E195E09F938F9349
:104870001F930F93D9C480913F01909140010697F7
:1048800010F00C94652C8CE380934D028EE295E041
:10489000A5C78091820817EFC12E12E2D12EC091D8
:1048A0004C04D0914D0480FF6BC010924D0280915A
:1048B000080390910903A0910A03B0910B03BC0176
:1048C000CD0125E030E040E050E00E94768F3F933C
:1048D0002F938BE395E09F938F93DF92CF92FE010E
:1048E000099584E180934D028DB79EB706968DBFE2
:1048F0008091040390910503A0910603B0910703F2
:10490000BC01CD0125E030E040E050E00E94768F10
:104910003F932F9388E495E09F938F93DF92CF92FC
:10492000E0914C04F0914D04099588E280934D028A
:10493000EDB7FEB73696EDBF809116019091170145
:104940009F938F9385E595E09F938F93DF92CF920E
:10495000E0914C04F0914D0409958CE380934D0255
:104960002DB73EB72A5F3F4F2DBF87B599279F933D
:104970008F9382E695E09F938F93DF92CF928EC0C4
:1049800010924D028FE695E09F938F93DF92CF9226
:10499000FE01099584E180934D020F900F900F90D6
:1049A0000F908EE795E09F938F93DF92CF921AC777
:1049B00010924D0287E895E09F938F9307EF12E2E4
:1049C000DF92CF92FE01099584E180934D020F9012
:1049D0000F900F900F908091640390916503A091C8
:1049E0006603B0916703B7FF04C081509C4FAF4F7F
:1049F000BF4FCAE0B595A79597958795CA95D1F70A
:104A0000BF93AF939F938F9384E995E09F938F9388
:104A10001F930F93E0914C04F0914D04099588E2A7
:104A200080934D02EDB7FEB73896EDBF80915C03E1
:104A300090915D03A0915E03B0915F03B7FF04C046
:104A400081509C4FAF4FBF4FFAE0B595A795979512
:104A50008795FA95D1F7BF93AF939F938F9383EA8E
:104A600095E09F938F931F930F93E0914C04F091E7
:104A70004D0409958CE380934D022DB73EB7285F16
:104A80003F4F2DBF80913D0890913E089F938F939B
:104A900082EB95E09F938F931F930F93E0914C04CB
:104AA000F0914D0409958DB79EB706968DBF0DC741
:104AB000E1E0FE2EC1E0D0E008EC17E09F2D9695D6
:104AC00084E1989FC001112480934D02F8018281F6
:104AD00093819F938F932196DF93CF93219780812A
:104AE00091819F938F93DF93CF9381EC95E09F9378
:104AF0008F9387EF92E29F938F93E0914C04F09114
:104B00004D0409952DB73EB7245F3F4F2DBF32E0CE
:104B1000F30E22960C5F1F4F88E08F1578F6D5C6EE
:104B200010924D0280919506E82FFF27EE0FFF1F90
:104B3000EA53F84F808191819F938F9380919406DF
:104B4000E82FFF27EE0FFF1FEA53F84F8081918176
:104B50009F938F9383ED95E09F938F93DF92CF92F6
:104B6000FE01099584E180934D02EDB7FEB73896BA
:104B7000EDBF80919706E82FFF27EE0FFF1FEA5346
:104B8000F84F808191819F938F9380919606E82FB3
:104B9000FF27EE0FFF1FEA53F84F80819181815864
:104BA0009F4F9F938F9383EE95E09F938F93DF9218
:104BB000CF92E0914C04F0914D04099588E28093E6
:104BC0004D022DB73EB7285F3F4F2DBF809199060C
:104BD000E82FFF27EE0FFF1FEA53F84F80819181E6
:104BE00081589F4F9F938F9380919806E82FFF27BE
:104BF000EE0FFF1FEA53F84F8081918181589F4F3C
:104C00009F938F9383EF95E09F938F93DF92CF9243
:104C1000E0914C04F0914D0409958CE380934D0292
:104C20008DB79EB708968DBF80919B06E82FFF2712
:104C3000EE0FFF1FEA53F84F8081918181589F4FFB
:104C40009F938F9380919A06E82FFF27EE0FFF1F07
:104C5000EA53F84F8081918181589F4F9F938F93A2
:104C600083E096E063C210924D0283E196E09F9349
:104C70008F9307EF12E2DF92CF92FE0109958091A8
:104C800002010F900F900F900F908A3009F09DC095
:104C900084E180934D028091790390917A039C0185
:104CA00097FF02C0295F3F4F287F821B930B9F9382
:104CB0008F938091790390917A0397FD079673E023
:104CC000959587957A95E1F79F938F932091790336
:104CD00030917A0337FF02C0295F3F4F63E035957B
:104CE00027956A95E1F780912E0290912F02821B01
:104CF000930B9F938F9381E296E09F938F931F93E3
:104D00000F93E0914C04F0914D04099588E2809353
:104D10004D022DB73EB7265F3F4F2DBF80917703E1
:104D2000909178039C0197FF02C0295F3F4F287F35
:104D3000821B930B9F938F938091770390917803BD
:104D400097FD079653E0959587955A95E1F79F93C0
:104D50008F93209177033091780337FF02C0295F4A
:104D60003F4F43E0359527954A95E1F780912C0216
:104D700090912D02821B930B9F938F9382E396E079
:104D80009F938F931F930F93E0914C04F0914D04E8
:104D900009958CE380934D028DB79EB70A968DBF1F
:104DA00080917503909176039F938F938091750303
:104DB0009091760320912A0230912B02821B930B53
:104DC0009F938F9383E496E0ADC08B3019F08431CC
:104DD00008F4ADC084E180934D02809179039091F5
:104DE0007A039C0197FF02C0215F3F4F207F821B07
:104DF000930B97FD0196959587959F938F9380913F
:104E0000790390917A0397FD0F9624E09595879505
:104E10002A95E1F79F938F932091790330917A033C
:104E200037FF02C0295F3F4FC3E035952795CA95EC
:104E3000E1F780912E0290912F02821B930B9F939A
:104E40008F9381E596E09F938F931F930F93E0914B
:104E50004C04F0914D04099588E280934D022DB7E2
:104E60003EB7265F3F4F2DBF809177039091780327
:104E70009C0197FF02C0215F3F4F207F821B930B55
:104E800097FD0196959587959F938F9380917703D2
:104E90009091780397FD0F96A4E095958795AA9534
:104EA000E1F79F938F93209177033091780337FF39
:104EB00002C0295F3F4FF3E035952795FA95E1F75A
:104EC00080912C0290912D02821B930B9F938F93C4
:104ED00083E696E09F938F931F930F93E0914C048A
:104EE000F0914D0409958CE380934D028DB79EB7E8
:104EF0000A968DBF809175039091760397FD019678
:104F0000959587959F938F938091750390917603E4
:104F100020912A0230912B02821B930B9F938F9337
:104F200085E796E09F938F931F930F9303C18D3076
:104F300009F0CBC484E180934D028091150199273B
:104F40009F938F938091790390917A0397FD0F96A9
:104F500074E0959587957A95E1F79F938F932091CB
:104F6000790330917A0337FF02C0295F3F4F63E036
:104F7000359527956A95E1F780912E0290912F0241
:104F8000821B930B9F938F9384E896E09F938F935C
:104F90001F930F93E0914C04F0914D04099588E222
:104FA00080934D022DB73EB7265F3F4F2DBF8091B6
:104FB000140199279F938F938091770390917803A1
:104FC00097FD0F9654E0959587955A95E1F79F9335
:104FD0008F93209177033091780337FF02C0295FC8
:104FE0003F4F43E0359527954A95E1F780912C0294
:104FF00090912D02821B930B9F938F9388E996E0EB
:105000009F938F931F930F93E0914C04F0914D0465
:1050100009958CE380934D028DB79EB70A968DBF9C
:105020008091130199279F938F938091750390919D
:10503000760397FD0196959587959F938F93809121
:1050400075039091760320912A0230912B02821BE6
:10505000930B9F938F938CEA96E09F938F931F936C
:105060000F93E0914C04F0914D040995EDB7FEB714
:105070003A9668C010924D0280EC96E09F938F9311
:10508000DF92CF92FE01099584E180934D020F904B
:105090000F900F900F9080916F03909170039F93EA
:1050A0008F9380912602909127029F938F938DEC8E
:1050B00096E09F938F93DF92CF92E0914C04F09112
:1050C0004D04099588E280934D022DB73EB7285FC5
:1050D0003F4F2DBF80916D0390916E039F938F93EF
:1050E00080912802909129029F938F938CED96E0F6
:1050F0009F938F93DF92CF92E0914C04F0914D04F7
:1051000009958CE380934D028DB79EB708968DBFAD
:105110008091690390916A039F938F9380912402F9
:10512000909125029F938F938BEE96E09F938F93A0
:10513000DF92CF92E0914C04F0914D040995EDB7C8
:10514000FEB73896EDBFC1C310924D028091200189
:10515000909121016AE070E00E94418F9F938F93AC
:1051600080912001909121016AE070E00E94418FBE
:105170007F936F938AEF96E09F938F93DF92CF9206
:10518000FE01099584E180934D022DB73EB7285F5B
:105190003F4F2DBF80912C0990912D096AE070E05E
:1051A0000E942D8F9F938F9380912C0990912D09B0
:1051B0006AE070E00E942D8F7F936F938EE097E0FE
:1051C0009F938F93DF92CF92E0914C04F0914D0426
:1051D000099588E280934D028DB79EB708968DBFE2
:1051E00080912E0990912F099F938F9382E297E0EF
:1051F0009F938F93DF92CF92E0914C04F0914D04F6
:1052000009958CE380934D02EDB7FEB73696EDBF5E
:1052100080913009909131099F938F9382E397E0B9
:105220009F938F93DF92CF92E0914C04F0914D04C5
:1052300009952DB73EB72A5F3F4F4FC110924D02DF
:1052400084E497E09F938F93DF92CF92FE010995BC
:1052500084E180934D020F900F900F900F908091FA
:10526000C6079091C7079F938F938DE497E09F9314
:105270008F93DF92CF92E0914C04F0914D04099509
:1052800088E280934D028DB79EB706968DBF8091C0
:105290000E0399279F938F938DE597E09F938F93AC
:1052A000DF92CF92E0914C04F0914D0409958CE38C
:1052B00080934D02EDB7FEB73696EDBF8091C507DE
:1052C000992701979F938F938DE697E0A9CF10922E
:1052D0004D028DE797E09F938F93DF92CF92FE016F
:1052E000099584E180934D020F900F900F900F90DD
:1052F0008091B2019091B3019F938F9385E897E0DD
:105300009F938F93DF92CF92E0914C04F0914D04E4
:10531000099588E280934D028DB79EB706968DBFA2
:1053200080913D0890913E089F938F9383E997E089
:105330009F938F93DF92CF92E0914C04F0914D04B4
:1053400009958CE380934D02EDB7FEB73696EDBF1D
:1053500080912603909127039F938F9381EA97E092
:105360005FCFCFE0CC2EC3E0DC2E20E030E0E901BF
:10537000B3E0FB2EC0934D02F60181916F01992796
:105380009F938F9389010F5F1F4F1F930F938FEA96
:1053900097E09F938F9387EF92E29F938F93E09193
:1053A0004C04F0914D0409952DB73EB7285F3F4F4F
:1053B0002DBFFA9464969801F7FEDCCF86C2A3E174
:1053C000CA2EA3E0DA2EC0E0D0E08E01F3E0FF2E7B
:1053D00000934D02F60181916F0199279F938F935E
:1053E0002596DF93CF938CEB97E09F938F9387EF76
:1053F00092E29F938F93E0914C04F0914D040995B4
:105400002DB73EB7285F3F4F2DBFFA940C5E1F4F5C
:105410002497F7FEDDCF59C210924D0289EC97E038
:105420009F938F9307EF12E2DF92CF92FE010995CF
:1054300084E180934D020F900F900F900F90809118
:105440008F0199279F938F9381ED97E09F938F937F
:10545000DF92CF92E0914C04F0914D04099588E2DF
:1054600080934D028DB79EB706968DBF8091060240
:105470009091070297FD0396959587959595879549
:105480009F938F938FED97E09F938F931F930F932D
:10549000E0914C04F0914D0409958CE380934D020A
:1054A000EDB7FEB73696EDBF8091C30699279F935F
:1054B0008F938091C20699279F938F938DEE97E0EB
:1054C0009F938F931F930F93E0914C04F0914D04A1
:1054D00009952DB73EB7285F3F4F2DBFF6C11092FB
:1054E0004D028BEF97E09F938F9377EFA72E72E299
:1054F000B72EDF92CF92FE0109950F900F900F907B
:105500000F90C5E6D7E000E010E062E0F62E802FB5
:105510008C5E80934D028B8D99278F7790709F932F
:105520008F938B8999278F7790709F938F938B851B
:1055300099278F7790709F938F938B8199278F777F
:1055400090709F938F938BE098E09F938F93BF927F
:10555000AF92E0914C04F0914D0409958DB79EB740
:105560000C968DBFFA940C5E1F4FA096F7FECFCF1E
:10557000ACC110924D028CE198E09F938F9357EF4E
:10558000A52E52E2B52EDF92CF92FE0109950F9023
:105590000F900F900F90C5E6D7E000E010E042E0DA
:1055A000F42E802F8C5E80934D028F8D992787FD7E
:1055B00090959F938F938F89992787FD90959F93BF
:1055C0008F938F85992787FD90959F938F938F81D8
:1055D000992787FD90959F938F938BE298E09F93F7
:1055E0008F93BF92AF92E0914C04F0914D040995D6
:1055F000EDB7FEB73C96EDBFFA940C5E1F4FA09638
:10560000F7FECFCF62C110924D028CE398E09F93DA
:105610008F9307EF12E2DF92CF92FE01099584E1AA
:1056200080934D020F900F900F900F908091800704
:10563000881F8827881F97E0899FC00111248D96B5
:105640009F938F9380917807881F8827881F96E003
:10565000899FC00111248D969F938F93809170072D
:10566000881F8827881F95E0899FC00111248D9687
:105670009F938F9380916807881F8827881F992799
:10568000880F991F880F991F8D969F938F938BE496
:1056900098E09F938F93DF92CF92E0914C04F0912A
:1056A0004D04099588E280934D022DB73EB7245FE3
:1056B0003F4F2DBF8091A007881F8827881F9BE040
:1056C000899FC00111248D969F938F938091980795
:1056D000881F8827881F9AE0899FC00111248D9612
:1056E0009F938F9380919007881F8827881F99E048
:1056F000899FC00111248D969F938F938091880775
:10570000881F8827881F992723E0880F991F2A95CB
:10571000E1F78D969F938F938FE598E09F938F93FA
:10572000DF92CF92E0914C04F0914D0409958CE307
:1057300080934D028DB79EB70C968DBF8091A807C0
:10574000881F8827881F9CE0899FC00111248D969F
:105750009F938F9383E798E09F938F93DF92CF92ED
:10576000E0914C04F0914D0409958091B007EDB79C
:10577000FEB73696EDBF87FF12C080E480934D02DE
:1057800084E898E09F938F93DF92CF92E0914C044E
:10579000F0914D0409950F900F900F900F9080910C
:1057A000B80787FF12C084E480934D0287E898E031
:1057B0009F938F931F930F93E0914C04F0914D04AE
:1057C00009950F900F900F900F908091C00787FF61
:1057D0007CC088E480934D028AE898E09F938F9381
:1057E0001F930F93E0914C04F0914D0409950F9095
:1057F0000F900F900F9069C010924D028DE898E0C5
:105800009F938F93DF92CF92FE01099584E180935D
:105810004D020F900F900F900F908091DA019091B0
:10582000DB019F938F938BE998E09F938F93DF9297
:10583000CF92E0914C04F0914D04099588E2809359
:105840004D022DB73EB72A5F3F4F2DBF8091DC013F
:105850009091DD019F938F9388EA98E09F938F93B7
:10586000DF92CF92E0914C04F0914D04099589E4C8
:1058700080934D028DB79EB706968DBF85EB98E05D
:105880009F938F93DF92CF92E0914C04F0914D045F
:10589000099580914B020F900F900F900F9083FF0E
:1058A00014C01092DD011092DC0160E070E08EE027
:1058B00090E00E947B2E09C080912201281719F4E4
:1058C00021502093220110924C0210924B02DF9142
:1058D000CF911F910F91FF90DF90CF90BF90AF902D
:1058E0000895F999FECF92BD81BDF89A80B59927A8
:1058F0000895F999FECF1FBA92BD81BD60BD0FB664
:10590000F894FA9AF99A0FBE08954AEA20E030E036
:105910002617370740F4FC018191480F2F5F3F4F56
:1059200026173707C8F3842F99270895EAEA40E03D
:1059300050E04617570778F49C01F999FECF32BD25
:1059400021BDF89A80B5E80F4F5F5F4F2F5F3F4F43
:105950004617570790F38E2F9927089581E080937B
:10596000960682E08093950683E08093940684E017
:105970008093970685E08093980686E08093990649
:1059800087E080939A0688E080939B0689E0809365
:105990009C068AE080939D068BE080939E068CE0B7
:1059A00080939F0608958AE5809393068091020173
:1059B000843150F08AE08093B3061092D7068BE1D1
:1059C0008093AF068EE40AC083E08093B30680E242
:1059D0008093D7068EE18093AF0685E58093D40649
:1059E0008093D50690E29093D6061092FE068AE642
:1059F0008093A00682E28093000710920107E4E002
:105A0000E093BA061092F6061092F30668E06093EF
:105A1000AD0676EE7093AE0680E48093B0068EE11C
:105A20008093A1068FEF8093A30680E18093A40664
:105A30009093A2061092A6066093A70684E1809335
:105A4000A8061092A9065FE05093A5061092BC0626
:105A500048E24093BD0687E08093BE066093BF0690
:105A60001092D9061092DA061092DB069DE7909309
:105A7000DC0620E82093C00632E33093C10682E0C2
:105A80008093FF065093C2067093C306E093C80646
:105A90009093CB069093CC069093CD062093C406AA
:105AA00025E52093C50686E48093C6068CED809399
:105AB000C7068CE38093C9061092CA068FE58093CF
:105AC000DD0683EF8093DF068AEA8093E106809308
:105AD000E2064093DE064093E0063093CE069AE558
:105AE0009093CF063093D0068EEF8093E30684E642
:105AF0008093E4069093E5069093E6069093E7067C
:105B00008BE48093E8062093E9068093EA061092DE
:105B1000EB0686E08093EC066093ED069093EE062C
:105B20008AE28093EF0685EF8093F0068CE88093FD
:105B3000F10685E08093F2061092F4061092F506C5
:105B400081E28093B70681E48093B8069093B9060A
:105B50001092F7061092F8061092F90686E98093E3
:105B6000FA069093D10687E38093D2061092FB0643
:105B70001092FC061092FD060895CF93DF930E94C9
:105B8000D32C8AE08093AA0680E18093AB0626E0BE
:105B90002093AC069AE59093B10688E78093B2060D
:105BA0009093B4068093B5062093B60680E2809366
:105BB000BB068CE38093D3068BE48093D806A2E0E7
:105BC000B7E08CE0E3E2F1E0ED01019009928A9503
:105BD000E1F76BE770E0CD018F5690400E94852C75
:105BE00080930E07DF91CF910895CF93DF930E94AA
:105BF000D32C88E08093AA0630E13093AB0626E0F0
:105C00002093AC0694E69093B10688E78093B206A1
:105C10009093B4068093B5062093B6063093BB06E6
:105C200086E48093D3068093D806A2E0B7E08CE0A8
:105C3000E9E2F1E0ED01019009928A95E1F76BE765
:105C400070E0CD018F5690400E94852C80930E0706
:105C5000DF91CF910895CF93DF930E94D32C26E05C
:105C60002093AA068AE08093AB0684E08093AC067A
:105C700094E69093B10688E78093B2069093B406B9
:105C80008093B5062093B60680E18093BB0686E438
:105C90008093D3068093D806A2E0B7E08CE0E1E3DE
:105CA000F1E0ED01019009928A95E1F76BE770E070
:105CB000CD018F5690400E94852C80930E07DF9176
:105CC000CF910895F999FECF92BD81BDF89A80B524
:105CD00099270895F999FECF1FBA92BD81BD60BD85
:105CE0000FB6F894FA9AF99A0FBE089561E77CE22C
:105CF0000E94908D089549E75CE20E94CA8D089544
:105D0000EF92FF920F931F93CF93C82F815085304E
:105D100008F0C3E08CE7C89F8001112488EEE82ECC
:105D20008FEFF82EE00EF11E6BE770E0C7010E94C6
:105D3000962C682F98012D593F4F8FB39927AC01AE
:105D40004270507081FDF9CF32BD21BDF89A80B507
:105D5000861711F0CA0123C08FB399279C012270C6
:105D6000307081FDF9CFF2BCE1BCF89A80B58A357C
:105D700011F0C90114C08CE7C89FC00111244897D5
:105D800021E73CE24CE750E0BC0183E996E00E9449
:105D90006B8D0E942E6F0E94658981E090E0CF910B
:105DA0001F910F91FF90EF900895282F863010F0EB
:105DB00025E003C0882309F421E0F999FECF1FBA3A
:105DC00082E090E092BD81BD20BD0FB6F894FA9AB2
:105DD000F99A0FBE0895CF93C82F809193068A3504
:105DE00009F051C0C63010F0C5E003C0CC2309F45F
:105DF0004AC00E945D8C8091010782FF07C080919C
:105E0000B806843618F080E58093B8066BE770E03A
:105E100083E996E00E94852C80930E078CE7C89F4B
:105E2000C001112429E73CE24CE750E063E976E049
:105E300048970E94A88D29E73CE24CE050E064E9D5
:105E400076E080E590E00E94A88D6CE070E084E947
:105E500096E00E94852C282FF999FECF1FBA8CE579
:105E600090E092BD81BD20BD0FB6F894FA9AF99AE0
:105E70000FBE8C2F0E94D52E0E942E6F0E94658926
:105E800081E090E002C080E090E0CF9108956DE461
:105E900070E088EE93E00E94962C482F8FB39927EC
:105EA0009C012270307081FDF9CF85E394E092BDB2
:105EB00081BDF89A80B5841779F48FB399279C0136
:105EC0002270307081FDF9CF88EE93E092BD81BDE4
:105ED000F89A80B5813011F0C901089521E73CE2BC
:105EE0004EE450E068EE73E08FE097E00E946B8D27
:105EF00081E090E0089580910F078130A9F46DE46E
:105F000070E08FE097E00E94852C80935C0729E782
:105F10003CE24EE450E06FE077E088EE93E00E94D0
:105F2000A88D81E090E0089580E090E00895CF93FF
:105F3000DF9381E080930F07EFE0F7E08FE01586B5
:105F400016861786108A8150349687FFF8CF80E432
:105F500080931C0780931D0710921E0780931F07D4
:105F60008093200790EC9093210710922207809352
:105F70002307809324071092250790932607909378
:105F80002707809328071092290780932A07909368
:105F90002B07A0E1B7E087E0E7E3F1E0ED01019036
:105FA00009928A95E1F76DE470E0CD0101970E94B6
:105FB000852C80935C07DF91CF910895F999FECFEE
:105FC00082E090E092BD81BDF89A80B5282F86309E
:105FD00078F023E0322FF999FECF1FBA82E090E0EB
:105FE00092BD81BD30BD0FB6F894FA9AF99A0FBEF2
:105FF000822F992708951F93CF93C82F162F86308D
:1060000010F0C5E003C0882309F4C1E08C2F992764
:106010008230910541F08330910544F4019731F4C9
:106020000E94BD2D05C00E94F52D02C00E942B2E9E
:106030001123E1F06CE070E080E590E00E94962C86
:10604000282FF999FECF8CE590E092BD81BDF89A9A
:1060500080B5821759F421E73CE24CE050E060E55E
:1060600070E084E996E00E946B8D02C00E94AE2C25
:106070008C2F0E94EB2ECF911F910895DF92EF920B
:10608000FF920F931F93CF93FF24DF2CEF2C81E01F
:1060900090E00E94622E8A3511F031E0E32E6CE030
:1060A00070E080E590E00E94962CC82FF999FECF11
:1060B0008CE590E092BD81BDF89A80B58C1711F403
:1060C00021E0D22EC1E001E010E0EE2029F48C2F77
:1060D0000E94802E8823C9F591E0F92E1F930F931B
:1060E0008DEB98E09F938F9380EF94E19F938F9334
:1060F000E0914C04F0914D0409952DB73EB72A5F0D
:106100003F4F2DBF0230110549F0033011054CF40B
:106110000130110531F40E94BD2D05C00E94F52DFE
:1061200002C00E942B2EDD2059F021E73CE24CE01A
:1061300050E060E570E084E996E00E946B8D02C05B
:106140000E94AE2C8C2F0E94EB2ECF5F0F5F1F4F53
:10615000C63008F4BACFFF2019F083E00E94D52E94
:106160000E94DE2FC82F0E94802E8C2F99279F938C
:106170008F9383EE98E09F938F9300EF14E11F932A
:106180000F93E0914C04F0914D04099581E090E06B
:106190000E94622E2DB73EB72A5F3F4F2DBF8F3F23
:1061A00021F00E94472F882399F48CEF98E09F9369
:1061B0008F931F930F93E0914C04F0914D04099538
:1061C0000E94972F0E947B2F0F900F900F900F909F
:1061D000EE2029F06AE581E090E00E946A2E10929C
:1061E000920690E0ECE1F7E0CFE08081349618165B
:1061F0000CF49F5FC150C7FFF8CF90939206892F90
:1062000099279F938F9380E197E09F938F938DE1E0
:1062100099E09F938F931F930F93E0914C04F0911B
:106220004D0409950E94EC088DB79EB708968DBF66
:10623000CF911F910F91FF90EF90DF900895982FCD
:106240002FB7F8943998389A88B1836088B98091CB
:10625000B9008C7F8093B9008AE28093B8001092D5
:1062600058021092560210925502992379F0E5E6F1
:10627000F7E08BE010821182128213821482158261
:10628000168217828150389687FFF4CF78942FBFFB
:1062900008951092580284E98093BC0080E88093AE
:1062A000BC001092BD001092BA001092BB00109278
:1062B000B9001092B8001092540280E00E941F3181
:1062C0001092BB0085E88093BC00809152028260EE
:1062D0008093520208951F920F920FB60F921124CD
:1062E0002F933F934F935F938F939F93EF93FF93DE
:1062F00080915802282F3327442755278F5F80939A
:106300005802F9012731310508F0C2C2E759FF4FA1
:106310000C94C88F81E08093540209C0809156028A
:106320008C3090F4809156028F5F8093560280915A
:106330005602E82FFF27EE0FFF1FEE0FFF1FE15F52
:10634000F84F8585181654F7809156028C3070F0FE
:1063500010925102109250021092560285E08093E2
:10636000580280915502880F8D5A04C080915602C0
:10637000880F8E5A8093BB0085E87FC280915602B9
:10638000E82FFF2783E0EE0FFF1F8A95E1F7EB5917
:10639000F84F81818093BB0085E88093BC00809199
:1063A0005602E82FFF27EE0FFF1FEE0FFF1FEE0F25
:1063B000FF1FEB59F84F808180FF91C080915602FA
:1063C000E82FFF27EE0FFF1FEE0FFF1FEE0FFF1F3F
:1063D000EB59F84F8281882329F08091920687300B
:1063E00008F46CC28091500290915102892B09F0FF
:1063F00065C280914E0290914F02892B09F05EC2D6
:106400006EC08091560221E030E002C0220F331F9F
:106410008A95E2F780914E0290914F02282339230A
:10642000232B79F080915602E82FFF27EE0FFF1FF4
:10643000EE0FFF1FEE0FFF1FEB59F84F80E1848333
:106440000DC080915602E82FFF27EE0FFF1FEE0FC1
:10645000FF1FEE0FFF1FEB59F84F14828091560279
:10646000E82FFF2753E0EE0FFF1F5A95E1F7EB5996
:10647000F84F8481282F332743E0220F331F4A959A
:10648000E1F780915602E82FFF2793E0EE0FFF1F00
:106490009A95E1F7EB59F84F82818770822B8093B0
:1064A000BB0085E88093BC002091560281E090E01B
:1064B00002C0880F991F2A95E2F72091500230916F
:1064C000510282239323892B51F08DE597E090931D
:1064D0005C0280935B0288E080935D02EFC184E000
:1064E00089C1E0915B02F0915C0281918093BB00D5
:1064F00085E88093BC00F0935C02E0935B0280919E
:106500005D02815080935D02882309F4D7C183E046
:1065100071C18091B900803351F58091590288236F
:1065200029F4809156028F5F809359028091560220
:10653000E82FFF2783E0EE0FFF1F8A95E1F7EB5965
:10654000F84F838199278F7790708F3791057CF46E
:1065500080915602E82FFF27EE0FFF1FEE0FFF1F5F
:10656000EE0FFF1FEB59F84F83818F5F83831092EB
:10657000580284E98093BC008AE090E09093400147
:1065800080933F01809156028F5F80935602109254
:1065900058026DC18091B9008034C9F180915502D3
:1065A000E82FFF27EE0FFF1FEE0FFF1FEE0FFF1F5D
:1065B000EB59F84F83818F778383809155028F5FEA
:1065C00080935502809155028C30A0F010925502B4
:1065D00010924F0210924E0280915A028F5F809368
:1065E0005A028C3038F010925A02809152028D7FFC
:1065F00080935202809152028160809352021092E5
:10660000580284E98093BC001092540273C08091B8
:106610005502E82FFF27EE0FFF1FEE0FFF1FEE0FB3
:10662000FF1FEB59F84F8381806883838091550267
:10663000E82FFF27EE0FFF1FEE0FFF1FEE0FFF1FCC
:10664000EB59F84F808180FF2FC080915502E82FD1
:10665000FF2753E0EE0FFF1F5A95E1F7EB59F84F74
:1066600084819927009751F04097D9F58DE597E0FF
:1066700090935C0280935B0288E031C08091550268
:10668000992743E0880F991F4A95E1F78659984F5B
:1066900090935C0280935B029091550280915A0224
:1066A0009817E1F483E01BC080915502992733E0ED
:1066B000880F991F3A95E1F78659984F90935C029D
:1066C00080935B028091520281FD06C09091550239
:1066D00080915A02981711F482E001C081E0809302
:1066E0005D0280915D02813011F485E801C085EC86
:1066F0008093BC00809159028093530210925902FA
:10670000DDC0E0915B02F0915C028091BB00808370
:1067100080915B0290915C02019690935C02809361
:106720005B0280915D02815080935D02823010F0A7
:1067300085EC5DC0813011F485E859C0809152022A
:1067400081FF2DC08091D20280FD1DC08091550235
:10675000E82FFF2723E0EE0FFF1F2A95E1F7EB5903
:10676000F84F86818A3F79F480915502E82FFF2700
:1067700093E0EE0FFF1F9A95E1F7EB59F84F8081F8
:10678000816080830CC080915502E82FFF2783E051
:10679000EE0FFF1F8A95E1F7EB59F84F10828091B9
:1067A00055028F5F80935502809155028C30A0F086
:1067B0001092550210924F0210924E0280915A028E
:1067C0008F5F80935A028C3038F010925A02809179
:1067D00052028D7F809352021092580284E9809376
:1067E000BC008091520281608093520265C0809308
:1067F000BC0086E08093580261C088E9BBCD8091DF
:106800005702880F805FB6CD80915702992781305B
:10681000910561F0823091051CF4892B21F04EC066
:10682000029739F04BC080911501A4CD80911401DD
:10683000A1CD809113019ECD80E89CCD109258028D
:1068400084E98093BC00109254028AE090E0909317
:10685000400180933F0180915702823088F48091FB
:1068600057028F5F8093570282E180935802809194
:1068700052028E7F8093520285EA8093BC001EC034
:10688000109257028091520281608093520216C08A
:106890001092580284E98093BC008091520281607A
:1068A000809352028AE090E09093400180933F01F0
:1068B000109256021092550210925402FF91EF91DD
:1068C0009F918F915F914F913F912F910F900FBEAC
:1068D0000F901F9018951F93CF93DF93182F8091DF
:1068E0000D03882321F48091E901882319F081E0C8
:1068F00090E097C01D3008F092C01123B1F0E12F55
:10690000FF2723E0EE0FFF1F2A95E1F7EB59F84F21
:1069100035978081359688230CF081C03897808127
:1069200080FD03C083E090E07CC080915D078230F1
:1069300019F084E090E075C067E070E08DE597E0C5
:106940000E94852C90916407891719F085E090E0EA
:1069500068C080ED97E00E94FF18EC018091520220
:1069600080FD05C0CE010E9408198823B9F31123C8
:1069700019F48FEF90E00BC0212F332721503040C6
:1069800081E090E002C0880F991F2A95E2F790936A
:10699000510280935002A1E0B0E0E5E6F7E040E06C
:1069A00050E06BE0CD01042E02C0880F991F0A94BD
:1069B000E2F7209150023091510282239323892BD8
:1069C00011F01182128261504F5F5F4F389667FF5E
:1069D000E9CF1092560210925802809152028E7F97
:1069E0008093520285EA8093BC008091520280FD20
:1069F00005C0CE010E9408198823B9F38091500286
:106A000090915102892B29F0CE010E940819882308
:106A100011F38091500290915102009711F082E0A1
:106A200090E0DF91CF911F9108950F931F93CF9323
:106A3000DF93982F80910D03882321F48091E90141
:106A4000882319F081E090E092C09D30A0F4992352
:106A500019F486E090E08BC0C92FDD27FE0133E0FA
:106A6000EE0FFF1F3A95E1F7EB59F84F359780810C
:106A7000359687FD03C082E090E079C03897808129
:106A800080FD03C083E090E072C080ED97E00E943B
:106A9000FF188C018091520280FD05C0C8010E9440
:106AA00008198823B9F3219721E030E0C90102C019
:106AB000880F991FCA95E2F790934F0280934E0278
:106AC000D901E5E6F7E040E050E06BE0CD01042EAF
:106AD00002C0880F991F0A94E2F720914E0230916C
:106AE0004F0282239323892B11F01182128261506D
:106AF0004F5F5F4F389667FFE9CF109255021092B3
:106B00005D071092640710925802809152028E7FA6
:106B10008093520285EA8093BC008091520280FDEE
:106B200005C0C8010E9408198823B9F380914E025C
:106B300090914F02892B29F0C8010E9408198823DF
:106B400011F380915D07823019F084E090E00FC06E
:106B500067E070E08DE597E00E94852C90916407D6
:106B6000891719F085E090E002C080E090E0DF91A5
:106B7000CF911F910F910895CF93DF9380E022E88A
:106B80003FEFCAEFD7E0E6ECF7E0DF01853020F415
:106B900011961C921E9202C03183208319821882A2
:106BA00022968F5F129632968A3180F31092760386
:106BB00010927503109278031092770310927A0363
:106BC00010927903DF91CF9108951F920F920FB623
:106BD0000F9211240F931F932F933F934F935F9323
:106BE0006F937F938F939F93AF93BF93CF93DF93D5
:106BF000EF93FF938091000782FDE1C040918600F2
:106C00005091870080915F0290916002481B590B60
:106C100080918600909187009093600280935F023C
:106C2000CA018D549440A0916102B0916202835FC9
:106C30009A4178F4809161028093C507149714F00B
:106C40001092430181E090E0909362028093610290
:106C50002BC2AD30B1050CF027C2CA018B5F90404A
:106C6000845B914008F086C080914101909142017F
:106C7000481B590BE091FB06EE2351F0FF27EE0F66
:106C8000FF1FEA53F84F8081918184369105ECF41F
:106C9000FD01EA0FFB1FEA53F84F80819181FA0151
:106CA000E81BF90BCF01F7FF03C0909581959F4F2B
:106CB00006975CF480910E03883C20F480910E03CB
:106CC000865F01C088EC80930E03FD01EA0FFB1F75
:106CD000EA53F84F808191819C01220F331F280FC6
:106CE000391F240F351F37FF02C02D5F3F4FE901C9
:106CF000D595C795D595C795CA0101968C179D075F
:106D000014F4219706C041505040C417D5070CF425
:106D1000219680910E03833CE0F08D010A0F1B1F2A
:106D2000F801EA53F84F808191819E01281B390BAD
:106D3000C90163E070E00E94418FCB01880F991F69
:106D4000860F971F0650184FD80111969C938E936B
:106D500007C0AA0FBB1FA650B84F11961C921E92D7
:106D6000E0916102F0916202EE0FFF1FEA53F84FCB
:106D7000D183C08320916102309162022F5F3F4F27
:106D8000309362022093610280910201843108F005
:106D90008BC12530310511F45D9A01C05D98809159
:106DA0006102909162028630910511F45C9A01C0F3
:106DB0005C98079711F45B9A77C15B9875C1409115
:106DC0008600509187008091630290916402481B75
:106DD000590B809186009091870090936402809374
:106DE0006302CA018D5494406091CD02835F9A4141
:106DF00008F07AC060935E0280915E02843008F4ED
:106E000053C09091C50780915E02981709F04CC05D
:106E10005091CE025B3008F43FC0109243011092B3
:106E2000CD0240E05F31C0F0E42FFF27EE0FFF1FDF
:106E30009F0127563D4FDF01AA53B84F8D919C917A
:106E4000D9018D939C93DF01A650B84F8D919C91F1
:106E5000ED54FD4F91838083E42FFF27EE0FFF1F3A
:106E60009F012A53384FDF01AB59BD4F8D919C9143
:106E7000D90111969C938E93DF01A158BD4F8D913E
:106E80009C91E650F84F91838083842F8F5F482F29
:106E90008D3040F28093CD028091CE028F3FB9F0C9
:106EA0008F5F8093CE0213C08091CE02853620F092
:106EB0008AE08093CE0202C01092CE02809102013D
:106EC0008A3011F0843110F0289A01C0289881E0AE
:106ED0008093CD0280910D03882309F0E5C0809155
:106EE0005E028093C507E0C06D3008F0B5C0CA01EE
:106EF0008B5F9040845B914008F090C0809141018D
:106F000090914201481B590BE62FFF27EE0FFF1F00
:106F1000EB59FD4F80819181FA01E81BF90BCF01FC
:106F200005960B9720F5E091FB06EE2351F0FF2725
:106F3000EE0FFF1FEA53F84F80819181843691054F
:106F4000B4F48091CE028A3120F080910E03865FE6
:106F500005C08B3028F080910E038E5F80930E0366
:106F600080910E03893C18F088EC80930E03E62F85
:106F7000FF27EE0FFF1FEB59FD4F808191819C0190
:106F8000220F331F280F391F240F351F37FF02C070
:106F90002D5F3F4FE901D595C795D595C795CA0196
:106FA00001968C179D0714F4219706C0415050405C
:106FB000C417D5070CF4219680910E038E3BD8F0B0
:106FC000E62FFF27EE0FFF1FDF01AB59BD4F8D915D
:106FD0009C919E01281B390BC90163E070E00E945F
:106FE000418FCB01880F991F860F971FE158FD4FE6
:106FF0009183808308C0E62FFF27EE0FFF1FE15823
:10700000FD4F118210828091CD02E82FFF27EE0FF5
:10701000FF1FEB59FD4FD183C08309C0809102014E
:107020008A3011F0843110F0289A01C0289880919C
:107030000201843188F48091CD02853011F45D9A8B
:1070400005C05D98863011F45C9A05C05C98873065
:1070500011F45B9A01C05B988091CD02843120F4D9
:107060008F5F8093CD0220C08431F1F480910201C2
:107070008A3011F0843110F0289A01C028988EE1EE
:107080008093CD022CE0CAEFD7E0A9E9B2E0E6ECAC
:10709000F7E08D919D9191838083329619821882B9
:1070A0002296215027FFF5CFFF91EF91DF91CF91ED
:1070B000BF91AF919F918F917F916F915F914F9110
:1070C0003F912F911F910F910F900FBE0F901F9026
:1070D0001895EF92FF920F931F938091AF06992717
:1070E000880F991F880F991F7C010027F7FC0095D6
:1070F000102F8091640390916503A0916603B09175
:107100006703BC01CD01A80197010E94768F3093DF
:10711000F3052093F20580915C0390915D03A091AB
:107120005E03B0915F03BC01CD01A80197010E94ED
:10713000768F3093F5052093F40580918608909121
:10714000870897FD039695958795959587959093D4
:10715000F7058093F60580919F089091A00897FD10
:10716000039695958795959587959093F9058093C6
:10717000F805809175039091760320912A02309151
:107180002B02821B930B9093FB058093FA05809151
:10719000080390910903A0910A03B0910B03BC016D
:1071A000CD0125E030E040E050E00E94768F309342
:1071B000FD052093FC058091240290912502909377
:1071C000FF058093FE058091B2019091B3019093E9
:1071D00003068093020680912001909121019093F3
:1071E00005068093040680910E0399279093070665
:1071F0008093060680913D0890913E089093090681
:107200008093080680916607992790930B068093D8
:107210000A0680916E07992790930D0680930C06BD
:1072200080917607992790930F0680930E068091A0
:107230007E0799279093110680931006809180080D
:10724000992787FD9095909313068093120680915D
:107250006708992787FD90959093150680931406EB
:107260008091020290910302909317068093160674
:10727000809104029091050290931906809318065C
:10728000809106029091070290931B0680931A0644
:1072900080912C0990912D0990931F0680931E06D2
:1072A00080913009909131099093210680932006B6
:1072B0008091040390910503A0910603B091070308
:1072C000BC01CD0125E030E040E050E00E94768F27
:1072D0003093230620932206809126039091270362
:1072E00090932906809328068091340999279093DA
:1072F0002D0680932C068091EA039091EB039093E6
:107300002F0680932E068091E8039091E9039093D5
:1073100031068093300680916604882321F48091A1
:107320006704882321F08091F105816003C080917A
:10733000F1058E7F8093F1051F910F91FF90EF90E3
:1073400008951F93CF93DF93182FEB0180910D03C6
:10735000882309F5809102018C3010F4299801C02E
:10736000299A11501F3F81F0D0930D02C0930C0257
:1073700080910C0290910D02892BD1F7CE018C0FD8
:107380009D1F0E941419EDCF809102018C3010F4E2
:10739000299A01C02998DF91CF911F910895CF9329
:1073A000DF93809102018D3011F40E94F71D10923D
:1073B0007A0080912E0290912F0290934908809339
:1073C000480880912C0290912D0290933808809368
:1073D000370880912A0290912B0290938D08809318
:1073E0008C082091260230912702C901880F991F2D
:1073F000880F991F820F931F820F931F9093870806
:10740000809386082091280230912902C901880FB3
:10741000991F880F991F820F931F820F931F9093BC
:10742000A00880939F088FEC80937A00AFE0B3E0D0
:10743000C8E9D6E097E08991E82FFF27EE0FFF1FFC
:10744000EA53F84F0190F081E02DE158FF4F1E16EE
:107450001F061CF0E0E0F0E005C0EF3FF10514F07E
:10746000EFEFF0E08C91282F3327E217F30714F4A5
:10747000815004C02E173F0714F48F5F8C939150F6
:10748000119697FFD8CF8091D4069927AA27BB27BA
:10749000BC01CD0124EC39E040E050E00E94028FB5
:1074A000DC01CB018093AA019093AB01A093AC01C6
:1074B000B093AD018091D5069927AA27BB27BC01BF
:1074C000CD010E94028FDC01CB018093A601909335
:1074D000A701A093A801B093A901DF91CF910895CE
:1074E000A0E0B0E0E6E7FAE30C94978F882EC0E0C6
:1074F000D0E07E016E0110926604469AD09370032C
:10750000C0936F03D0936E03C0936D03D0936A034F
:10751000C0936903D0937A03C0937903D09378031F
:10752000C0937703D0937603C093750310928C01B8
:1075300010928B0110921F020E94CF3984E690E0D6
:107540000E9421190E94CF398091A00680FF10C0AF
:107550008091160190911701875B934038F48091D8
:107560001601909117018E5E924010F40E94751DD5
:107570000FE18AE090E00E94211980912A02909107
:107580002B02C80FD91F80912E0290912F02E80E76
:10759000F91E80912C0290912D02C80ED91E015027
:1075A00007FFE7CF9701205F3F4F36952795369528
:1075B000279530937A0320937903C60140969695D8
:1075C0008795969587959093780380937703609637
:1075D000F5E0D695C795FA95E1F7D0937603C09379
:1075E0007503909374038093730330937203209315
:1075F0007103882009F441C0809186089091870822
:1076000097FF03C0909581959F4F6CE070E00E94BA
:10761000418F9B017093700360936F0380919F086B
:107620009091A00897FF03C0909581959F4F6CE0C3
:1076300070E00E94418F70936E0360936D038091A0
:1076400035069091360690936A0380936903B901D9
:1076500084E090E00E947B2E60916D0370916E0338
:1076600086E090E00E947B2E6091690370916A032E
:1076700088E090E00E947B2E65C084E090E00E944C
:10768000762E9093700380936F0386E090E00E94C3
:10769000762E90936E0380936D0388E090E00E94B5
:1076A000762E9C0190936A038093690380916F0307
:1076B000909170038150984050F480916D039091A7
:1076C0006E038150984018F421503440D8F18EE375
:1076D00099E09F938F9380EF94E19F938F93E09134
:1076E0004C04F0914D04099580918608909187088B
:1076F00097FF03C0909581959F4F6CE070E00E94CA
:10770000418F7093700360936F0380919F089091F5
:10771000A00897FF03C0909581959F4F6CE070E0A3
:107720000E94418F70936E0360936D0380913506C4
:107730009091360690936A03809369030F900F909F
:107740000F900F9010924908109248081092380834
:107750001092370810928D0810928C0884E690E001
:107760000E94211980912602909127029C01220FEC
:10777000331F220F331F280F391F280F391F309353
:1077800087082093860880912802909129028C0115
:10779000000F111F000F111F080F191F080F191FCD
:1077A0001093A00800939F088091AF06C82EDD2497
:1077B000EE24FF24442737FD4095542FC701B6011E
:1077C0000E94028F4B015C01609364037093650318
:1077D00080936603909367039801442737FD409593
:1077E000542FC701B6010E94028FDC01CB018093A8
:1077F0005C0390935D03A0935E03B0935F0380925C
:10780000440390924503A0924603B09247038093AD
:107810003C0390933D03A0933E03B0933F0310922B
:10782000340310923503109236031092370380917F
:10783000180190911901A0911A01B0911B01909328
:1078400038068093370610921E0210921D02109285
:1078500028031092290310922A0310922B030091FF
:10786000B2011091B301109327030093260384E61D
:1078700090E09093AF018093AE0182E390E090930B
:107880000D0280930C028091D4069927AA27BB276A
:10789000BC01CD0124EC39E040E050E00E94028FB1
:1078A000DC01CB018856954CAF4FBF4F8093AA01A6
:1078B0009093AB01A093AC01B093AD018091D5063C
:1078C0009927AA27BB27BC01CD010E94028FDC01AA
:1078D000CB018856954CAF4FBF4F8093A601909334
:1078E000A701A093A801B093A90110924A01109298
:1078F0004901C801AA2797FDA095BA2F20914501FB
:10790000309146014091470150914801BC01CD01A1
:107910000E94028FDC01CB0180939308909394081E
:10792000A0939508B0939608109223031092220317
:107930000E942E6F8091D20284608093D2028FEFDA
:1079400080931C0910921D0980E280931E09CFE0EC
:10795000D3E0A8E9B6E007E08D91E82FFF27EE0F0E
:10796000FF1FEA53F84F808191818158899301501C
:1079700007FFF2CF84E680930E0380910A028823EA
:1079800011F0469A579A8091790390917A03805624
:107990009940815C9B4228F08091660481608093CD
:1079A0006604809177039091780380569940815CBA
:1079B0009B4228F0809166048260809366048091E7
:1079C0007503909176038C5291408957954028F029
:1079D0008091660484608093660480916F03909127
:1079E00070038C529140835C914028F08091660432
:1079F00088608093660480916D0390916E038C5231
:107A00009140835C914028F080916604806180936E
:107A100066048091690390916A0380509240835577
:107A2000914028F08091660480628093660486E429
:107A30008093A1010E946589ECE0CDB7DEB70C947C
:107A4000B38FA3E1B0E0E7E2FDE30C94918F809166
:107A500075039091760320912A0230912B02821BAC
:107A6000930B90938D0880938C0820913402309171
:107A70003502309349082093480880913202909152
:107A8000330290933808809337083093540820933A
:107A9000530890934C0880934B08809186089091EE
:107AA0008708AC01440F551F480F591F209126022B
:107AB00030912702C901880F991F880F991F820FE3
:107AC000931F820F931F480F591F57FF02C04D5F2E
:107AD0005F4F559547955595479550938708409327
:107AE000860880919F089091A008AC01440F551F13
:107AF000480F591F2091280230912902C901880F8F
:107B0000991F880F991F820F931F820F931F480F91
:107B1000591F57FF02C04D5F5F4F559547955595CB
:107B200047955093A00840939F08209126023091DA
:107B30002702C901880F991F880F991F820F931F71
:107B4000820F931F9C01442737FD4095542F80914D
:107B5000540390915503A0915603B0915703820F9F
:107B6000931FA41FB51F8093540390935503A093B4
:107B70005603B09357032091280230912902C9017E
:107B8000880F991F880F991F820F931F820F931FD1
:107B90009C01442737FD4095542F809150039091CC
:107BA0005103A0915203B0915303820F931FA41F5E
:107BB000B51F8093500390935103A0935203B09349
:107BC000530380915D0890915E08209126023091C8
:107BD0002702820F931F90935E0880935D08809127
:107BE0008F08909190082091280230912902820FED
:107BF000931F9093900880938F0880916B039091CE
:107C00006C03019690936C0380936B03809135060F
:107C1000909136062091690330916A03821B930B81
:107C20009C01442737FD4095542F80914C0390913F
:107C30004D03A0914E03B0914F03820F931FA41FD9
:107C4000B51F80934C0390934D03A0934E03B093C4
:107C50004F038FEC80937A001092120120913C0325
:107C600030913D0340913E0350913F0329873A876D
:107C70004B875C8729543B46414050402CF028E418
:107C80003BE641E050E00DC089859A85AB85BC8517
:107C9000885B9449AE4FBF4F4CF428EB34E94EEF6C
:107CA0005FEF2D833E834F83588708C089859A856F
:107CB000AB85BC858D839E83AF83B88720914403B9
:107CC0003091450340914603509147032D873E87ED
:107CD0004F87588B29543B46414050402CF028E4B4
:107CE0003BE641E050E00DC08D859E85AF85B889AB
:107CF000885B9449AE4FBF4F4CF428EB34E94EEF0C
:107D00005FEF29833A834B835C8308C08D859E8512
:107D1000AF85B88989839A83AB83BC83A0918C0893
:107D2000B0918D08BB8BAA8BFD01CF01AA2797FDCF
:107D3000A095BA2FA0903403B0903503C0903603BD
:107D4000D0903703A80EB91ECA1EDB1EA0923403C2
:107D5000B0923503C0923603D0923703E090930877
:107D6000F09094080091950810919608E80EF91E7D
:107D70000A1F1B1FE0929308F09294080093950845
:107D800010939608F091F102F98BFF2309F09CC142
:107D90008091F002882309F097C18091820886FFC4
:107DA00093C18091370890913808AA2797FDA09534
:107DB000BA2FBC01CD0129813A814B815C810E949F
:107DC000028F9B01AC0197FF04C02150384F4F4FE9
:107DD0005F4FBBE05595479537952795BA95D1F7F5
:107DE00080918B01682E772488249924CA01B901D7
:107DF000A40193010E94028FDC01CB0180939203C6
:107E000090939303A0939403B0939503B7FF04C09A
:107E10008150904FAF4FBF4F1C012D01ACE05594E6
:107E2000479437942794AA95D1F7209292033092E1
:107E30009303409294035092950380914808909147
:107E40004908AA2797FDA095BA2FBC01CD012D8125
:107E50003E814F8158850E94028F97FF04C0615078
:107E6000784F8F4F9F4FFBE0959587957795679556
:107E7000FA95D1F7A40193010E94028FDC01CB0196
:107E80008093960390939703A0939803B0939903DC
:107E9000B7FF04C08150904FAF4FBF4F9C01AD0161
:107EA000ECE05595479537952795EA95D1F72093BE
:107EB00096033093970340939803509399038091CE
:107EC00092039091930390932F0880932E088091B2
:107ED0009603909197039093330880933208221968
:107EE000330944095509209396033093970340932F
:107EF00098035093990380916608882331F1E20E2C
:107F0000F31E041F151FE0929308F092940800934B
:107F100095081093960880918A018823B1F457FF41
:107F200004C02F5F3F4F4F4F5F4F55954795379593
:107F30002795A21AB30AC40AD50AA0923403B092B4
:107F40003503C0923603D09237032A893B897901E1
:107F50000027F7FC0095102F8091960390919703CE
:107F6000A0919803B0919903E80EF91E0A1F1B1FF8
:107F7000C801B70129813A814B815C810E94028F3F
:107F80009B01AC0197FF04C02150384F4F4F5F4F0A
:107F90006BE055954795379527956A95D1F7809170
:107FA0008C01A82EBB24CC24DD24CA01B901A60172
:107FB00095010E94028FDC01CB0180938A0390938C
:107FC0008B03A0938C03B0938D03B7FF04C0815043
:107FD000904FAF4FBF4F3C014D013CE095948794CB
:107FE000779467943A95D1F760928A0370928B03E5
:107FF00080928C0390928D03C801B7012D813E8140
:108000004F8158850E94028F97FF04C06150784FBE
:108010008F4F9F4F2BE095958795779567952A957C
:10802000D1F7A60195010E94028FDC01CB0180935C
:108030008E0390938F03A0939003B0939103B7FFA7
:1080400004C08150904FAF4FBF4FAC01BD018CE0D9
:1080500075956795579547958A95D1F740938E0307
:1080600050938F0360939003709391032A893B8907
:1080700037FF03C0309521953F4F21343105E4F19E
:10808000D401C30197FE07C0B095A0959095819546
:108090009F4FAF4FBF4F81389105A105B10584F4C3
:1080A000DB01CA0177FF07C0B095A0959095819537
:1080B0009F4FAF4FBF4F81389105A105B105E4F047
:1080C00081E08093240318C0109233081092320884
:1080D00010922F0810922E0810928E0310928F0388
:1080E000109290031092910310928A0310928B03C6
:1080F00010928C0310928D0380918E0390918F03C8
:10810000A0919003B0919103BC01CD0124E630E031
:1081100040E050E00E94768FE0908A03F0908B035D
:10812000E21AF30AF0924708E092460880918A0327
:1081300090918B03A0918C03B0918D03BC01CD0174
:1081400024E630E040E050E00E94768FDA01C90179
:1081500020918E0330918F038C01021B130B10931F
:108160003A08009339088091450190914601A09109
:108170004701B0914801BC01CD0128E631E040E063
:1081800050E00E94028F2091930830919408409112
:10819000950850919608261737074807590764F045
:1081A000261B370B480B590B2093930830939408E8
:1081B0004093950850939608209193083091940825
:1081C000409195085091960857FF0CC0260F371F15
:1081D000481F591F209393083093940840939508A3
:1081E0005093960860913708709138086E0D7F1D86
:1081F0009B01442737FD4095542F8091380390917F
:108200003903A0913A03B0913B03820F931FA41F3F
:10821000B51F8093380390933903A0933A03B0932A
:108220003B038091F6029091F702681B790BCB011A
:10823000AA2797FDA095BA2F29853A854B855C859D
:10824000820F931FA41FB51F80933C0390933D039F
:10825000A0933E03B0933F03C090A601D090A70126
:10826000E090A801F090A901C816D906EA06FB061D
:10827000C4F488EA91E6A0E0B0E08C199D09AE094B
:10828000BF0980933C0390933D03A0933E03B093BA
:108290003F038093380390933903A0933A03B0933C
:1082A0003B0322273327A9012C193D094E095F09F9
:1082B00080913C0390913D03A0913E03B0913F0318
:1082C00082179307A407B507B4F4D701C601885AEB
:1082D0009146A040B04080933C0390933D03A0930F
:1082E0003E03B0933F038093380390933903A093E8
:1082F0003A03B0933B036091480870914908600FBE
:10830000711F9B01442737FD4095542F80914003F6
:1083100090914103A0914203B0914303820F931FB8
:10832000A41FB51F8093400390934103A093420381
:10833000B09343038091F4029091F502681B790B8E
:10834000CB01AA2797FDA095BA2F2D853E854F8595
:108350005889820F931FA41FB51F809344039093E5
:108360004503A0934603B0934703E090AA01F09021
:10837000AB010091AC011091AD01E816F9060A07B6
:108380001B07C4F488EA91E6A0E0B0E08E199F09CB
:10839000A00BB10B8093440390934503A093460335
:1083A000B09347038093400390934103A09342030B
:1083B000B093430322273327A9012E193F09400B0D
:1083C000510B8091440390914503A0914603B091D5
:1083D000470382179307A407B507B4F4D801C70170
:1083E000885A9146A040B04080934403909345033F
:1083F000A0934603B09347038093400390934103B7
:10840000A0934203B09343038091340390913503CA
:10841000A0913603B09137038093480390934903AA
:10842000A0934A03B0934B0380914403909145037A
:10843000A0914603B0914703809364039093650332
:10844000A0936603B093670380913C0390913D0332
:10845000A0913E03B0913F0380935C0390935D0332
:10846000A0935E03B0935F0380914003909141031A
:10847000A0914203B0914303809360039093610302
:10848000A0936203B0936303809138039091390302
:10849000A0913A03B0913B03809358039093590302
:1084A000A0935A03B0935B0380911E0190911F012A
:1084B000909349088093480880911C0190911D0178
:1084C0009093380880933708809102018A3009F030
:1084D00062C080912E0290912F02835F934034F00E
:1084E00088E592E0909349088093480880912E0295
:1084F00090912F028A5F934034F080E293E0909352
:1085000049088093480880912E0290912F020F977E
:1085100034F488EA9DEF909349088093480880914D
:108520002E0290912F02079734F480EE9CEF9093E7
:1085300049088093480880912C0290912D02835F16
:10854000934034F088E592E09093380880933708A0
:1085500080912C0290912D028A5F934034F080E24A
:1085600093E0909338088093370880912C02909183
:108570002D020F9734F488EA9DEF9093380880938A
:10858000370880912C0290912D0207970CF067C05C
:1085900080EE9CEF60C080912E0290912F02815D51
:1085A000974034F080EB94E090934908809348081A
:1085B00080912E0290912F02805E974034F080E4EB
:1085C00096E0909349088093480880912E029091FC
:1085D0002F020F9734F480E59BEF90934908809326
:1085E000480880912E0290912F02079734F480EC76
:1085F00099EF909349088093480880912C029091BC
:108600002D02815D974034F080EB94E09093380820
:108610008093370880912C0290912D02805E9740C4
:1086200034F080E496E09093380880933708809186
:108630002C0290912D020F9734F480E59BEF9093DC
:1086400038088093370880912C0290912D0207976B
:1086500034F480EC99EF9093380880933708609158
:108660009601662309F4B3C040911E0150911F0189
:1086700080919A0390919B03481B590B5093A1033F
:108680004093A00320911E0130911F01280F391F34
:1086900037FF02C02F5F3F4F3595279530939B03DF
:1086A00020939A03413151051CF080E190E005C010
:1086B000405F5F4F34F480EF9FEF9093A10380936E
:1086C000A00340911C0150911D0180919C03909149
:1086D0009D03481B590B50939F0340939E03209189
:1086E0001C0130911D01280F391F37FF02C02F5F79
:1086F0003F4F3595279530939D0320939C0341313F
:1087000051051CF080E190E005C0405F5F4F34F4FC
:1087100080EF9FEF90939F0380939E03462F5527F2
:108720008091A0039091A103849FB001859F700D5B
:10873000949F700D11249B0177FF02C02F5F3F4F64
:10874000359527958091480890914908820F931F8D
:10875000909349088093480880919E0390919F03CD
:10876000849FD001859FB00D949FB00D1124AD0161
:108770009D01B7FF02C02F5F3F4F35952795809130
:10878000370890913808820F931F90933808809390
:108790003708F3E0660F771FFA95E1F780911E0125
:1087A00090911F01860F971F90931F0180931E01C8
:1087B000E3E0440F551FEA95E1F780911C01909189
:1087C0001D01840F951F90931D0180931C01009142
:1087D0004B0810914C0880912E0890912F0810168C
:1087E00011065CF59C0197FF04C022273327281B44
:1087F000390BC901AA2797FDA095BA2F20918A01AC
:10880000332744275527BC01CD010E94028F9B01CD
:10881000AC0197FF04C0215C3F4F4F4F5F4F76E0A4
:1088200055954795379527957A95D1F780914608C4
:1088300090914708820F931F27C097FF03C0909520
:1088400081959F4FAA2797FDA095BA2F20918A0165
:10885000332744275527BC01CD010E94028F9B017D
:10886000AC0197FF04C0215C3F4F4F4F5F4F66E064
:1088700055954795379527956A95D1F78091460884
:1088800090914708821B930B90934708809346086A
:10889000E0905308F090540880913208909133088A
:1088A0001E141F045CF59C0197FF04C02227332788
:1088B000281B390BC901AA2797FDA095BA2F209133
:1088C0008A01332744275527BC01CD010E94028F1E
:1088D0009B01AC0197FF04C0215C3F4F4F4F5F4F9E
:1088E00096E055954795379527959A95D1F78091BC
:1088F000390890913A08820F931F27C097FF03C051
:10890000909581959F4FAA2797FDA095BA2F20910A
:108910008A01332744275527BC01CD010E94028FCD
:108920009B01AC0197FF04C0215C3F4F4F4F5F4F4D
:1089300086E055954795379527958A95D1F780918B
:10894000390890913A08821B930B90933A088093D0
:1089500039088091820887FF44C0B989BB2309F098
:1089600040C08091F0028823E1F5E1E0EE16E1E0FD
:10897000FE064CF080914808909149088E0D9F1D8D
:10898000805091400DC0F0E0EF16FFEFFF0664F459
:1089900080914808909149088E0D9F1D80509F4FEF
:1089A000909349088093480821E0013012074CF069
:1089B0008091370890913808800F911F8050914026
:1089C0000CC03FEF0030130764F48091370890919A
:1089D0003808800F911F80509F4F909338088093E4
:1089E0003708E2E1CD5E0C94AD8F80910D038823B2
:1089F00001F58091D2028C7F8093D202ABE6B4E085
:108A0000E5E6F7E09BE08091E901882309F48C9387
:108A10008D91818312829150389697FFF4CF809187
:108A2000E901882359F08091E90181508093E9019F
:108A300005C08091D20281608093D202809154025D
:108A4000882319F01092540208958093560280935F
:108A50005802809152028E7F8093520285EA809361
:108A6000BC000895CF93DF93AFE0B3E0C8E9D6E050
:108A700057E09991E92FFF27EE0FFF1FEA53F84FB8
:108A80000190F081E02DE158FF4FEF3FF10521F01B
:108A90001CF0EFEFF0E004C0F7FF02C0E0E0F0E010
:108AA000993111F4EC931BC04C91242F3327E2171A
:108AB000F307A9F0CF01821B930B97FD03969595C1
:108AC000879595958795242F280F2C93822F99278A
:108AD000E817F90714F4215001C02F5F2C9351506F
:108AE000119657FFC6CF8091A206883F38F0EFEF6E
:108AF000F0E0E81BF109E15FFC4F808180939C016D
:108B000080919C01882329F0843618F084E68093B4
:108B10009C018091A406883F38F0EFEFF0E0E81B5D
:108B2000F109E15FFC4F808180939A0180919A0165
:108B3000882329F0843618F084E680939A01809186
:108B4000B106883F38F0EFEFF0E0E81BF109E15F94
:108B5000FC4F808180939501809195018B3010F4BA
:108B60008AE002C08F3F11F4809395018091DE0668
:108B7000883F38F0EFEFF0E0E81BF109E15FFC4FD0
:108B8000808180935F0880915F08863010F485E0D3
:108B900002C08F3F11F480935F088091E006883F08
:108BA00038F0EFEFF0E0E81BF109E15FFC4F808166
:108BB0008093890880918908863010F485E002C08E
:108BC0008F3F11F4809389088091CB06873F19F479
:108BD000429905C006C0863F31F4439B02C08CE831
:108BE0000BC086E409C0883F38F0EFEFF0E0E81BE7
:108BF000F109E15FFC4F808180935C088091CC0695
:108C0000873F19F4429905C006C0863F31F4439B63
:108C100002C08CE80BC086E409C0883F38F0EFEF53
:108C2000F0E0E81BF109E15FFC4F8081809334089C
:108C30008091CD06883F38F0EFEFF0E0E81BF109B6
:108C4000E15FFC4F8081809365088091A306883F97
:108C500038F0EFEFF0E0E81BF109E15FFC4F8081B5
:108C600080939B018091A606883F38F0EFEFF0E0FB
:108C7000E81BF109E15FFC4F8081809399018091AD
:108C8000A806883F38F0EFEFF0E0E81BF109E15F5C
:108C9000FC4F8081809397018091B006883F38F027
:108CA000EFEFF0E0E81BF109E15FFC4F808180937A
:108CB00098018091B206883F38F0EFEFF0E0E81BB2
:108CC000F109E15FFC4F8081809394018091B306AC
:108CD000883F38F0EFEFF0E0E81BF109E15FFC4F6F
:108CE0008081809396018091B406883F38F0EFEF41
:108CF000F0E0E81BF109E15FFC4F80818093930174
:108D00008091B506883F38F0EFEFF0E0E81BF109FD
:108D1000E15FFC4F8081809392018091BB06883F88
:108D200038F0EFEFF0E0E81BF109E15FFC4F8081E4
:108D3000809390018091BC06883F38F0EFEFF0E01F
:108D4000E81BF109E15FFC4F80818093EB02809189
:108D5000BD06883F38F0EFEFF0E0E81BF109E15F76
:108D6000FC4F80818093EA028091BE06883F38F0F4
:108D7000EFEFF0E0E81BF109E15FFC4F80818093A9
:108D8000E9028091BF06883F38F0EFEFF0E0E81B82
:108D9000F109E15FFC4F80818093E8028091D90660
:108DA000883F38F0EFEFF0E0E81BF109E15FFC4F9E
:108DB00080818093E7028091DA06883F38F0EFEFF8
:108DC000F0E0E81BF109E15FFC4F80818093E6024F
:108DD0008091DB06883F38F0EFEFF0E0E81BF10907
:108DE000E15FFC4F80818093E5028091DC06883F43
:108DF00038F0EFEFF0E0E81BF109E15FFC4F808114
:108E00008093E4028091C006883F38F0EFEFF0E0F5
:108E1000E81BF109E15FFC4F808180938F01809115
:108E2000C406883F38F0EFEFF0E0E81BF109E15F9E
:108E3000FC4F808180938E018091CE06883F38F070
:108E4000EFEFF0E0E81BF109E15FFC4F80818093D8
:108E50008D018091D106883F38F0EFEFF0E0E81BFC
:108E6000F109E15FFC4F808180938C018091D206F3
:108E7000883F38F0EFEFF0E0E81BF109E15FFC4FCD
:108E8000808180938B018091D306883F38F0EFEF8B
:108E9000F0E0E81BF109E15FFC4F808180938A01DB
:108EA0008091FA06883F38F0EFEFF0E0E81BF10917
:108EB000E15FFC4F8081809344089091F4039923F3
:108EC00021F080914408981720F08091440888236D
:108ED00011F4909344088091A006809382088091B9
:108EE0000007809364088091D806883F38F0EFEF40
:108EF000F0E0E81BF109E15FFC4F8081809389017C
:108F00008091F306883F38F0EFEFF0E0E81BF109BD
:108F1000E15FFC4F80818093A20880919001282F0F
:108F200033272F5F3F4F8CE398E2B9010E94418FB6
:108F30007093A00160939F018091EB02833380F0D6
:108F40008091EA02282F33272F5F3F4F8CE398E26E
:108F5000B9010E94418F70939E0160939D0104C0EE
:108F600070939E0160939D018091E3068093450874
:108F700080916608882311F4809345088091AE069D
:108F800080938A088091AD0680934D089091F506F4
:108F90009333E0F181E08093E302983F58F0EFEFE4
:108FA000F0E0E91BF109E15FFC4F8081823310F4AE
:108FB0001092E3028091A1012091E3028217B1F0A7
:108FC000833088F4222319F08CED95E002C088EC00
:108FD00090E090930D0280930C0285E08093F8025C
:108FE0002093A10103C081508093A1018091E308E7
:108FF0009091E40897FF0FC08091E302882359F015
:109000008091660480688093660405C01092E30234
:109010008AE08093A1018091E3089091E40897FF92
:109020001DC080910D038823C9F08091E30288233D
:10903000A9F080910801909109018F5F9F4F71F411
:1090400088E99AE390930D0280930C0280E094EA01
:1090500090930901809308011092E3028091E3024A
:10906000882369F08091D10281608093D102809140
:109070008C01823D48F4825E80938C0105C0809112
:10908000D1028E7F8093D102DF91CF910895AEE11E
:10909000B0E0EDE4F8E40C94918F0E94213D8091C2
:1090A000010782FF27C08091F2029091F30200979E
:1090B000F1F022E088359207D4F49C0197FF02C0BA
:1090C0002D5F3F4F35952795359527958091B806AB
:1090D0009927289FA001299F500D389F500D1124DA
:1090E000CA0164E670E00E94418FCB0106C08DE2A8
:1090F00090E003C08091B80699279093D0028093A6
:10910000CF0260911803709119037A83698380916B
:109110004D0899270A966817790714F49A8389836A
:1091200080910E03843608F06AC08091D10282FDDE
:1091300066C08091BE039091BF03009731F0019704
:109140009093BF038093BE030BC010920D039093C6
:10915000D4028093D3028091D2028D7E8093D2027A
:10916000809102018A3011F0843110F0289A01C0F8
:1091700028988091D3029091D402895E9340E0F1C7
:10918000809134098536C0F18091CF029091D00250
:109190009A8389838091D20280618093D2028091E8
:1091A0009406A82FBB27AA0FBB1FFD01E650F84F5E
:1091B0001182108280919506282F3327220F331FAA
:1091C000C9018650984FFC0111821082AA53B84FF2
:1091D00011961C921E922A53384FD90111961C9257
:1091E0001E9280919706E82FFF27EE0FFF1FEA538C
:1091F000F84F11821082C4C210920D03C1C2809137
:109200000E038D3808F4BCC28091D2028F7E809309
:10921000D2029091B90682E3989FC00111249093E5
:10922000BF038093BE03E981FA81B9978CF08091E6
:109230000D03882369F08091D3029091D402FFEF4F
:109240008F3F9F0729F001969093D4028093D30219
:109250008091D3029091D4028F3F910509F008F5D7
:1092600010923003109231031092320310923303A4
:1092700010922C0310922D0310922E0310922F03A4
:109280001092AA031092AB031092AC031092AD039C
:109290001092340310923503109236031092370364
:1092A00005C08091D20282608093D202809196069E
:1092B000E82FFF27EE0FFF1FEA53F84F80819181BF
:1092C000813591050CF458C120910D03222309F03A
:1092D00053C180919706E82FFF27EE0FFF1FEA5337
:1092E000F84F808191818C3491050CF422C18091DA
:1092F000C0038F5F8093C003893C08F43DC1209375
:10930000C0031092D4021092D30230919406E32F3E
:10931000FF27EE0FFF1FEA53F84F808191818734BA
:109320009105B4F480919506E82FFF27EE0FFF1FFB
:10933000EA53F84F808191810190F081E02DF7FF91
:1093400003C0F095E195FF4FE734F1050CF478C0C8
:1093500041E020919506A22FBB27AA0FBB1FAA535D
:10936000B84F8D919C9111978734910544F0E32F6C
:10937000FF27EE0FFF1FEA53F84F808191818D91F7
:109380009C918734910574F080919406E82FFF2713
:10939000EE0FFF1FEA53F84F8081918187349105CA
:1093A0000CF042E0E22FFF27EE0FFF1FEA53F84FC9
:1093B000808191818634910574F480919406E82F20
:1093C000FF27EE0FFF1FEA53F84F8081918187340A
:1093D00091050CF043E0E22FFF27EE0FFF1FEA5349
:1093E000F84F808191818A5B9F4F74F4809194063D
:1093F000E82FFF27EE0FFF1FEA53F84F808191817E
:10940000873491050CF044E0E22FFF27EE0FFF1F99
:10941000EA53F84F808191818A5B9F4F74F4809169
:109420009406E82FFF27EE0FFF1FEA53F84F8081C5
:109430009181863491050CF445E0842F0E94D52E4D
:1094400080919506E82FFF27EE0FFF1FEA53F84F94
:10945000808191810190F081E02DF7FF03C0F095AC
:10946000E195FF4F7E97CCF480919406E82FFF277B
:10947000EE0FFF1FEA53F84F808191818A5B9F4F67
:1094800064F481E0809381041092F90288EE93E005
:1094900090930D0280930C026FC00E94DE2F0E94F9
:1094A000802E80E00E9433098091BA060E94078BCB
:1094B0008091820880FF10C0809116019091170161
:1094C000875B934038F480911601909117018E5E6E
:1094D000924010F40E94751D10920A0280E00E94D2
:1094E000703A81E08093F90280930A02579A0E94B1
:1094F000DE2FE82FFF27ED54FE4F80818093D601A9
:109500000E94DE2F68E770E00E94A1398091E70297
:1095100099278F5790409093E1078093E0078091BF
:10952000E60299278F5790409093E3078093E207D4
:1095300023C080819181855B9F4FE4F48091C003BB
:109540008F5F8093C003893CB8F020930D03209374
:10955000C0031092D4021092D30281E00E94703AAC
:1095600081E08093F9020E94DE2F68E770E00E949C
:10957000A13902C02093C00380919606E82FFF27EF
:10958000EE0FFF1FEA53F84F808191818B5A9F4F56
:109590000CF0F6C030910D03E0919706332309F0EB
:1095A000C4C0FF27EE0FFF1FEA53F84F808191815F
:1095B000855B9F4F0CF0B6C02091F606E22FFF2787
:1095C000EE0FFF1FEA53F84F80819181855B9F4F1B
:1095D0001CF0222309F0A6C08091C1038F5F809305
:1095E000C103893C08F4CCC03093C1038091660468
:1095F000882309F090C08091F902882309F48BC078
:109600008091F903882309F086C081E090E090936F
:10961000D4028093D30281E080930D031092AA03B9
:109620001092AB031092AC031092AD03109234036E
:109630001092350310923603109237038091AF06D3
:10964000E82EFF2400271127809186089091870833
:109650009C01442737FD4095542FC801B7010E9453
:10966000028FDC01CB018093440390934503A093C8
:109670004603B093470380919F089091A0089C01F6
:10968000442737FD4095542FC801B7010E94028F2F
:10969000DC01CB0180933C0390933D03A0933E03F8
:1096A000B0933F038091640390916503A09166039A
:1096B000B09167038093400390934103A0934203CA
:1096C000B093430380915C0390915D03A0915E038E
:1096D000B0915F038093380390933903A0933A03CA
:1096E000B0933B0310923003109231031092320377
:1096F0001092330310922C0310922D0310922E031C
:1097000010922F038091D20288608093D20284E667
:109710008093F80235C08CED95E090930D02809314
:109720000C022EC01092C1032BC0FF27EE0FFF1FAB
:10973000EA53F84F808191818C349105FCF020919F
:10974000F606E22FFF27EE0FFF1FEA53F84F808146
:109750009181855B9F4F14F0222381F48091C20395
:109760008F5F8093C203893C58F010920D031092D2
:10977000C2031092D4021092D30202C01092C2030C
:1097800080914301815080934301809143018F3F39
:1097900021F08091D20284FF4BC40E943245D090C8
:1097A000AA068091EB02E09194064091CB03509180
:1097B000CC03833308F45AC09A01220F331F240FBD
:1097C000351FFF27EE0FFF1FEA53F84F8091E90284
:1097D000482F552780819181849FB001859F700D0E
:1097E000949F700D1124260F371F8091D7029091FE
:1097F000D802281B390B37FF02C02D5F3F4F35952C
:109800002795359527953093CC032093CB038091F2
:10981000CD039091CE039C01220F331F280F391FD7
:1098200080919506E82FFF27EE0FFF1FEA53F84FB0
:1098300080819181849FD001859FB00D949FB00D50
:1098400011242A0F3B1F8091D5029091D602281B2C
:10985000390B37FF02C02D5F3F4F35952795359562
:1098600027953093CE032093CD0355C09A01220F44
:10987000331F240F351FFF27EE0FFF1FEA53F84F4A
:109880004D2D552780819181849FF001859FF00D9A
:10989000949FF00D11242E0F3F1F37FF02C02D5F44
:1098A0003F4FB90175956795759567957093CC0392
:1098B0006093CB038091CD039091CE039C01220F46
:1098C000331F280F391F80919506E82FFF27EE0FD1
:1098D000FF1FEA53F84F80819181849FD001859FBB
:1098E000B00D949FB00D11242A0F3B1F37FF02C00B
:1098F0002D5F3F4FC90195958795959587959093D5
:10990000CE038093CD037093D8026093D7029093D7
:10991000D6028093D502609166086623D1F18091CA
:109920009406E82FFF27EE0FFF1FE650F84F8091B7
:10993000AB06482F552780819181849F9001859F98
:10994000300D949F300D11248091CB039091CC0366
:10995000820F931F9093CC038093CB038091950645
:10996000E82FFF27EE0FFF1FE650F84F808191810F
:10997000849F9001859F300D949F300D112480911C
:10998000CD039091CE03820F931F9093CE038093CB
:10999000CD038091E302882309F451C0662309F4C2
:1099A0004EC08091CB039091CC0397FD0396DC01D0
:1099B000B595A795B595A7958091CD039091CE03C8
:1099C00097FD0396FC01F595E795F595E795809150
:1099D000CD01682F772767FD70956A9F90016B9F77
:1099E000300D7A9F300D11248091FB03482F5527AD
:1099F00047FD50954E9FC0014F9F900D5E9F900D6B
:109A00001124280F391F37FF02C0295F3F4F93E011
:109A1000359527959A95E1F730931F0320931E0300
:109A20006E9F90016F9F300D7E9F300D11244A9FD5
:109A3000C0014B9F900D5A9F900D112450C08091F2
:109A4000F406E82FFF27EE0FFF1FE55BFE4F84852E
:109A500087FD8F5F982F95959093CD01808187FD2D
:109A60008F5F85958093FB03E92FFF27E7FDF09536
:109A7000A091CB03B091CC03EA9F9001EB9F300DF6
:109A8000FA9F300D1124682F772767FD709540915C
:109A9000CD035091CE03649FC001659F900D749FCC
:109AA000900D1124280F391F37FF02C0295F3F4F47
:109AB00083E0359527958A95E1F730931F0320932E
:109AC0001E03E49F9001E59F300DF49F300D11249B
:109AD0006A9FC0016B9F900D7A9F900D1124281BE7
:109AE000390B37FF02C0295F3F4F03E035952795BB
:109AF0000A95E1F730931D0320931C03809197068C
:109B0000E82FFF27EE0FFF1FEA53F84F8081918166
:109B1000909581959F4F90931B0380931A038530F6
:109B2000910514F0049705C0BFEF8C3F9B0734F4F8
:109B3000049690931B0380931A0304C010921B0396
:109B400010921A038091E703882309F43EC0282F5E
:109B5000332780911E0390911F0397FD079613E012
:109B6000959587951A95E1F7289FF001299FF00DAB
:109B7000389FF00D1124CF01F7FD0F96B4E09595B5
:109B80008795BA95E1F790931F0380931E03809108
:109B90001C0390911D0397FD0796A3E0959587956B
:109BA000AA95E1F7289FA001299F500D389F500DDD
:109BB0001124CA0157FD0F96F4E095958795FA9503
:109BC000E1F790931D0380931C03A0901E03B090B7
:109BD0001F038091EA039091EB03A81AB90AB0928F
:109BE0001F03A0921E0300911C0310911D0380917E
:109BF000E8039091E903081B190B10931D030093D0
:109C00001C0380919606E82FFF27EE0FFF1FEA53F3
:109C1000F84FE080F1806FE770E0E60EF71EF092FB
:109C20001903E0921803809195019927AA2797FDBF
:109C3000A095BA2FBC01CD010E94768EDC01CB012C
:109C400020E030E040E251E4BC01CD010E94E48D0F
:109C5000DC01CB01BC01CD010E94488EDC01CB01AF
:109C6000809391088091940180936608809193017C
:109C70009927AA2797FDA095BA2FBC01CD010E9474
:109C8000768EDC01CB0120E030E040E251E4BC0103
:109C9000CD010E94E48DDC01CB01BC01CD010E940D
:109CA000488EDC01CB0180933F0880919201809324
:109CB000550880918D0480FF59C08091A208813899
:109CC00008F454C080918604992787FD90952D2D26
:109CD0003327829FD001839FB00D929FB00D112436
:109CE000AA0EBB1EB0921F03A0921E038091870490
:109CF000992787FD9095829FF001839FF00D929F99
:109D0000F00D11240E0F1F1F10931D0300931C0351
:109D100080918804282F332727FD309580911A03DE
:109D200090911B03820F931F90931B0380931A0340
:109D300080918A04282F332727FD30958091A5062E
:109D40009927289FA001299F500D389F500D11245D
:109D500050934A01409349018091890499278E15B7
:109D60009F0524F49093190380931803809118039E
:109D70009091190397FF04C01092190310921803D1
:109D80008091820882FF02C01092660840911E03F3
:109D900050911F03CA0157FD03969C0135952795E5
:109DA0003595279537FF03C0309521953F4F80911A
:109DB000DB029091DC0282179307B4F4CA0157FFCB
:109DC00003C0909581959F4F97FD03969595879534
:109DD000959587959093DC028093DB0285369105FB
:109DE00044F084E690E001C001979093DC028093F8
:109DF000DB0240911C0350911D03CA0157FD0396DD
:109E00009C01359527953595279537FF03C03095EB
:109E100021953F4F8091D9029091DA0282179307E2
:109E2000B4F4CA0157FF03C0909581959F4F97FDE9
:109E3000039695958795959587959093DA028093EB
:109E4000D9028536910544F084E690E001C001977F
:109E50009093DA028093D9028091D20284FF08C0E5
:109E60001092DC021092DB021092DA021092D902F8
:109E700050919506E52FFF27EE0FFF1FEA53F84F8D
:109E80004091CF06242F33278081918128173907ED
:109E900044F48091FE0682FF04C081E08093EF02CB
:109EA00013C0E52FFF27EE0FFF1FEA53F84F842F53
:109EB00099272091D006821B910920813181281792
:109EC000390714F41092EF0240919506E42FFF2712
:109ED000EE0FFF1FEA53F84F5091CF06852F9927B9
:109EE00022273327281B390B808191818217930702
:109EF00044F48091FE0683FF04C081E08093EE026B
:109F000016C08091EE02882391F0E42FFF27EE0F18
:109F1000FF1FEA53F84F8091D0069927851B9109BE
:109F2000208131818217930714F41092EE02509130
:109F30009406E52FFF27EE0FFF1FEA53F84F4091DD
:109F4000CF06242F3327808191812817390744F4C5
:109F50008091FE0680FF04C081E08093EC0217C070
:109F60008091EC02882399F0E52FFF27EE0FFF1F69
:109F7000EA53F84F842F99272091D006821B91092C
:109F8000208131812817390714F41092EC02409196
:109F90009406E42FFF27EE0FFF1FEA53F84F50916E
:109FA000CF06852F992722273327281B390B80813D
:109FB00091818217930744F48091FE0681FF04C0CB
:109FC00081E08093ED0216C08091ED02882391F02C
:109FD000E42FFF27EE0FFF1FEA53F84F8091D006C2
:109FE0009927851B9109208131818217930714F4E9
:109FF0001092ED028091EF02882319F48091EE0215
:10A00000811181E08093F0028091EC02882321F499
:10A010008091ED02882351F081E08093F10210924B
:10A02000F0021092EF021092EE0202C08093F10251
:10A030008091F002882321F48091F102882369F055
:10A040008091CE06992769817A818617970714F443
:10A050009A83898381E0809324038091D102992798
:10A060009C012470307082FF2DC08091EA03909192
:10A07000EB03909581959F4F90931F0380931E0350
:10A080008091E8039091E903909581959F4F90937B
:10A090001D0380931C038091A4019091A5019093CE
:10A0A000190380931803809182088B778B668093C5
:10A0B0008208809164088C7B8093640888EC80938C
:10A0C0009B011EC08091D20284FF1AC030931B03F3
:10A0D00020931A0330931F0320931E0330931D0314
:10A0E00020931C039AE59093910888E78093660873
:10A0F00090933F08809355081092F0021092F1025D
:10A100008091580890915908A0915A08B0915B0825
:10A110002091640330916503409166035091670379
:10A12000820F931FA41FB51F80935808909359085E
:10A13000A0935A08B0935B088091600890916108E1
:10A14000A0916208B091630820915C0330915D0397
:10A1500040915E0350915F03820F931FA41FB51FB0
:10A160008093600890936108A0936208B09363089D
:10A1700080914F0890915008A0915108B0915208D9
:10A180002091600330916103409162035091630319
:10A190002F83388749875A87820F931FA41FB51FC3
:10A1A00080934F0890935008A0935108B0935208A1
:10A1B0008091400890914108A0914208B0914308D5
:10A1C000409158035091590360915A0370915B0379
:10A1D0004B875C876D877E87840F951FA61FB71FEF
:10A1E0008093400890934108A0934208B09343089D
:10A1F0005091F1025F87552321F58091F002882369
:10A2000001F520E030E080916608882311F421E018
:10A2100030E040E050E08091EB02823310F441E006
:10A2200050E0242335238091A006992796958795A1
:10A23000969587958095909582239323892B09F491
:10A240005CC0109254031092550310925603109262
:10A250005703109250031092510310925203109220
:10A260005303109258081092590810925A081092ED
:10A270005B081092600810926108109262081092B8
:10A28000630810924F0810925008109251081092D3
:10A290005208109240081092410810924208109201
:10A2A00043088091440390914503A0914603B091E7
:10A2B00047038093400390934103A0934203B093DC
:10A2C000430380913C0390913D03A0913E03B091E4
:10A2D0003F038093380390933903A0933A03B093DC
:10A2E0003B0310921C0210921B021092F502109276
:10A2F000F4021092F7021092F60280916608882309
:10A3000009F05BC08091EB02823308F056C0809167
:10A31000A00682FD52C01092640310926503109251
:10A3200066031092670310925C0310925D03109213
:10A330005E0310925F031092440310924503109243
:10A3400046031092470310923C0310923D03109273
:10A350003E0310923F031092340310923503109283
:10A36000360310923703109248031092490310925B
:10A370004A0310924B038091B2019091B3019093E4
:10A38000270380932603AA2797FDA095BA2F209133
:10A390004501309146014091470150914801BC016F
:10A3A000CD010E94028FDC01CB0180939308909332
:10A3B0009408A0939508B09396086091A006688BC6
:10A3C00062FD04C08091EB02823318F0109266089F
:10A3D00004C080919401809366087F85772309F0FB
:10A3E00008C28091F002882309F003C280913506EB
:10A3F00090913606815092402CF480910D03882371
:10A4000009F4F7C190901C09A090AF06209086082F
:10A410003090870840909F085090A0086091640396
:10A4200070916503809166039091670320915C03AE
:10A4300030915D0340915E0350915F032F8B388F05
:10A44000498F5A8F19140CF0E1C0BB24CC24DD24B1
:10A45000A60195010E94768F79018A018091E50815
:10A460009091E608281A390AC101AA2797FDA095FC
:10A47000BA2FE81AF90A0A0B1B0B6F89788D898DA0
:10A480009A8DA60195010E94768F59016A018091EB
:10A49000E7089091E808481A590AC201AA2797FDCF
:10A4A000A095BA2FA81AB90ACA0ADB0A292C3324A4
:10A4B00027FC3094432C532CC801B701A201910111
:10A4C0000E94028F97FF04C061507E4F8F4F9F4FB5
:10A4D0003B014C0129E095948794779467942A95E1
:10A4E000D1F7C601B501A20191010E94028F97FF29
:10A4F00004C061507E4F8F4F9F4F5B016C0199E00C
:10A50000D594C794B794A7949A95D1F78091DB021C
:10A510009091DC02813491053CF48091D9029091B4
:10A52000DA0281349105D4F0D401C30197FE03C04F
:10A530000196A11DB11D3C014D019594879477941E
:10A540006794D601C501D7FE03C00196A11DB11DB8
:10A550005C016D01D594C794B794A7948091970638
:10A56000E82FFF27EE0FFF1FEA53F84F80819181FC
:10A570000190F081E02DF7FF03C0F095E195FF4FCA
:10A580007A97A4F0C401B30123E030E040E050E04A
:10A590000E94768F39014A01C601B50123E030E0FF
:10A5A00040E050E00E94768F59016A0180911E09B7
:10A5B000282F332727FD3095432F532F2615370596
:10A5C0004805590514F439014A01992787FD9095EA
:10A5D000909581959F4FAA2797FDA095BA2F681651
:10A5E00079068A069B0614F43C014D012A153B05A9
:10A5F0004C055D0514F459016A01A816B906CA068E
:10A60000DB060CF0CEC05C016D01CBC0EA2CFF2450
:10A6100000271127A80197010E94768F39014A016E
:10A62000C101AA2797FDA095BA2F681A790A8A0A4C
:10A630009B0A6F89788D898D9A8DA80197010E9458
:10A64000768F59016A01C201AA2797FDA095BA2FFA
:10A65000A81AB90ACA0ADB0AD401C30197FE03C0CB
:10A660000F96A11DB11D3C014D0114E095948794F6
:10A67000779467941A95D1F7D601C501D7FE03C028
:10A680000F96A11DB11D5C016D01B4E0D594C79476
:10A69000B794A794BA95D1F78091DB029091DC0230
:10A6A000813491053CF48091D9029091DA02813491
:10A6B0009105A4F0C401B30123E030E040E050E094
:10A6C0000E94768F39014A01C601B50123E030E0CE
:10A6D00040E050E00E94768F59016A018091970610
:10A6E000E82FFF27EE0FFF1FEA53F84F808191817B
:10A6F0000190F081E02DF7FF03C0F095E195FF4F49
:10A700007A97A4F0C401B30123E030E040E050E0C8
:10A710000E94768F39014A01C601B50123E030E07D
:10A7200040E050E00E94768F59016A0189E18093F0
:10A73000B00131E263167104810491042CF0A0E2AF
:10A740006A2E712C812C912C40EE64164FEF74060A
:10A750004FEF84064FEF940644F4F0EE6F2EFFEFB8
:10A760007F2EFFEF8F2EFFEF9F2E51E2A516B10433
:10A77000C104D1042CF0E0E2AE2EB12CC12CD12CBE
:10A7800060EEA6166FEFB6066FEFC6066FEFD60641
:10A7900044F470EEA72E7FEFB72E7FEFC72E7FEF2A
:10A7A000D72E8091440390914503A0914603B09128
:10A7B000470386199709A809B90980934403909320
:10A7C0004503A0934603B093470380913C039091C7
:10A7D0003D03A0913E03B0913F038A199B09AC0948
:10A7E000BD0980933C0390933D03A0933E03B09337
:10A7F0003F0380911B0290911C028F3F910509F04D
:10A8000008F4C9C57F85772309F053C58091F0020C
:10A81000882309F04EC580912403882309F049C597
:10A820008091D706898B882309F443C580916608F7
:10A83000882309F43EC58091580890915908A09149
:10A840005A08B0915B08B7FF04C081509F4FAF4FCB
:10A85000BF4FE92EFA2E0B2F112707FD1A95E09214
:10A860005808F092590800935A0810935B08809199
:10A87000600890916108A0916208B0916308B7FFE9
:10A8800004C081509F4FAF4FBF4F892F9A2FAB2FDE
:10A89000BB27A7FDBA958A8B9B8BAC8BBD8B809316
:10A8A000600890936108A0936208B0936308809158
:10A8B000AF06A82EBB24CC24DD2420915403309174
:10A8C00055034091560350915703C601B5010E94AC
:10A8D000028F97FF04C061507F4F8F4F9F4F672EAD
:10A8E000782E892E992487FC9A9460925403709252
:10A8F0005503809256039092570320915003309154
:10A9000051034091520350915303C601B5010E9477
:10A91000028F97FF04C061507F4F8F4F9F4F272EAC
:10A92000382E492E552447FC5A94209250033092D9
:10A930005103409252035092530380914C039091E3
:10A940004D03A0914E03B0914F03B7FF04C0815057
:10A950009F4FAF4FBF4F892F9A2FAB2FBB27A7FD1C
:10A96000BA9580934C0390934D03A0934E03B093FC
:10A970004F03D801C70186199709A809B90980931F
:10A98000B6039093B703A093B803B093B903209193
:10A99000D606E22EFF2400271127BC01CD01A80115
:10A9A00097010E94768F59016A012093C303309367
:10A9B000C4034093C5035093C6038A899B89AC891D
:10A9C000BD8982199309A409B5098093BA039093AC
:10A9D000BB03A093BC03B093BD03BC01CD01A80190
:10A9E00097010E94768F2093C7033093C80340934A
:10A9F000C9035093CA03D601C501D7FE04C08150D4
:10AA00009F4FAF4FBF4F892F9A2FAB2FBB27A7FD6B
:10AA1000BA959093F5028093F40257FF04C0215039
:10AA20003F4F4F4F5F4FBB2757FDBA95A52F942F30
:10AA3000832F9093F7028093F6028091DB0290912E
:10AA4000DC0281349105DCF48091D9029091DA0224
:10AA500081349105A4F480919706E82FFF27EE0F2B
:10AA6000FF1FEA53F84F808191810190F081E02D22
:10AA7000F7FF03C0F095E195FF4F7A97E4F08091DE
:10AA80001C098F3FC1F48091F4029091F50297FD6B
:10AA90000196959587959093F5028093F4028091A5
:10AAA000F6029091F70297FD019695958795909300
:10AAB000F7028093F60280914F0890915008A09180
:10AAC0005108B0915208B7FF04C081509F4FAF4F5B
:10AAD000BF4F892F9A2FAB2FBB27A7FDBA95809325
:10AAE0004F0890935008A0935108B093520880915A
:10AAF000400890914108A0914208B0914308B7FFE7
:10AB000004C081509F4FAF4FBF4F892F9A2FAB2F5B
:10AB1000BB27A7FDBA958093400890934108A09366
:10AB20004208B09343088091640390916503A0911B
:10AB30006603B09167032F81388549855A85281BA4
:10AB4000390B4A0B5B0B2093AE033093AF0340935A
:10AB5000B0035093B10380915C0390915D03A09189
:10AB60005E03B0915F03EB84FC840D851E85E81ABB
:10AB7000F90A0A0B1B0BE092B203F092B3030093A5
:10AB8000B4031093B5032093B6033093B7034093F7
:10AB9000B8035093B903E092BA03F092BB03009359
:10ABA000BC031093BD038091400390914103A09199
:10ABB0004203B0914303821B930BA40BB50B80930C
:10ABC000400390934103A0934203B09343038091C9
:10ABD000380390913903A0913A03B0913B038E1949
:10ABE0009F09A00BB10B8093380390933903A09376
:10ABF0003A03B0933B0399899923E1F02091220312
:10AC000030912303213831054CF0809175039091E8
:10AC100076030196909376038093750320583F4FF7
:10AC20004CF480917503909176030197909376038D
:10AC300080937503109223031092220381E090E029
:10AC40009093D0038093CF03E090B603F090B703C6
:10AC50000091B8031091B903D801C70117FF07C0CD
:10AC600088279927DC018E199F09A00BB10B815011
:10AC70009240A040B04034F084E090E09093D00344
:10AC80008093CF038091D5039091D603A091D703F1
:10AC9000B091D803209158083091590840915A0832
:10ACA00050915B08821B930BA40BB50B815E914BFB
:10ACB000AF4FBF4F8F539C49A040B04028F08091C8
:10ACC0001D0989310CF4FFC021E0E21620E1F206F3
:10ACD00020E0020720E012070CF473C08091D1033A
:10ACE000882309F46AC0D801C70117FF07C0882765
:10ACF0009927DC018E199F09A00BB10B9C01AD01B6
:10AD0000B7FF04C021503E4F4F4F5F4F69E055954C
:10AD10004795379527956A95D1F78091CF03909104
:10AD2000D003820F931F9093D0038093CF03D80159
:10AD3000C70117FF03C00796A11DB11D23E0B595FC
:10AD4000A795979587952A95D1F78093C3039093FC
:10AD5000C403A093C503B093C60389589341A04090
:10AD6000B04064F088E893E1A0E0B0E08093C303D2
:10AD70009093C403A093C503B093C6032091C3036B
:10AD80003091C4034091C5035091C60357FF04C0DE
:10AD900021503F4F4F4F5F4F232F342F452F5527C3
:10ADA00047FD5A958091F4029091F502820F931F0E
:10ADB0009093F5028093F40206C081E08093D10362
:10ADC00002C01092D10340E0E41640EFF4064FEFCA
:10ADD00004074FEF14070CF073C08091D20388234F
:10ADE00009F46AC0D801C70117FF07C0882799274F
:10ADF000DC018E199F09A00BB10B9C01AD01B7FFBF
:10AE000004C021503E4F4F4F5F4F89E05595479505
:10AE1000379527958A95D1F78091CF039091D003EC
:10AE2000820F931F9093D0038093CF03D801C70163
:10AE300017FF03C00796A11DB11D13E0B595A79597
:10AE4000979587951A95D1F78093C3039093C40380
:10AE5000A093C503B093C60388579C4EAF4FBF4F16
:10AE600064F488E79CEEAFEFBFEF8093C303909349
:10AE7000C403A093C503B093C6032091C3033091CC
:10AE8000C4034091C5035091C60357FF04C021502D
:10AE90003F4F4F4F5F4F232F342F452F552747FDEF
:10AEA0005A958091F4029091F502820F931F90932E
:10AEB000F5028093F40211C081E08093D2030DC0AB
:10AEC0001092D2030AC01092D0031092CF0384E6EE
:10AED00090E09093AF018093AE016989262F3327CC
:10AEE0008091CF039091D0032817390724F4309331
:10AEF000D0032093CF0310911D09112379F0212F46
:10AF0000332727FD30958091CF039091D0032817E8
:10AF1000390724F43093D0032093CF034091B60334
:10AF20005091B7036091B8037091B903413851054E
:10AF30006105710574F08091790390917A032091F5
:10AF4000CF033091D003820F931F90937A038093A5
:10AF5000790340585F4F6F4F7F4F74F480917903AE
:10AF600090917A032091CF033091D003821B930BF1
:10AF700090937A038093790381E090E09093D003DB
:10AF80008093CF03C090BA03D090BB03E090BC0382
:10AF9000F090BD03D701C601F7FE07C088279927A7
:10AFA000DC018C199D09AE09BF0981509240A04077
:10AFB000B04034F084E090E09093D0038093CF03CE
:10AFC0008091D9039091DA03A091DB03B091DC0367
:10AFD00020916008309161084091620850916308A7
:10AFE000821B930BA40BB50B815E914BAF4FBF4FF0
:10AFF0008F539C49A040B04018F019310CF4FFC0A9
:10B0000021E0C21620E1D20620E0E20620E0F206AE
:10B010000CF473C08091D303882309F46AC0D7016C
:10B02000C601F7FE07C088279927DC018C199D0906
:10B03000AE09BF099C01AD01B7FF04C021503E4FCE
:10B040004F4F5F4FF9E05595479537952795FA95FE
:10B05000D1F78091CF039091D003820F931F9093EB
:10B06000D0038093CF03D701C601F7FE03C0079634
:10B07000A11DB11DE3E0B595A79597958795EA9534
:10B08000D1F78093C7039093C803A093C903B093EB
:10B09000CA0389589341A040B04064F088E893E126
:10B0A000A0E0B0E08093C7039093C803A093C903C6
:10B0B000B093CA032091C7033091C8034091C903DC
:10B0C0005091CA0357FF04C021503F4F4F4F5F4F6D
:10B0D000232F342F452F552747FD5A958091F6028F
:10B0E0009091F702820F931F9093F7028093F602DC
:10B0F00006C081E08093D30302C01092D30340E0E6
:10B10000C41640EFD4064FEFE4064FEFF4060CF000
:10B1100073C08091D403882309F46AC0D701C601A3
:10B12000F7FE07C088279927DC018C199D09AE0915
:10B13000BF099C01AD01B7FF04C021503E4F4F4FE6
:10B140005F4F69E055954795379527956A95D1F7F3
:10B150008091CF039091D003820F931F9093D003DF
:10B160008093CF03D701C601F7FE03C00796A11D48
:10B17000B11D23E0B595A795979587952A95D1F7A9
:10B180008093C7039093C803A093C903B093CA03E5
:10B1900088579C4EAF4FBF4F64F488E79CEEAFEFEB
:10B1A000BFEF8093C7039093C803A093C903B093E4
:10B1B000CA032091C7033091C8034091C90350913D
:10B1C000CA0357FF04C021503F4F4F4F5F4F232FFB
:10B1D000342F452F552747FD5A958091F6029091BF
:10B1E000F702820F931F9093F7028093F60211C02B
:10B1F00081E08093D4030DC01092D4030AC0109252
:10B20000D0031092CF0384E690E09093AF01809337
:10B21000AE016989262F33278091CF039091D00307
:10B220002817390724F43093D0032093CF0380915B
:10B230001D09882379F0282F332727FD3095809129
:10B24000CF039091D0032817390724F43093D0030B
:10B250002093CF034091BA035091BB036091BC038C
:10B260007091BD03413851056105710574F08091FD
:10B270007703909178032091CF033091D003820F10
:10B28000931F909378038093770340585F4F6F4FDD
:10B290007F4FCCF480917703909178032091CF0376
:10B2A0003091D003821B930B9093780380937703A4
:10B2B0000AC01092F7021092F6021092F502109254
:10B2C000F4021092240380916608882341F41092BE
:10B2D000F7021092F6021092F5021092F402809199
:10B2E000580890915908A0915A08B0915B08809332
:10B2F000D5039093D603A093D703B093D80380913E
:10B30000600890916108A0916208B09163088093F1
:10B31000D9039093DA03A093DB03B093DC0310927C
:10B320005403109255031092560310925703109233
:10B330005003109251031092520310925303109233
:10B340004C0310924D0310924E0310924F03109233
:10B3500058081092590810925A0810925B081092DF
:10B3600060081092610810926208109263081092AF
:10B370004F081092500810925108109252081092E3
:10B38000400810924108109242081092430810920F
:10B390001C0210921B02E0901A03F0901B03C701DD
:10B3A000F7FE04C0882799278E199F0904973CF05F
:10B3B0008091820884FD03C082E38093F80210919B
:10B3C000AC06A12EBB24CC24DD24B701882777FD51
:10B3D0008095982F9701F7FE04C0222733272E1956
:10B3E0003F09442737FD4095542F0E94028F9B014F
:10B3F000AC01C601B5010E94028F97FF04C06150E5
:10B400007E4F8F4F9F4F09E095958795779567956C
:10B410000A95D1F77C8F6B8F812F99278E9DD00154
:10B420008F9DB00D9E9DB00D1124CD01B7FD0396EB
:10B430009595879595958795EB8DFC8DE80FF91F70
:10B44000FC8FEB8F8091FA029091FB02E80FF91FBD
:10B45000CF01AA2797FDA095BA2F8093AA039093B6
:10B46000AB03A093AC03B093AD039F01A3E0220F05
:10B47000331FAA95E1F72E0F3F1F2E0F3F1F37FFF7
:10B4800002C0295F3F4FE3E035952795EA95E1F744
:10B49000442737FD4095542F809134039091350314
:10B4A000A0913603B0913703821B930BA40BB50B0D
:10B4B0008093340390933503A0933603B0933703FE
:10B4C00081599F45A140B04064F080E99FE5A1E02B
:10B4D000B0E08093340390933503A0933603B09388
:10B4E00037038091340390913503A0913603B091D6
:10B4F00037038057904AAE4FBF4F64F480E790EA1D
:10B50000AEEFBFEF8093340390933503A0933603DF
:10B51000B09337030091B2011091B30117FD00C140
:10B52000388933FFFDC08091EB02833308F0F8C007
:10B530008091B10181508093B101882309F0F4C05A
:10B540008DE08093B1018091640390916503A09197
:10B550006603B0916703B7FF04C081509E4FAF4FA1
:10B56000BF4F79E0B595A795979587957A95D1F7CF
:10B570007C0197FF04C0F094E194F108F39480916A
:10B580005C0390915D03A0915E03B0915F03B7FFF0
:10B5900004C081509E4FAF4FBF4F69E0B595A7954E
:10B5A000979587956A95D1F79C0197FF03C03095D1
:10B5B00021953F4FE216F3060CF47901B701F7FE2F
:10B5C00002C0695F7F4F2B0153E0559447945A9511
:10B5D000E1F742E050E0440E551E609093087090F1
:10B5E000940880909508909096082091450130919C
:10B5F00046014091470150914801C401B3010E94A6
:10B60000768F59016A0130933E0820933D08021B52
:10B61000130BC801845E9D4F68E671E00E94418F64
:10B620009C01245B30408091AE019091AF01009766
:10B6300031F001979093AF018093AE011BC059E1A7
:10B64000E516F104BCF48091220390912303820F4C
:10B65000931F90932303809322038091F802882301
:10B6600049F081508093F802882321F4B092270397
:10B67000A09226038091AE019091AF01892BF9F43D
:10B680008091B0019927289FB001299F700D389FA4
:10B69000700D1124CB01B2010E94418FCB01AA276A
:10B6A00097FDA095BA2F680E791E8A1E9B1E609288
:10B6B00093087092940880929508909296088091D1
:10B6C000F802882369F58091260390912703209141
:10B6D0003D0830913E08821B930B845E9D4F68E6C7
:10B6E00071E00E94418F9C01245B30408091980161
:10B6F00086959927289FD001299FB00D389FB00DBE
:10B7000011249D01B7FF02C0215F3F4F44E03595F2
:10B7100027954A95E1F73093FB022093FA0204C083
:10B720001092FB021092FA0280912403882381F088
:10B7300010922C0310922D0310922E0310922F03BF
:10B74000109230031092310310923203109233039F
:10B75000F090F102FF20F9F480916608282F33273A
:10B76000442755278091640390916503A091660357
:10B77000B0916703BC01CD010E94028FDC01CB01B7
:10B78000BC01CD0128EF3AE240E050E00E94768F04
:10B790003C832B8302C01C821B821091F002112378
:10B7A000F9F480916608282F332744275527809184
:10B7B0005C0390915D03A0915E03B0915F03BC01B7
:10B7C000CD010E94028FDC01CB01BC01CD0128EF2D
:10B7D0003AE240E050E00E94768F3E832D8302C023
:10B7E0001E821D828091390890913A08893C91050A
:10B7F0001CF088EC90E005C088539F4F34F488E338
:10B800009FEF90933A088093390880914608909171
:10B810004708893C91051CF088EC90E005C08853EE
:10B820009F4F34F488E39FEF909347088093460836
:10B8300080916608209191086091480870914908AC
:10B84000882309F040C0CB01AA2797FDA095BA2F05
:10B85000A22EBB24CC24DD24BC01CD01A601950180
:10B860000E94028F97FF04C0615C7F4F8F4F9F4FF4
:10B8700036E095958795779567953A95D1F77093CA
:10B880004908609348088091370890913808AA27A2
:10B8900097FDA095BA2FBC01CD01A60195010E948C
:10B8A000028F97FF04C0615C7F4F8F4F9F4F26E050
:10B8B00095958795779567952A95D1F77093380870
:10B8C0006093370871C0CB01AA2797FDA095BA2FC6
:10B8D000A22EBB24CC24DD24BC01CD01A601950100
:10B8E0000E94028F9B01AC018091390890913A0827
:10B8F000AA2797FDA095BA2F07E0880F991FAA1FC6
:10B90000BB1F0A95D1F7280F391F4A1F5B1F57FF2E
:10B9100004C0215C3F4F4F4F5F4FA6E055954795C0
:10B9200037952795AA95D1F78B819C81820F931F1C
:10B93000909349088093480880913708909138087F
:10B94000AA2797FDA095BA2FBC01CD01A6019501AC
:10B950000E94028F9B01AC0180914608909147089C
:10B96000AA2797FDA095BA2FF7E0880F991FAA1F65
:10B97000BB1FFA95D1F7280F391F4A1F5B1F57FFCE
:10B9800004C0215C3F4F4F4F5F4FE6E05595479510
:10B9900037952795EA95D1F78D819E81820F931F68
:10B9A000909338088093370880918C0890918D0887
:10B9B000880F991FAA2797FDA095BA2F20913F08BD
:10B9C000332744275527BC01CD010E94028F5B011C
:10B9D0006C0197FF08C02FE330E040E050E0A20E7A
:10B9E000B31EC41ED51E76E0D594C794B794A79411
:10B9F0007A95D1F780915508282F3327442755276A
:10BA00008091480390914903A0914A03B0914B0360
:10BA1000BC01CD010E94028FDC01CB01BC01CD0134
:10BA200020EF35E540E050E00E94768FB501620FCF
:10BA3000731F70938D0860938C08809148089091D3
:10BA400049088150904134F080E090E1909349089A
:10BA50008093480880914808909149088050904F01
:10BA600034F480E090EF90934908809348088091E7
:10BA70003708909138088150904134F080E090E18F
:10BA80009093380880933708809137089091380850
:10BA90008050904F34F480E090EF9093380880937A
:10BAA00037086150704134F080E090E190938D0848
:10BAB00080938C0880918C0890918D088050904FD5
:10BAC00034F480E090EF90938D0880938C088091FF
:10BAD0000001482F5527809120019091210148179E
:10BAE000590794F4209120013091210169817A81D4
:10BAF000649FC001659F900D749F900D1124B90142
:10BB00000E942D8F7A83698389819A81880F991F7A
:10BB1000880F991F9A8389834091820840FD02C053
:10BB20000C94BD65112311F00C94BD65FF2011F03C
:10BB30000C94BD6500E010E028018091F202909124
:10BB4000F30290931D0680931C0620917B03309195
:10BB50007C032115310509F03FC0809116019091B9
:10BB600017018959934058F087B5803F20F48091A0
:10BB70001F02815011C081E08093E6034EC0809186
:10BB80001601909117018436910508F587B580312B
:10BB9000D0F080911F028F5F80931F029FE0890287
:10BBA0009001112480913F06821B87BD8CE291E0B9
:10BBB00090930D0280930C028EE591E090937C03AC
:10BBC00080937B032AC081E08093E50326C0F09236
:10BBD000E503F092E60321C08091080390910903E8
:10BBE000A0910A03B0910B0354E0880F991FAA1F7C
:10BBF000BB1F5A95D1F78093200290932102A09306
:10BC00002202B093230210931E0200931D022150C2
:10BC1000304030937C0320937B0320919B0141FFB4
:10BC200029C0223320F08091EB028D38E0F0809122
:10BC3000C10181508093C1018F3F09F042C0109231
:10BC400025038091080390910903A0910A03B09104
:10BC50000B038093040390930503A0930603B09312
:10BC6000070381E004C081E08093250388EC809382
:10BC7000C10127C08091490190914A01820F911D15
:10BC80002091A5063327829FF001839FF00D929F9C
:10BC9000F00D1124CF01AA2797FDA095BA2F80930C
:10BCA000040390930503A0930603B09307038091C8
:10BCB000EB028D3818F01092250303C081E08093C9
:10BCC00025038091640390916503A0916603B09170
:10BCD0006703E0904501F090460100914701109103
:10BCE0004801BC01CD01A80197010E94768F59013E
:10BCF0006A0180915C0390915D03A0915E03B09115
:10BD00005F03BC01CD01A80197010E94768FB901A4
:10BD1000C5010E942B831C01CC971CF0ACE32A2E9A
:10BD2000312CC1010E943E731C0180E280934401CA
:10BD3000109203031092020380912503882309F4D3
:10BD40008EC58091D20299279C012071307084FDAC
:10BD500086C58091D10282608093D102709164087F
:10BD600070FD04C08091820881FD10C0E980FA80D6
:10BD70003093DE032093DD0330930303209302030B
:10BD80008091D202806C8093D202E0C200910803BD
:10BD9000109109038091040390910503081B190B6E
:10BDA0008091D20281FFA5C2E090A401F090A5018C
:10BDB000C7010F96C0901803D09019038C159D05EC
:10BDC0000CF063C08091E503882309F05EC0809188
:10BDD000D20287FF24C08091D2028F778093D20253
:10BDE000980117FF02C02F5F3F4F359527954427D5
:10BDF00037FD4095542F8091080390910903A0913D
:10BE00000A03B0910B03821B930BA40BB50B809319
:10BE1000040390930503A0930603B0930703809156
:10BE2000D20280648093D202109144081123F1F071
:10BE30008091040390910503A0910603B09107033C
:10BE4000BC01CD0124E630E040E050E00E94768F56
:10BE5000812F9927AA27BB2782179307A407B50725
:10BE60002CF410920303109202035AC0C6018E19DB
:10BE70009F090F9797FF03C0909581959F4F9093CF
:10BE80000303809302038BE249C0C7010F97C816D2
:10BE9000D9060CF048C08091E603882309F043C01E
:10BEA0008091D20286FF24C08091D2028F7B809342
:10BEB000D202980117FF02C02F5F3F4F359527959B
:10BEC000442737FD4095542F809108039091090332
:10BED000A0910A03B0910B03821B930BA40BB50B2B
:10BEE0008093040390930503A0930603B093070384
:10BEF0008091D20280688093D202C6018E199F0978
:10BF00000F9697FF03C0909581959F4F90958195CF
:10BF10009F4F90930303809302038DE2809344012B
:10BF20001092FC02E8C08DE3809344016091FD0211
:10BF3000662371F12091FE023091FF0240910003CF
:10BF4000509101038091040390910503A091060391
:10BF5000B091070382179307A407B507CCF480912B
:10BF6000D20280648093D202862F99279093030394
:10BF7000809302038AE08093FC028EE58093440163
:10BF80008091D20287FFB7C08091D2028F7733C0F1
:10BF9000662309F452C02091FE023091FF024091C5
:10BFA0000003509101038091040390910503A09137
:10BFB0000603B0910703281739074A075B07ECF51A
:10BFC0008091D20280688093D202862F9927909523
:10BFD00081959F4F909303038093020386EF809394
:10BFE000FC0286E7809344018091D20286FF83C0E1
:10BFF0008091D2028F7B8093D202980117FF02C0FA
:10C000002F5F3F4F35952795442737FD4095542F97
:10C010008091080390910903A0910A03B0910B034A
:10C02000821B930BA40BB50B809304039093050321
:10C03000A0930603B09307035EC08091D202807C78
:10C0400009F459C08091FC02882379F5E090080337
:10C05000F090090300910A0310910B03D801C70166
:10C0600080589040A040B0402091040330910503D7
:10C07000409106035091070382179307A407B50761
:10C080005CF4D801C70180589F4FAF4FBF4F2817AE
:10C0900039074A075B075CF080930403909305031C
:10C0A000A0930603B093070302C01092FC02809194
:10C0B000D2028F738093D2021092DE031092DD03BE
:10C0C00071FF06C084EF91E090930D0280930C0203
:10C0D00080910C03882379F48091080390910903DF
:10C0E000A0910A03B0910B03C397A105B1051CF001
:10C0F00081E080930C036091DD037091DE038091F9
:10C10000020390910303680F791F7093DE0360931D
:10C11000DD03CB0177FF04C088279927861B970B87
:10C12000855F91400CF4CEC04091FC02442389F11C
:10C130008091FE029091FF0220910403309105034B
:10C14000821B930B0996439748F48091FE029091CD
:10C15000FF02A0910003B091010312C0242F3327E6
:10C1600027FD3095432F532F8091040390910503B1
:10C17000A0910603B0910703820F931FA41FB51F60
:10C180008093040390930503A0930603B0930703E1
:10C1900024C08091A50620910403309105034091AD
:10C1A0000603509107031616170644F463E00E9435
:10C1B000218F280F311D411D511D07C063E00E94D2
:10C1C000218F281B31094109510920930403309321
:10C1D000050340930603509307031092DE03109269
:10C1E000DD03E0900803F090090300910A03109129
:10C1F0000B03D801C70180509440A040B04020916B
:10C200000403309105034091060350910703821700
:10C210009307A407B5075CF4D801C70180509C4F71
:10C22000AF4FBF4F281739074A075B0744F0809389
:10C23000040390930503A0930603B0930703809132
:10C24000640881FF06C084E690E090930D0280931D
:10C250000C028091A9068823A9F58091FD0288230C
:10C2600089F54091F2025091F30257FF02C04D5FF1
:10C270005F4F559547955595479580912001909131
:10C280002101209100013327489FB001499F700D83
:10C29000589F700D1124CB01B9010E94418F7093FA
:10C2A000A5016093A401663471051CF486E490E056
:10C2B00005C06739710534F086E990E09093A501D7
:10C2C0008093A40180917B0390917C03892BD1F111
:10C2D0008091080390910903A0910A03B0910B0388
:10C2E0008093040390930503A0930603B093070380
:10C2F00029C08091080390910903A0910A03B0918D
:10C300000B0380599140A040B04080930403909368
:10C310000503A0930603B09307038091A906882321
:10C3200011F0992702C088E790E09093A5018093CF
:10C33000A40189819A819093F3028093F2028EE2A4
:10C3400080934401E090F202F090F302A090080381
:10C35000B0900903C0900A03D0900B0360900403CF
:10C360007090050380900603909007036A147B0485
:10C370008C049D0424F08091640880FDBCC28091EF
:10C380007B0390917C03892B39F0E090F202F090CE
:10C39000F30200E010E03EC1D601C50186199709FD
:10C3A000A809B9098093AE039093AF03A093B0039B
:10C3B000B093B1038230E0E89E07EFEFAE07EFEFF6
:10C3C000BE072CF481E090E8AFEFBFEF09C08F5FAC
:10C3D0009F47A040B04064F08FEF9FE7A0E0B0E03F
:10C3E0008093AE039093AF03A093B003B093B103D7
:10C3F0000091AE031091AF03D601C501805C9F4F41
:10C40000AF4FBF4F86159705A805B9055CF0D6015B
:10C41000C50180549040A040B040681679068A0655
:10C420009B06DCF480919A01282F33274427552757
:10C430008091AE039091AF03A091B003B091B1038E
:10C44000BC01CD010E94028FDC01CB01BC01CD01FA
:10C4500026E430E040E050E01AC080919A01282F95
:10C460003327442755278091AE039091AF03A091C5
:10C47000B003B091B103BC01CD010E94028FDC0179
:10C48000CB01BC01CD012AE530E040E050E00E9444
:10C49000768F2093AE033093AF034093B003509355
:10C4A000B1038091AE039091AF03A091B003B0911E
:10C4B000B10381302EEF92072FEFA2072FEFB207C3
:10C4C0002CF480E09EEFAFEFBFEF09C080509240A8
:10C4D000A040B04064F080E092E0A0E0B0E0809343
:10C4E000AE039093AF03A093B003B093B103409019
:10C4F000AE035090AF0360911D0270911E0277FF52
:10C5000002C06D5F7F4F75956795759567957C8FB8
:10C510006B8FD601C50180509E4FAF4FBF4F861520
:10C520009705A805B9056CF040E05EEF6FEF7FEF6F
:10C53000A40EB51EC61ED71E6A147B048C049D046F
:10C540006CF4C8016CE170E00E94418FCB016B8DEF
:10C550007C8D680F791F7C8F6B8F0EC0C80117FD13
:10C560004F9635E0959587953A95E1F7AB8DBC8D63
:10C57000A80FB91FBC8FAB8FEB8DFC8DE258FF4F1E
:10C580002CF441E85FEF5C8F4B8F09C06B8D7C8D85
:10C590006038710524F080E890E09C8F8B8FEB8DE4
:10C5A000FC8DCF01AA2797FDA095BA2F20919C0161
:10C5B000332744275527BC01CD010E94028F97FFE6
:10C5C00004C06D5F7F4F8F4F9F4F22E095958795F9
:10C5D000779567952A95D1F77C8F6B8F61507F4F48
:10C5E0002CF420E03FEF3C8F2B8F0AC04B8D5C8DED
:10C5F0004F3F510529F024F060E071E07C8F6B8F94
:10C600008B8D9C8D97FD0396959587959595879530
:10C61000480E591E80919701282F332780912009B9
:10C62000992787FD9095289FD001299FB00D389FAD
:10C63000B00D11249D01B7FF02C021583F4F220FBA
:10C64000232F221F330B3C8F2B8F21583F4F2CF46D
:10C65000E0E8FFEFFC8FEB8F09C02B8D3C8D20387D
:10C66000310524F040E850E05C8F4B8F6B8D7C8D62
:10C67000460E571EC201AA2797FDA095BA2FC0905B
:10C68000F202D090F3029601442737FD4095542FD3
:10C69000BC01CD010E94028F97FF04C061507E4F04
:10C6A0008F4F9F4FF9E09595879577956795FA9508
:10C6B000D1F7E61AF70A8091020390910303892BC0
:10C6C00009F060C01C141D040CF05CC0980117FF39
:10C6D00003C0309521953F4F2D33310540F48091B3
:10C6E0002003909121038E159F0574F526C02C53CD
:10C6F0003040E5E036952795EA95E1F720313105A0
:10C7000010F02FE030E040912003509121031016EB
:10C710001106E4F480E190E0821B930B489F9001A6
:10C72000499F300D589F300D112474E036952795A0
:10C730007A95E1F72E153F0520F58091A2019091A1
:10C74000A301E816F906F4F07C011CC0205F3F4FFE
:10C750008091A2019091A301829FD001839FB00D8F
:10C76000929FB00D11249D0164E0369527956A953E
:10C77000E1F74E155F0514F07A0104C0E216F306E6
:10C7800008F07901C701AA2797FDA095BA2F5DE0AF
:10C79000880F991FAA1FBB1F5A95D1F791014427F3
:10C7A00037FD4095542FBC01CD010E94768F209318
:10C7B000B2033093B3034093B4035093B503E090B6
:10C7C000B203F090B3038091DF039091E0039C01EA
:10C7D000220F331F280F391F2E0D3F1D37FF02C0B8
:10C7E0002D5F3F4FA9015595479555954795509316
:10C7F000E0034093DF038091A106282F3327220F07
:10C80000331F220F331F241735076CF480918A08D9
:10C81000282F3327220F331F220F331F205530407C
:10C820004217530724F03093E0032093DF038091F5
:10C8300064082091DF033091E00380FF0DC0E9819F
:10C84000FA812E173F0724F0F093E003E093DF0313
:10C850002091DF033091E0033A8329834CC080911B
:10C86000A906882301F56091F2027091F30277FF27
:10C8700002C06D5F7F4F759567957595679540917F
:10C8800020015091210180910001282F3327649FBE
:10C89000C001659F900D749F900D1124B9010E94F5
:10C8A000418FCB0101C099279093A5018093A401EA
:10C8B0008091A4019091A501873491051CF486E430
:10C8C00090E005C08639910534F086E990E09093B8
:10C8D000A5018093A40149815A815093E0034093BC
:10C8E000DF038091D202806C8093D2028091D102CA
:10C8F0008D7F8093D1028091D20299279C01227072
:10C90000307081FF2BC18091E1039091E203A091EF
:10C91000E303B091E4030097A105B10521F08091F4
:10C920000C038130B1F469817A81CB01AA2797FD8C
:10C93000A095BA2F1EE0880F991FAA1FBB1F1A953A
:10C94000D1F78093E1039093E203A093E303B093C4
:10C95000E40380910C03813019F482E080930C038E
:10C96000E981FA81CF01AA2797FDA095BA2F9101FD
:10C97000442737FD4095542FBC01CD010E94028F02
:10C98000DC01CB018093B2039093B303A093B40373
:10C99000B093B503B7FF04C08150904EAF4FBF4F67
:10C9A0007C018D01FDE015950795F794E794FA95C4
:10C9B000D1F7E092B203F092B3030093B403109363
:10C9C000B5036091D3027091D402FFE0603A7F0713
:10C9D00050F58091E1039091E203A091E303B091BF
:10C9E000E4039C01AD01EAE05695479537952795FC
:10C9F000EA95D1F7821B930BA40BB50BA801970105
:10CA0000F4E0220F331F441F551FFA95D1F7820F10
:10CA1000931FA41FB51F8093E1039093E203A0939B
:10CA2000E303B093E40360547F4118F58091E10380
:10CA30009091E203A091E303B091E4039C01AD0166
:10CA4000ECE05695479537952795EA95D1F7821BE7
:10CA5000930BA40BB50BA801970172E0220F331FB3
:10CA6000441F551F7A95D1F7820F931FA41FB51F3E
:10CA700038C080911D0290911E0280911D029091FC
:10CA80001E0297FF03C0909581959F4F84369105B4
:10CA900084F580910803909109032091040330915B
:10CAA0000503821B930B81509F4F8F5F914008F5C8
:10CAB0008091E1039091E203A091E303B091E4033C
:10CAC0009C01AD016EE056954795379527956A957F
:10CAD000D1F7821B930BA40BB50B8E0D9F1DA01FCE
:10CAE000B11F8093E1039093E203A093E303B0931B
:10CAF000E4038091E1039091E203A091E303B091FC
:10CB0000E4031EE0B695A795979587951A95D1F7FA
:10CB10009093F3028093F2024091A706442399F088
:10CB200055279C01BA010E94418FC901861B970BB2
:10CB30009093210380932003260F371F3093A30186
:10CB40002093A2011FC010922103109220038FEFA7
:10CB500093E09093A3018093A20114C010920C0360
:10CB60001092E1031092E2031092E3031092E403A7
:10CB70003093F3022093F20205C08091D202806CC0
:10CB80008093D2028091F50381FF37C089819A8119
:10CB900097FD039695958795959587952091CF025A
:10CBA0003091D0022817390760F48091F2029091F9
:10CBB000F302892B31F0220F331F220F331F3A83E8
:10CBC00029838091080390910903A0910A03B091F1
:10CBD0000B038093040390930503A0930603B09383
:10CBE000070388E99AE390930D0280930C0280E09A
:10CBF0009EE0909309018093080120914D08822FB7
:10CC00009927880F991F880F991F889649815A8103
:10CC10008417950714F09A83898350918A085E8B54
:10CC2000852F9927880F991F880F991F805590404D
:10CC300069817A818617970714F49A838983809192
:10CC40005302882341F4809134098F3F21F480916D
:10CC5000F9038823D9F08091D3029091D4020297EE
:10CC6000C097A0F489819A81181619067CF481E096
:10CC700090E09093D4028093D302A22FBB27AA0FF7
:10CC8000BB1FAA0FBB1F9896BA83A983E981FA81BB
:10CC9000F0930106E09300068091AA039091AB0304
:10CCA000A091AC03B091AD0362E0880F991FAA1F59
:10CCB000BB1F6A95D1F700918C0810918D08081B55
:10CCC000190BE13AF1058CF0CF01F7FD019695952E
:10CCD0008795801791070CF48C01909581959F4F53
:10CCE000081719076CF48C010BC00135110514F0FD
:10CCF00000E510E0FFEF003B1F0714F400EB1FEF0F
:10CD00002E893327220F331F220F331F3C8F2B8F87
:10CD1000C90149815A81841B950B801791070CF436
:10CD20008C0129813A816B8D7C8D261B370B021774
:10CD300013070CF489012091480830914908A0910B
:10CD40001E03B0911F032A1B3B0B309357082093FF
:10CD50005608409137085091380860901C03709035
:10CD60001D034619570950933608409335088091A2
:10CD7000B606893008F5682F7727629FC001639F48
:10CD8000900D729F900D112497FD07964C0133E092
:10CD9000959487943A95E1F7649FC001659F900D43
:10CDA000749F900D112497FD07967C0123E0F59464
:10CDB000E7942A95E1F71FC08695682F7727629F31
:10CDC000C001639F900D729F900D112497FD0396F3
:10CDD0004C019594879495948794649FC001659FB6
:10CDE000900D749F900D112497FD03967C01F5948E
:10CDF000E794F594E79480916608882309F4C9C004
:10CE00008B819C818A1B9B0B9C01442737FD40959D
:10CE1000542F8091300390913103A0913203B0914F
:10CE20003303820F931FA41FB51F80933003909389
:10CE30003103A0933203B093330381509D47A04048
:10CE4000B04064F080E09DE7A0E0B0E08093300364
:10CE500090933103A0933203B09333038091300356
:10CE600090913103A0913203B091330380509348E5
:10CE7000AF4FBF4F64F480E093E8AFEFBFEF809314
:10CE8000300390933103A0933203B0933303809126
:10CE90009F019091A0015C01CC24B7FCC094DC2CD4
:10CEA0008091300390913103A0913203B09133030C
:10CEB000BC01CD01A60195010E94768F820E931EC2
:10CEC0001092A2031092A3031092A4031092A50340
:10CED0002D813E8126193709B9019B01442737FD71
:10CEE0004095542F80912C0390912D03A0912E03F7
:10CEF000B0912F03820F931FA41FB51F80932C03A3
:10CF000090932D03A0932E03B0932F0381509D4740
:10CF1000A040B04064F080E09DE7A0E0B0E08093E6
:10CF20002C0390932D03A0932E03B0932F03809195
:10CF30002C0390912D03A0912E03B0912F038050CC
:10CF40009348AF4FBF4F64F480E093E8AFEFBFEF7B
:10CF500080932C0390932D03A0932E03B0932F0363
:10CF600080912C0390912D03A0912E03B0912F035B
:10CF7000BC01CD01A60195010E94768FE20EF31E41
:10CF80001092A6031092A7031092A8031092A9036F
:10CF9000C7C080915608909157089C01442737FDDF
:10CFA0004095542F8091A2039091A303A091A403D4
:10CFB000B091A503820F931FA41FB51F8093A203F6
:10CFC0009093A303A093A403B093A50381509D471E
:10CFD000A040B04064F080E09DE7A0E0B0E0809326
:10CFE000A2039093A303A093A403B093A5038091FD
:10CFF000A2039091A303A091A403B091A503805034
:10D000009348AF4FBF4F64F480E093E8AFEFBFEFBA
:10D010008093A2039093A303A093A403B093A503CA
:10D0200080919D0190919E015C01CC24B7FCC0943D
:10D03000DC2C8091A2039091A303A091A403B09152
:10D04000A503BC01CD01A60195010E94768F820E39
:10D05000931E1092300310923103109232031092FB
:10D06000330380913508909136089C01442737FDA1
:10D070004095542F8091A6039091A703A091A803F7
:10D08000B091A903820F931FA41FB51F8093A6031D
:10D090009093A703A093A803B093A90381509D4741
:10D0A000A040B04064F080E09DE7A0E0B0E0809355
:10D0B000A6039093A703A093A803B093A90380911C
:10D0C000A6039091A703A091A803B091A903805053
:10D0D0009348AF4FBF4F64F480E093E8AFEFBFEFEA
:10D0E0008093A6039093A703A093A803B093A903EA
:10D0F0008091A6039091A703A091A803B091A903E2
:10D10000BC01CD01A60195010E94768FE20EF31EAF
:10D1100010922C0310922D0310922E0310922F03C5
:10D1200080918901682F772788279927980117FF11
:10D1300004C022273327201B310B37FF02C02F5F8B
:10D140003F4F35952795A981BA812A0F3B1F442768
:10D1500037FD4095542F0E94028F97FF04C0615CF9
:10D160007F4F8F4F9F4FE6E0959587957795679511
:10D17000EA95D1F77C8F6B8F681579050CF44B011C
:10D180002B8D3C8D309521953F4F821693060CF4E4
:10D190004901EB8DFC8DEE15FF050CF47B01E216C9
:10D1A000F3060CF4790180914D08282E3324509019
:10D1B000F70665E6A62E67E0B62E5CE1C52E57E0C1
:10D1C000D52E4BE0442E38E6632E38E0732ED60180
:10D1D0002C9112160CF029C1203429F4E981FA812E
:10D1E000FE8FED8F1FC049815A81CA01AA2797FD82
:10D1F000A095BA2F332727FD3095432F532FBC011D
:10D20000CD010E94028F97FF04C0615C7F4F8F4F5A
:10D210009F4F26E095958795779567952A95D1F745
:10D220007E8F6D8FF6012181203439F42D8D3E8D56
:10D23000280D391D3E8F2D8F2AC0203C39F44D8D8D
:10D240005E8D481959095E8F4D8F21C0C401AA27F0
:10D2500097FDA095BA2F332727FD3095432F532FE5
:10D26000BC01CD010E94028F97FF04C0615C7F4F1B
:10D270008F4F9F4FB6E09595879577956795BA95AF
:10D28000D1F7AD8DBE8DA60FB71FBE8FAD8FF60146
:10D290002281203439F42D8D3E8D2E0D3F1D3E8F81
:10D2A0002D8F2AC0203C39F44D8D5E8D4E195F09BB
:10D2B0005E8F4D8F21C0C701AA2797FDA095BA2F79
:10D2C000332727FD3095432F532FBC01CD010E94FA
:10D2D000028F97FF04C0615C7F4F8F4F9F4FA6E086
:10D2E0009595879577956795AA95D1F7AD8DBE8D64
:10D2F000A60FB71FBE8FAD8FF6012381203439F4FE
:10D300002D8D3E8D200F311F3E8F2D8F2AC0203C4A
:10D3100039F44D8D5E8D401B510B5E8F4D8F21C0BA
:10D32000C801AA2797FDA095BA2F332727FD30956E
:10D33000432F532FBC01CD010E94028F97FF04C0E1
:10D34000615C7F4F8F4F9F4FF6E09595879577955E
:10D350006795FA95D1F7AD8DBE8DA60FB71FBE8F1D
:10D36000AD8FF301808191812D8D3E8D82179307C2
:10D3700064F4B901680F791F77FF02C06F5F7F4FB8
:10D38000759567957E8F6D8F1DC0552049F44D8D25
:10D390005E8D440F551F481B590B5E8F4D8F12C079
:10D3A00051E0551578F4252D33276D8D7E8D861B24
:10D3B000970BB9010E94418FAD8DBE8DA60FB71F8F
:10D3C000BE8FAD8FC101880F991F880F991FED8DFA
:10D3D000FE8D8E179F0764F4FE898F2F9927880F83
:10D3E000991F880F991F2D8D3E8D2817390714F02E
:10D3F0009E8F8D8F8D8D9E8D97FD0396959587952C
:10D4000095958795F5018183880F991F880F991F3E
:10D410002D8D3E8D281B390BC901880F8283ED8D20
:10D42000FE8DD301ED93FC9303C0F50111821282AE
:10D430004A9422E030E0620E731E44E050E0C40ED5
:10D44000D51E68E070E0A60EB71E47FEC0CEE2E132
:10D45000C25E0C94AD8F84B1806A84B93D9A82E536
:10D460008CBD1DBC459A81E08093A6088AEA809312
:10D47000B70883E88093B8088AE08093B9081092CF
:10D48000BB081092BA081092BD081092BC08109206
:10D490001F091092DB0808953091A608332309F084
:10D4A00085C00DB407FE82C084E080930B02459ACC
:10D4B0002EB58091FC0399278130910589F0823047
:10D4C00091051CF4892B21F03EC00297B9F03BC0B6
:10D4D0003093DA082093FD032138A9F581E008C0D4
:10D4E000253549F48091FD03820F8093FD0382E08E
:10D4F0008093FC0328C03093FC0325C08091DA0898
:10D50000E82FFF27E450F74F20838F5F8093DA08DE
:10D510009091FD038032A0F0291769F480E2ACEF0E
:10D52000B8E0ECEDF8E00D9001928A95E1F781E02A
:10D530008093DB0802C03093DB081092FC0303C029
:10D54000920F9093FD032091B608223208F028C074
:10D5500045980000000000000000000000000000EE
:10D5600000000000000000000000000000000000BB
:10D5700000000000000000000000000000000000AB
:10D580000000E091AF08F091B008E20FF11D80813A
:10D590008EBD8091D8089081890F8093D80803C0F0
:10D5A00081E08093A6082F5F2093B6080895EF923C
:10D5B000FF920F931F938091AF069927880F991FB1
:10D5C000880F991F7C010027F7FC0095102F809190
:10D5D000640390916503A0916603B0916703BC0159
:10D5E000CD01A80197010E94768F3093BB0820934C
:10D5F000BA0880915C0390915D03A0915E03B091A5
:10D600005F03BC01CD01A80197010E94768F309382
:10D61000BD082093BC082091930830919408409154
:10D62000950850919608DA01C90163E0880F991FA7
:10D63000AA1FBB1F6A95D1F7820F931FA41FB51FA6
:10D64000820F931FA41FB51F209145013091460101
:10D650004091470150914801BC01CD010E94768F55
:10D660003093C3082093C20880917503909176038C
:10D6700020912A0230912B02821B930B9093C908B0
:10D680008093C808E0916B03F0916C0380915D0872
:10D6900090915E08BF010E94418F9B01220F331FB2
:10D6A000220F331F260F371F260F371F37FF02C0E9
:10D6B0002D5F3F4F35952795359527953093BF08BA
:10D6C0002093BE0880918F0890919008BF010E941E
:10D6D000418F9B01220F331F220F331F260F371F4D
:10D6E000260F371F37FF02C02D5F3F4F3595279517
:10D6F000359527953093C1082093C00810926C038C
:10D7000010926B0310925E0810925D0810929008C0
:10D7100010928F088091B90899278D30910509F4EE
:10D720008CC08E3091055CF48B30910509F4B4C047
:10D730008C3091050CF035C10A9761F0E7C18F304C
:10D74000910509F4B3C18F3091050CF480C1409765
:10D75000A9F1DCC18091EB028093CC088091EA02B0
:10D760008093CD088091E9028093CE088091E802F1
:10D770008093CF088091E7028093D0088091E602E1
:10D780008093D1088091E5028093D2088091E402D1
:10D790008093D3088091D2028093D4088091D202E2
:10D7A000837F8093D2020E94DE2F8093D5088091E0
:10D7B000F8068093D6088091D102A6C180912C09E9
:10D7C00090912D099093CD088093CC0880913009D9
:10D7D000909131099093CF088093CE0880912001D9
:10D7E000909121018093D008809100018093D1080D
:10D7F000809144018093D2089091FE039093D308C6
:10D80000E92FFF27A3E0EE0FFF1FAA95E1F7EB59E1
:10D81000F84F86818093D40883818093D5088781CF
:10D820008093D60885818093D708892F8F5F6CE01D
:10D830000E94218F9093FE0369C1809145088093D7
:10D84000CC088091E4068093CD088091E506809312
:10D85000CE088091E6068093CF088091E7068093FA
:10D86000D0088091EB068093D1088091EC068093DC
:10D87000D2088091ED068093D3088091F0068093C2
:10D88000D4088091EE068093D5088091EF068093AE
:10D89000D6088091F10638C1F89480919606E82F59
:10D8A000FF27EE0FFF1FEA53F84F0190F081E02DA4
:10D8B000E038F1051CF0EFE7F0E006C02FEFE138AB
:10D8C000F20714F4E1E8FFEFE093CC0880919706AB
:10D8D000E82FFF27EE0FFF1FEA53F84F0190F0816A
:10D8E000E02DE038F1051CF0EFE7F0E006C06FEF47
:10D8F000E138F60714F4E1E8FFEFE093CD088091FA
:10D900009506E82FFF27EE0FFF1FEA53F84F01900F
:10D91000F081E02DE038F1051CF0EFE7F0E006C003
:10D920008FEFE138F80714F4E1E8FFEFE093CE0859
:10D9300080919406E82FFF27EE0FFF1FEA53F84F60
:10D940000190F081E02DE038F1051CF0EFE7F0E008
:10D9500006C02FEFE138F20714F4E1E8FFEF789406
:10D96000E093CF0880910F038093D008809110033B
:10D970008093D108809111038093D2088091120383
:10D980008093D308809113038093D408809114036B
:10D990008093D508809115038093D6088091160353
:10D9A000B3C080918104863018F01092810485E024
:10D9B0008093CC088091F2068093CD088091080373
:10D9C00090910903A0910A03B0910B03BC01CD0112
:10D9D00025E030E040E050E00E94768F3093CF08A1
:10D9E0002093CE088091040390910503A091060333
:10D9F000B0910703BC01CD0125E030E040E050E0EC
:10DA00000E94768F3093D1082093D0088091E80649
:10DA10008093D2088091E9068093D3088091EA062A
:10DA20008093D40880910E038093D5088091C60717
:10DA30009091C7078093D6088091000690910106C7
:10DA400097FD039695958795959587955DC010925E
:10DA5000CC0888E58093CD0884E08093CE088FE1E0
:10DA60008093CF08809102018093D0088091660452
:10DA70008093D108809167048093D2081092660445
:10DA8000807180936704809168048093D3088091AB
:10DA900082088093D408809164088093D50880918F
:10DAA000F4068093D608809101072EC08091C806A5
:10DAB0008093CC088091FF068093CD0880918F01E0
:10DAC0008093CE088091C1068093CF088091C206D2
:10DAD0008093D0088091C3068093D10880918E01F5
:10DAE0008093D2088091C5068093D3088091C606A2
:10DAF0008093D4088091C7068093D508809134091B
:10DB00008093D60880912A068093D7088091DB08FD
:10DB1000882309F455C18AEF8093CC0181E080937A
:10DB2000B1014091DD085091DE08CA0181509E4F3D
:10DB30008F5F9340B0F42091DF083091E008C90175
:10DB400081509E4F8F5F934060F48091A00685FFC7
:10DB500008C05093EB034093EA033093E90320930A
:10DB6000E8038091E3089091E40821E08936920768
:10DB700024F49093B3018093B2012091ED08309189
:10DB8000EE0880910C0290910D028217930740F4E9
:10DB90008091DE01882321F430930D0220930C0242
:10DBA0008091DC0899278936910509F4A5C08A3649
:10DBB000910544F48736910571F08836910509F492
:10DBC00062C006C18A36910509F4F3C08B3691050F
:10DBD00009F4E2C0FDC08091EF0880931C09809198
:10DBE000F00880931E098091F10880931D098091AF
:10DBF000F2088093B0018091F3088093200980910E
:10DC0000F4088093CD018091F5088093FB03809107
:10DC1000F6088093E7038091E3028823F9F02091CE
:10DC2000F7083091F80837FD19C030932703209387
:10DC300026039091CA06992389F08FE0989FC0012E
:10DC40001124281B390BC90188599E4F68E671E0E1
:10DC50000E94418F90932703809326032091F20323
:10DC60003091F3038091F9089091FA08280F391F39
:10DC700037FF02C02F5F3F4F359527953093F30351
:10DC80002093F203A5C08091EF088093B1088091A2
:10DC9000F0088093B2088091F1088093B3088091D6
:10DCA000F2088093B4088091F3088093B5088091BE
:10DCB000F0059091F408892B8093F0059091F1057F
:10DCC00093708091F5088C70982B9093F10580915A
:10DCD000F6088093F9038091F7088093C201809140
:10DCE000F80880931F098091F9088093F5038091CB
:10DCF000FA088093F4036CC08091EF088093A70822
:10DD00008091F0088093A8088091F1088093A90879
:10DD10008091F2088093AA088091F3089091F4080A
:10DD20009093AC088093AB088091F5089091F60829
:10DD30009093AE088093AD088091F708992787FDEE
:10DD400090959093F9078093F8078091F808809355
:10DD5000FD028091F9089091FA089C01442737FD53
:10DD60004095542FDA01C90163E0880F991FAA1F5B
:10DD7000BB1F6A95D1F7820F931FA41FB51F820F97
:10DD8000931FA41FB51F8093FE029093FF02A093E0
:10DD90000003B09301031CC08091EF088093F80347
:10DDA0008091F0088093F7038091F1088093F60347
:10DDB0000FC08091BA06863059F40E94297508C0B8
:10DDC0001092EB031092EA031092E9031092E80319
:10DDD0001F910F91FF90EF9008958091A6088823DE
:10DDE00009F43BC0459887EB98E09093B008809386
:10DDF000AF089091FA03E92FFF27ED53FE4F9F5F85
:10DE00009093FA0380818093B908993010F01092B2
:10DE1000FA031092A6080E94D76A81E08093B608A0
:10DE200000000000000000000000000000000000F2
:10DE300000000000000000000000000000000000E2
:10DE400000000000000000000000000000000000D2
:10DE50008091B7088093D8088EBD089587B18C60F3
:10DE600087B9429843981092000480E88093CF01CC
:10DE70001092FF038093CE01089580910504815094
:10DE8000809305048F3F09F019C189E08093050450
:10DE90008091D202992780739070892B21F4809110
:10DEA000670480FF1DC08091E106882351F08091B6
:10DEB0000804882319F484E08093000481E08093AF
:10DEC00008048091E2068823B9F080910904882330
:10DED00019F484E08093FF0381E0809309040CC06F
:10DEE00010920804109209048091DD0680930604C4
:10DEF0008091DF068093070480910804882309F04D
:10DF000045C08091FE06282F332724FF07C080914B
:10DF10000D03882319F425FD52C053C09091DE06ED
:10DF2000983F48F080915F088D3D28F0809106046D
:10DF300088236CF00AC0983F78F080915F088530A4
:10DF400059F48091060487FF02C0429801C0429AAA
:10DF500081E08093CF0136C080910004815080938E
:10DF600000048F3F79F580915F08869580930004C7
:10DF70008091CF01813011F480E801C086958093B3
:10DF8000CF018091CF019091060417C080910004C9
:10DF90008150809300048F3FA9F489E080930004AE
:10DFA0008091CF01813011F480E801C08695809383
:10DFB000CF018091CF019091E106892311F0429A1F
:10DFC00001C0429880910904882309F043C09091D0
:10DFD000FE0697FF07C080910D03882319F496FD74
:10DFE00052C053C09091E006983F48F08091890854
:10DFF0008D3D28F08091070488236CF00AC0983F7B
:10E0000078F080918908853059F48091070487FF62
:10E0100002C0439801C0439A81E08093CE0136C08C
:10E020008091FF0381508093FF038F3F79F58091AA
:10E03000890886958093FF038091CE01813011F489
:10E0400080E801C086958093CE018091CE019091A9
:10E05000070417C08091FF0381508093FF038F3F17
:10E06000A9F489E08093FF038091CE01813011F4FF
:10E0700080E801C086958093CE018091CE01909179
:10E08000E206892311F0439A01C04398429B04C0E1
:10E090008091D102886003C08091D102877F8093F4
:10E0A000D102439B06C08091D10280618093D1024E
:10E0B00008958091D1028F7E8093D10208954FB749
:10E0C00024E130E0F8948091C9008F778093C900F3
:10E0D0008091C9008F7B8093C9008091C9008F7D9A
:10E0E0008093C9005A9A52985B9A539A832F992722
:10E0F0008093CD002093CC008091C80082608093F3
:10E10000C80080E18093C9008091CA008F77809316
:10E11000CA008091CA008F7B8093CA008091CA0098
:10E120008F7D8093CA008091CA008F7E8093CA0041
:10E130008091CA00877F8093CA008091C9008B7F3D
:10E140008093C9008091CA0084608093CA00809146
:10E15000CA0082608093CA008091C80087FF03C014
:10E160008091CE00F9CF8091C90080688093C9006A
:10E170004FBF0895A0E0B0E0E0ECF0E70C949B8F77
:10E18000482FC0E0D0E08091D001813061F410923E
:10E19000D00184E480930C0410920E0410920D04BC
:10E1A00010920F041AC280910C04882319F421E004
:10E1B00030E001C09E0190910D04992371F4232B4E
:10E1C00011F081E010C084E480930C0490930E045D
:10E1D00090930D0490930F04E9C1913069F4232BBF
:10E1E00009F0DAC182E080930D0480910E048F5F04
:10E1F00080930E0483E0D8C19230D1F4232B09F030
:10E20000CBC183E080930C0440930F0490910E04E3
:10E21000923039F41092100447FF03C081E08093DC
:10E22000100483E080930D049F5F90930E04BEC1A1
:10E23000933009F0B1C1232B09F0AEC190930C04C7
:10E2400082E080930D0480910E048F5F80930E0412
:10E2500020910F04822F9927782F6627842F9927E2
:10E26000682B792B8091BA06813051F47370CB0101
:10E270008050924063E070E00E94418F8B0119C092
:10E28000823069F47770CB018050944066E070E092
:10E290000E94418F8B012695269526950CC08B01F7
:10E2A000137008561140C80117FD01968C01159591
:10E2B000079526952695C22FDD27CF70D070219621
:10E2C000CD30D10508F062C1C230D10519F4C4E0E7
:10E2D000D0E005C0C430D10511F4C2E0D0E06E0139
:10E2E000CC0EDD1EF601EA53F84F80819181980132
:10E2F000281B390BC90137FF03C0909581959F4FAB
:10E30000069704F5E091FB06EE2351F0FF27EE0F90
:10E31000FF1FEA53F84F808191818436910594F470
:10E3200080910E03883C30F480910E03865F8093C9
:10E330000E0308C088EC80930E0380916F008F7DE0
:10E3400080936F00F601EA53F84F808191819C0120
:10E35000220F331F280F391F200F311F37FF02C034
:10E360002D5F3F4F7901F594E794F594E794C80148
:10E3700001968E159F0524F40894E108F10808C061
:10E38000C8010197E816F9061CF40894E11CF11C79
:10E39000C630D10509F0B4C0053611050CF48BC0A8
:10E3A00090910B04E92FFF27EF5DF64FE081ED37E9
:10E3B00029F480910A04809580930A04993009F029
:10E3C00076C080910A04882319F4E33821F06FC0E5
:10E3D000ED3709F06CC0809122098D3739F48091B6
:10E3E00023098338B1F483E89FEF0FC0833889F4A1
:10E3F00080912309833829F41092D1071092D00715
:10E4000008C08D3731F48DE790E09093D107809369
:10E41000D007809124098D3739F4809127098338FA
:10E42000B1F48DE790E00FC0833889F4809127091B
:10E43000833829F41092D3071092D20708C08D3781
:10E4400031F483E89FEF9093D3078093D2078091B4
:10E4500028098D3739F4809129098338B1F483E88C
:10E460009FEF0FC0833889F480912909833829F4FC
:10E470001092D9071092D80708C08D3731F48DE774
:10E4800090E09093D9078093D80780912609992727
:10E4900087FD90959093DB078093DA07809125099B
:10E4A000992787FD90959093DF078093DE07109260
:10E4B0000B0410920A040A3011055CF480910B04DD
:10E4C0008F5F80930B04E82FFF27EF5DF64F83E803
:10E4D000808380910B048A3011F410920B043FEF7B
:10E4E0000C3913076CF480910B04E82FFF27EF5DC4
:10E4F000F64F8DE7808380910A04809580930A040B
:10E5000080910E03843BD0F0F601EA53F84F8081EE
:10E510009181F701E81BF90BCF0163E070E00E94E5
:10E52000418FCB01880F991F860F971F2AEF37E085
:10E53000C20ED31EF6019183808307C02AEF37E015
:10E54000C20ED31EF60111821082C530D10538F4F7
:10E55000CC0FDD1FCA53D84FF982E88227C0C730DD
:10E56000D10529F41093D5070093D4071FC0C530F7
:10E57000D10529F41093D7070093D60717C0289721
:10E58000A9F41093DD070093DC0710C0629770F0C8
:10E5900081E08093D0010AC081E08093D001109285
:10E5A0000E041092100484E480930C0480910E04F5
:10E5B000803198F080911004882331F48091D0014B
:10E5C000882311F48093430110920E0410921004DA
:10E5D00010920D0484E480930C04E8E0CDB7DEB71C
:10E5E0000C94B78FCF93FC0197FF05C0CFEFF09548
:10E5F000E195FF4F01C0C1E028E631E0CF01B9014C
:10E600000E94418FFC018B35910554F08B55904051
:10E610008A35910538F484EB90E08E1B9F0BFC014A
:10E6200041E00DC0CF01855B90408A35910518F41B
:10E63000E45BF04003C02E1B3F0BF9014FEFEE0FE0
:10E64000FF1FEA5AF64F259134918C2F992787FDA9
:10E650009095289FB001299F700D389F700D11244F
:10E66000842F992787FD9095689FA001699F500D81
:10E67000789F500D1124CA01CF9108952AE530E00A
:10E68000281B390BC9010E94F2720895089508955C
:10E69000089508950895CF93C82F80E00E941185B2
:10E6A0008091E0079091E10781589F4F9F938F934E
:10E6B0008CE09AE09F938F9384E095E89F938F93EB
:10E6C000E0914C04F0914D0409958DB79EB70696E4
:10E6D0008DBFCF3231F48091E0079091E1074996E8
:10E6E00007C0CF3449F48091E0079091E107499742
:10E6F0009093E1078093E0078091E0079091E10714
:10E7000082589F4F1CF481E89FEF09C08091E00779
:10E710009091E1078038910534F080E890E0909383
:10E72000E1078093E007CF910895CF93C82F80E150
:10E730000E9411858091E2079091E30781589F4FD5
:10E740009F938F938CE19AE09F938F9384E095E859
:10E750009F938F93E0914C04F0914D0409958DB7F0
:10E760009EB706968DBFCF3231F48091E20790912B
:10E77000E307029607C0CF3449F48091E2079091F5
:10E78000E30702979093E3078093E2078091E20703
:10E790009091E30782589F4F1CF481E89FEF09C0D6
:10E7A0008091E2079091E3078038910534F080E88A
:10E7B00090E09093E3078093E207CF91089580E083
:10E7C00090E0089510922D0910922C0910923109B1
:10E7D0001092300910922F0910922E0910923409CC
:10E7E0008AE090E00E94FF18909312048093110435
:10E7F0000895CF93DF9380911104909112040E94A9
:10E800000819882309F4AFC0809111049091120473
:10E810000A969093120480931104E0E0F0E09F01C7
:10E8200090E05FEFA5E6B7E04BE0ED018B8187FF5D
:10E830000BC09F5F8D81E80FF11D8981280F311D6D
:10E840008E81851708F4582F4150189647FFEDCF59
:10E8500050933409232B41F520911704309118046B
:10E860004091190450911A04BB27A52F942F832F90
:10E870009093160480931504AA27BB27281B390BF5
:10E880004A0B5B0BCF01AA27BB27280F391F4A1F52
:10E890005B1F20931704309318044093190450937E
:10E8A0001A04E5E0F0E013C020911504309116043D
:10E8B0002E173F0718F4E21BF30B02C0E0E0F0E074
:10E8C000892F9927880F991FE80FF91F3596F09324
:10E8D0002D09E0932C09EF3FF10578F48091200198
:10E8E000909121018E9F90018F9F300D9E9F300D42
:10E8F0001124C90164E670E013C0CF019695879595
:10E90000969587952091200130912101289FA001A3
:10E91000299F500D389F500D1124CA0169E170E004
:10E920000E942D8F70932F0960932E09209113045C
:10E93000309114042E0F3F1F3093140420931304BE
:10E940005EE02131350778F08091300990913109EE
:10E950000196909331098093300920513E403093C5
:10E96000140420931304DF91CF9108953091200473
:10E97000E32FFF2783E0EE0FFF1F8A95E1F7EB59A6
:10E98000F84F2781422F552747FD5095809121044C
:10E990009927841795072CF420932104309323049E
:10E9A0000AC0222341F08091220499274817590771
:10E9B00014F420932204832F8F5F809320048D30E2
:10E9C000D0F010922004809122048F3F19F08093A0
:10E9D0001C0402C010921C048091210480931D0429
:10E9E0008091230480931B048FEF80932204109264
:10E9F000210410922304089595E1899F802D11240C
:10EA00000E9460898AE29CE09F938F9382E399E859
:10EA10009F938F93E0914C04F0914D0409950F90D2
:10EA20000F900F900F9008958091D20285FF03C040
:10EA300080E190E0089580910D03882339F0809162
:10EA4000F903882319F085E090E0089580E090E0D4
:10EA5000089540E050E030E08091FA0899278A3824
:10EA6000910591F08B38910524F48938910541F096
:10EA700016C08D38910581F08E38910549F00FC090
:10EA80004DE759E031E10BC04AE35AE03DE107C0F0
:10EA900045E359E036E203C04BE559E032E290919C
:10EAA000EF0820E08091F008281770F4931760F4C5
:10EAB000DA01A90FB11DE22FFF27E452F74F858934
:10EAC0008C939F5F2F5FEECF089520E335E7809111
:10EAD00044018B3211F08D32F9F48091A506282F74
:10EAE00033278091020390910303829FA001839FAB
:10EAF000500D929F500D1124CA0163E070E00E94F6
:10EB0000418FCB019B01205D3A48C196C19708F027
:10EB10003FC02EEF34E73CC0803229F58091D2020D
:10EB200081FF36C020911E0430911F04205D3A48B9
:10EB300055E72133350748F085E72439380718F4BD
:10EB400020E335E702C02456304045E72033340740
:10EB5000F8F454E72D3C350718F020E335E718C0EA
:10EB60002C593F4F15C08E3549F49091FD028AE033
:10EB7000989F90011124205D3A480AC0863741F4DD
:10EB80009091FD028AE0989FC0011124281B390B47
:10EB9000C9010895EF92FF920F931F9399278A3826
:10EBA000910509F45DC08B38910524F489389105ED
:10EBB00051F0D2C18D38910509F416C18E389105F6
:10EBC00009F483C0C9C18091080390910903A09101
:10EBD0000A03B0910B03BC01CD0124E630E040E014
:10EBE00050E00E94768FDA01C9018C509E4F9093BD
:10EBF0008109809380090E946575909387098093AD
:10EC00008609909389098093880990938B09809352
:10EC10008A0920918009309181098091840990911D
:10EC200085092817390724F430938509209384092E
:10EC300080918209909183098217930724F430937D
:10EC40008309209382090E94147580937F098DE7C0
:10EC500099E0909332048093310481E190E07EC189
:10EC60008091080390910903A0910A03B0910B03CE
:10EC7000BC01CD0124E630E040E050E00E94768FF8
:10EC8000DA01C9018C509E4F90934D0A80934C0A33
:10EC90000E94657590934F0A80934E0A88E790E032
:10ECA0009093510A8093500A1092530A1092520A7C
:10ECB0000E94147580933C0A8AE39AE09093320490
:10ECC000809331048DE190E049C10E94B674809137
:10ECD000080390910903A0910A03B0910B03BC01B2
:10ECE000CD0124E630E040E050E00E94768FDA016A
:10ECF000C9018C509E4F90934D0980934C0980918F
:10ED000020019091210190934709809346098091B9
:10ED100020019091210190934909809348098091A5
:10ED20003D0890913E0897FD0196959587958093B3
:10ED3000380980933F092091AD083091AE0837FF24
:10ED400002C02F5F3F4F3595279520933D09809155
:10ED5000AB089091AC0864E170E00E942D8F609345
:10ED60003E0920934409609345090E94657590937C
:10ED700055098093540988E790E090935709809350
:10ED8000560980912001909121019093510980931F
:10ED9000500980911C048C5E80934A0980911D0467
:10EDA0008C5E80934B0980913009909131096AE023
:10EDB00070E00E94418F70935309609352090E9442
:10EDC00014758093370980912C0990912D099093A7
:10EDD0004F0980934E0985E399E090933204809324
:10EDE000310486E290E0BAC00E94B6748091AB080C
:10EDF0009091AC0864E670E00E942D8F70936E09CC
:10EE000060936D0980913D0890913E0897FD0196B1
:10EE10009595879580935E098091AD089091AE0895
:10EE200097FD0196959587958093630980910001E0
:10EE3000482F55279A012B5F3F4F809120019091D9
:10EE400021012817390784F4809120019091210134
:10EE5000841B950B9C01220F331F280F391F822F13
:10EE6000825180936A0902C010926A09E0900803F7
:10EE7000F090090300910A0310910B03C801B70138
:10EE800024E630E040E050E00E94768F30936C0939
:10EE900020936B0937FF04C010926C0910926B0924
:10EEA000C801B70124E630E040E050E00E94768FD0
:10EEB000DA01C9018C509E4F9093700980936F09BD
:10EEC00080912001909121019093650980936409BC
:10EED00080912001909121019093670980936609A8
:10EEE0000E946575909372098093710988E78093F9
:10EEF000730980912001909121019093770980936B
:10EF0000760980911C048C5E8093680980911D04B1
:10EF10008C5E8093690980913009909131096AE093
:10EF200070E00E94418F70937909609378090E9484
:10EF3000147580935D0980912C0990912D0990930F
:10EF40007509809374098BE599E09093320480935E
:10EF5000310482E290E002C080E090E01F910F91C6
:10EF6000FF90EF900895EF92FF920F931F93CF932E
:10EF7000DF9380911E0490911F049C0103E0220FF7
:10EF8000331F0A95E1F7281B390B80911D029091E0
:10EF90001E02280F391F37FF02C0295F3F4F13E0C1
:10EFA000359527951A95E1F730931F0420931E0499
:10EFB00090912504992309F011C380912404282FEE
:10EFC0003327442755278F5F80932404F90121318B
:10EFD000310508F000C3E058FF4F0C94C88F8091B2
:10EFE000D20285FF2AC080E00E94608980912001C2
:10EFF000909121016AE070E00E94418F9F938F936E
:10F0000080912001909121016AE070E00E94418F7F
:10F010007F936F9380E49CE09F938F9383E599E8BF
:10F020009F938F93E0914C04F0914D0409952DB777
:10F030003EB7285F3F4F2DBF28C080E00E94608907
:10F0400080912001909121016AE070E00E94418F3F
:10F050009F938F9380912001909121016AE070E04D
:10F060000E94418F7F936F938DE49CE09F938F93D9
:10F0700082E399E89F938F93E0914C04F0914D04C3
:10F0800009958DB79EB708968DBF8091820880FF45
:10F0900039C0809125038823E9F08AE00E946089C5
:10F0A0008091440199279F938F93809108039091B9
:10F0B0000903A0910A03B0910B03BC01CD0124E622
:10F0C00030E040E050E00E94768F3F932F938AE536
:10F0D0009CE084C68AE00E94608980910803909138
:10F0E0000903A0910A03B0910B03BC01CD0124E6F2
:10F0F00030E040E050E00E94768F3F932F9386E609
:10F100009CE098C78AE00E94608981E79CE017C66E
:10F110008091D20285FF2AC085E10E94608980919A
:10F12000D8019091D9016CE370E00E942D8F9F93DC
:10F130008F938091D8019091D9016CE370E00E9487
:10F140002D8F7F936F938BE79CE09F938F9383E545
:10F1500099E89F938F93E0914C04F0914D040995A9
:10F160002DB73EB7285F3F4F2DBF28C085E10E94D5
:10F1700060898091D8019091D9016CE370E00E9480
:10F180002D8F9F938F938091D8019091D9016CE33B
:10F1900070E00E942D8F7F936F9388E89CE09F938F
:10F1A0008F9382E399E89F938F93E0914C04F091C1
:10F1B0004D0409958DB79EB708968DBF8FE10E94CB
:10F1C000608980E690E09F938F9380913D089091B5
:10F1D0003E089F938F9385E99CE09F938F93C2E3B2
:10F1E000D9E8DF93CF93E0914C04F0914D04099559
:10F1F0008091D1022DB73EB7285F3F4F2DBF80FFD2
:10F2000006C089E20E94608980EA9CE069C389E2C5
:10F210000E94608982EA9CE0A9C68091D20285FFA3
:10F220001BC08AE20E946089809130099091310967
:10F230009F938F9384EA9CE09F938F9383E599E853
:10F240009F938F93E0914C04F0914D0409958DB7F5
:10F250009EB706968DBF1BC08AE20E94608980918E
:10F260003009909131099F938F938CEA9CE09F9392
:10F270008F9382E399E89F938F93E0914C04F091F0
:10F280004D0409952DB73EB72A5F3F4F2DBF86E34A
:10F290000E94608980912C0990912D096AE070E0AC
:10F2A0000E942D8F9F938F9380912C0990912D090F
:10F2B0006AE070E00E942D8F7F936F9384EB9CE057
:10F2C0009F938F9382E399E89F938F93E0914C04EF
:10F2D000F0914D0409958DB79EB70896B9C689E09F
:10F2E0000E94608980EC9CE09F938F9302E319E871
:10F2F0001F930F93E0914C04F0914D0409958EE11A
:10F300000E9460890F900F900F900F9082EC9CE00C
:10F310009F938F931F930F93E0914C04F0914D04B2
:10F32000099583E30E9460890F900F900F900F90D2
:10F3300084EC9CE09F938F931F930F93E0914C0478
:10F34000F0914D0409958FE30E9460890F900F9012
:10F350000F900F9086EC9CE09F938F931F930F93D9
:10F36000E0914C04F0914D0409958EE70E9460896C
:10F370000F900F900F900F908CED9CE09F938F93C8
:10F380001F930F938AC78091CC01882309F462C030
:10F390008DE50E94608982EF9CE09F938F93C2E38A
:10F3A000D9E8DF93CF93E0914C04F0914D04099597
:10F3B00084E50E9460890F900F900F900F908091CC
:10F3C000A80899279F938F9384EF9CE09F938F9336
:10F3D000DF93CF93E0914C04F0914D0409958EE5B5
:10F3E0000E9460892DB73EB72A5F3F4F2DBF8091A5
:10F3F000AB089091AC086AE070E00E942D8F7F937B
:10F400006F938DEF9CE09F938F93DF93CF93E09169
:10F410004C04F0914D0409958DB79EB706968DBFAB
:10F420008091A908833081F48091A70881FF06C0EC
:10F430008BE50E94608987E09DE098C58BE50E947E
:10F4400060898AE09DE092C58BE50E9460898DE02D
:10F450009DE01DC784E0CDC38091CC01882309F4D1
:10F460007AC080912704C2E3EC2EC9E8FC2E8823E1
:10F4700009F44BC089E60E9460898091F8039927BE
:10F480009F938F9380E19DE09F938F93FF92EF92E4
:10F49000E0914C04F0914D04099585E70E94608944
:10F4A0002DB73EB72A5F3F4F2DBF8091C2019927EC
:10F4B0009F938F9300E610E01F930F938091AD0808
:10F4C0009091AE089F938F938BE19DE09F938F93D4
:10F4D000FF92EF92E0914C04F0914D04099582E780
:10F4E0000E9460898DB79EB70A968DBF8091F60302
:10F4F00099279F938F931F930F938091F7039927D9
:10F500009F938F9387E29DE063C689E60E9460899E
:10F510008091C20199279F938F9380E690E09F93FB
:10F520008F938091AD089091AE089F938F938091B7
:10F53000AA0899279F938F9387E39DE09F938F93CA
:10F54000FF92EF92E0914C04F0914D0409958DB734
:10F550009EB70C967DC585E04CC39091F903992325
:10F56000D1F080912E04882381F09E3170F487E0E1
:10F570000E94FC7483E90E9460898091F9039927B5
:10F580009F938F9380E59DE09EC383E90E946089ED
:10F590008BE59DE0ADC383E90E94608981E69DE033
:10F5A000CEC30E941475809390098091700A8630B2
:10F5B00059F480912704882319F01092270499C6E2
:10F5C00081E08093270495C6883009F092C60E9496
:10F5D000658981E0D5C39093240493C6913009F0E6
:10F5E000DAC380912404282F3327442755278F5FBF
:10F5F00080932404F9012131310508F07DC6EF56CE
:10F60000FF4F0C94C88F8091D20285FF43C080E0E9
:10F610000E94608980913009909131099F938F9366
:10F6200080912001909121016AE070E00E94418F59
:10F630009F938F9380912001909121016AE070E067
:10F640000E94418F7F936F938091D8019091D9014F
:10F650006CE370E00E942D8F9F938F938091D8016F
:10F660009091D9016CE370E00E942D8F7F936F938E
:10F6700087E79DE09F938F9383E599E89F938F930E
:10F68000E0914C04F0914D0409952DB73EB7225FEF
:10F690003F4FABC580E00E94608980913009909116
:10F6A00031099F938F9380912001909121016AE00D
:10F6B00070E00E94418F9F938F93809120019091E1
:10F6C00021016AE070E00E94418F7F936F938091E7
:10F6D000D8019091D9016CE370E00E942D8F9F9327
:10F6E0008F938091D8019091D9016CE370E00E94D2
:10F6F0002D8F7F936F9382E99DE0C6C285E10E94C2
:10F70000608980E690E09F938F938091B201909101
:10F71000B3019F938F938DEA9DE09F938F93C2E3F4
:10F72000D9E8DF93CF93E0914C04F0914D04099513
:10F73000809182082DB73EB7285F3F4F2DBF80FFD5
:10F7400051C080912503882339F18FE10E9460899F
:10F750008091080390910903A0910A03B0910B03D3
:10F76000BC01CD0124E630E040E050E00E94768FFD
:10F770003F932F9387EB9DE09F938F9382E499E8CB
:10F780009F938F93E0914C04F0914D0409958DB7B0
:10F790009EB706968DBF38C08FE10E946089809128
:10F7A000080390910903A0910A03B0910B03BC01D7
:10F7B000CD0124E630E040E050E00E94768F3F9398
:10F7C0002F9380EC9DE09F938F93DF93CF93E091F5
:10F7D0004C04F0914D0409952DB73EB72A5F3F4F79
:10F7E0002DBF12C08FE10E94608989EC9DE09F933C
:10F7F0008F93DF93CF93E0914C04F0914D040995E2
:10F800000F900F900F900F9089E20E946089809175
:10F81000440199279F938F9383ED9DE09F938F934E
:10F82000DF93CF930DC48091CC018823F9F08BE254
:10F830000E9460898091C20199279F938F93809144
:10F84000AB089091AC086AE070E00E942D8F7F9326
:10F850006F9380E690E09F938F938091AD08909195
:10F86000AE089F938F9386ED9DE05CC182E0C1C19D
:10F870008FE30E94608980912E0990912F099F93B8
:10F880008F9380912C0990912D096AE070E00E947D
:10F890002D8F9F938F9380912C0990912D096AE071
:10F8A00070E00E942D8F7F936F938DEE9DE09F936C
:10F8B0008F93C2E3D9E8DF93CF93E0914C04F091AA
:10F8C0004D0409958091D1022DB73EB7265F3F4F79
:10F8D0002DBF80FF0AC082E50E94608981E09EE022
:10F8E0009F938F9382E499E8D6C482E50E94608951
:10F8F00084E09EE03BC38091CC01B2E3EB2EB9E8FB
:10F90000FB2E882309F449C084E50E946089809118
:10F91000A80899279F938F938091AA0899279F936E
:10F920008F9387E09EE09F938F93E701FF92EF9282
:10F93000E0914C04F0914D0409958DB79EB708965F
:10F940008DBF8091A908833051F484E60E946089BC
:10F950008AE19EE09F938F93FF92EF920BC084E623
:10F960000E94608980E29EE09F938F9383E599E8EF
:10F970009F938F93E0914C04F0914D0409950F9063
:10F980000F900F900F908091A70881FFBAC484E672
:10F990000E94608986E29EE0E9C284E50E94608957
:10F9A0008CE29EE09F938F93FF92EF9276C48091BA
:10F9B0002604A2E3EA2EA9E8FA2E882309F450C00F
:10F9C00089E60E946089809182076AE00E94218F07
:10F9D000892F99279F938F93809182070E94218F6F
:10F9E00099279F938F9380917A070E94218F892F67
:10F9F00099279F938F9380917A070E94218F99274F
:10FA00009F938F93809172070E94218F892F99274E
:10FA10009F938F93809172070E94218F99279F93C4
:10FA20008F9380916A070E94218F892F99279F9336
:10FA30008F9380916A070E94218F99279F938F93BC
:10FA400082E49EE09F938F93FF92EF92E0914C04AB
:10FA5000F0914D0409952DB73EB72C5E3F4FC5C3BD
:10FA600089E60E94608980E690E09F938F93809161
:10FA70008407992787FD90959F938F9380917C07AA
:10FA8000992787FD90959F938F938091740799276D
:10FA900087FD90959F938F9380916C07992787FDA1
:10FAA00090959F938F938FE59EE09F938F93FF9206
:10FAB000EF92E0914C04F0914D0409958DB79EB7FB
:10FAC0000E96C6C28091260490919206882309F46E
:10FAD0008DC0943009F48CC09630A1F58EE70E9459
:10FAE0006089809192076AE00E94218F892F99276F
:10FAF0009F938F93809192070E94218F99279F93C4
:10FB00008F9380918A070E94218F892F99279F9335
:10FB10008F9380918A070E94218F99279F938F93BB
:10FB200082E79EE09F938F9382E399E89F938F9360
:10FB3000E0914C04F0914D0409952DB73EB7245F38
:10FB40003F4F53C3973008F4DCC38EE70E946089AF
:10FB50008091A2076AE00E94218F892F99279F93A5
:10FB60008F938091A2070E94218F99279F938F9353
:10FB700080919A070E94218F892F99279F938F93B5
:10FB800080919A070E94218F99279F938F9380914C
:10FB900092070E94218F892F99279F938F9380919D
:10FBA00092070E94218F99279F938F9380918A07B4
:10FBB0000E94218F892F99279F938F9380918A0785
:10FBC0000E94218F99279F938F9381E89EE09F93B6
:10FBD0008F9382E399E89F938F93E0914C04F09187
:10FBE0004D0409958DB79EB7449632C2943021F4E6
:10FBF00086E00E94FC7485C39630F1F48EE70E9483
:10FC0000608980E690E09F938F9380919407992775
:10FC100087FD90959F938F9380918C07992787FDFF
:10FC200090959F938F938EE99EE09F938F9382E3AD
:10FC300099E89F938F93D0C2973008F462C38EE700
:10FC40000E94608980E690E09F938F938091A40743
:10FC5000992787FD90959F938F9380919C07992773
:10FC600087FD90959F938F9380919407992787FDA7
:10FC700090959F938F9380918C07992787FD9095FE
:10FC80009F938F9381EB9EE09F938F9382E399E8FC
:10FC90009F938F930ECF9091F903992309F44AC053
:10FCA00080912E048823F9F09E31E8F487E00E94C9
:10FCB000FC7483E90E9460898091F90399279F93DE
:10FCC0008F9384EC9EE09F938F9382E499E89F93B7
:10FCD0008F93E0914C04F0914D0409952DB73EB7F8
:10FCE0002A5F3F4F82C283E90E9460898FEC9EE0C9
:10FCF0009F938F9302E319E81F930F93E0914C04B5
:10FD0000F0914D0409951F921F929091F90381E1A2
:10FD1000989FC0011124845D954F9F938F931F93EB
:10FD20000F93E0914C04F0914D0409958DB79EB767
:10FD30000A968EC183E90E94608985ED9EE09F93BB
:10FD40008F9382E399E8A7C20E941475809390096B
:10FD50008091700A863079F480912604882319F006
:10FD60001092260403C081E08093260485E00E945F
:10FD7000FC7486E0B3C2883031F40E94658982E069
:10FD800080932504B4C2813009F0B3C20E94658912
:10FD900010922504ACC2923009F0B1C280912404C3
:10FDA000282F3327442755278F5F80932404F90198
:10FDB0002131310508F0A0C2EE55FF4F0C94C88FD9
:10FDC00080E00E94608982E097E09F938F930E9479
:10FDD000DE2F99279F938F938BEE9EE09F938F93B7
:10FDE00082E499E89F938F93E0914C04F0914D0445
:10FDF00009952DB73EB7285F3F4FF7C185E10E94B7
:10FE0000608980E197E09F938F93809100016AE081
:10FE10000E94218F892F99279F938F9380910001B2
:10FE20000E94218F99279F938F938AEF9EE09F9343
:10FE30008F9382E399E89F938F93E0914C04F09124
:10FE40004D04099573CF8AE20E9460898BE09FE0A0
:10FE50009F938F93C2E3D9E8DF93CF93E0914C0453
:10FE6000F0914D040995809182080F900F900F90AA
:10FE70000F9080FF41C08091A00690919B0181FD71
:10FE80000BC0892F99279F938F9380E19FE09F93C9
:10FE90008F93DF93CF931DCFE0914C04F0914D04ED
:10FEA000933318F08AE19FE002C081E29FE09F93C4
:10FEB0008F93DF93CF9309950F900F900F900F9032
:10FEC00080916408E0914C04F0914D0490919B0165
:10FED00080FF0BC0892F99279F938F9388E29FE023
:10FEE0009F938F93DF93CF93AFC0892F99279F93D1
:10FEF0008F938EE29FE0CFC084E39FE037C08FE313
:10FF00000E9460898DE39FE09F938F93C2E3D9E8BD
:10FF1000DF93CF93E0914C04F0914D0409950F903D
:10FF20000F900F900F908091F506882319F481E4CB
:10FF30009FE01CC08091E302E0914C04F0914D04DD
:10FF4000882319F08AE49FE002C081E59FE09F9337
:10FF50008F93DF93CF9309950F900F900F900F9091
:10FF60008091000786FFCDC188E59FE09F938F9326
:10FF7000DF93CF9392C184E50E9460898FE59FE073
:10FF80009F938F93C2E3D9E8DF93CF93E0914C0422
:10FF9000F0914D040995809182080F900F900F9079
:10FFA0000F9085FD03C084E69FE011C08091E306B9
:10FFB000883F10F4E82F07C0EFEFF0E0E81BF109ED
:10FFC000E15FFC4FE081E23358F48DE69FE09F93C0
:10FFD0008F93DF93CF93E0914C04F0914D0416C0C2
:10FFE000E43B18F084E79FE0F2CF80910007E091B6
:10FFF0004C04F0914D0485FF03C08BE79FE002C0E5
:020000021000EC
:1000000082E89FE09F938F93DF93CF9309950F90A2
:100010000F900F900F908091F906882309F471C119
:100020008EE50E9460898091F90699279F938F93AE
:1000300089E89FE09F938F9382E399E89F938F9342
:10004000E0914C04F0914D0409958DB79EB706964A
:100050008DBF57C189E60E94608984E99FE09F9324
:100060008F93C2E3D9E8DF93CF93E0914C04F091F2
:100070004D0409950F900F900F900F908091F80606
:10008000E0914C04F0914D04882351F099279F93FF
:100090008F938EE99FE09F938F93DF93CF931DCE35
:1000A00082EA9FE09F938F93DF93CF93FAC0809172
:1000B0002804F2E3EF2EF9E8FF2E882309F053C05D
:1000C0008EE70E94608980918F0199279F938F937B
:1000D00080919506E82FFF27EE0FFF1FEA53F84F98
:1000E000808191819F938F9380919406E82FFF27C1
:1000F000EE0FFF1FEA53F84F808191819F938F93FA
:1001000088EA9FE09F938F93FF92EF92E0914C04D7
:10011000F0914D04099583E90E9460898DB79EB7DF
:100120000A968DBF80919706E82FFF27EE0FFF1FDD
:10013000EA53F84F808191819F938F938091960627
:10014000E82FFF27EE0FFF1FEA53F84F80819181C0
:1001500081589F4F9F938F938CEB9FE09F938F933A
:10016000FF92EF9241CE8EE70E9460898091110349
:1001700099279F938F938091100399279F938F9333
:1001800080910F0399279F938F938BEC9FE09F9310
:100190008F93FF92EF92E0914C04F0914D040995FA
:1001A00083E90E9460898DB79EB70A968DBF8091C2
:1001B000140399279F938F938091130399279F93FB
:1001C0008F938091120399279F938F938FED9FE0D8
:1001D0009F938F93FF92EF92E0914C04F0914D0426
:1001E00009952DB73EB7265F3F4F2DBF8AC080913E
:1001F0002E04882309F485C08EE70E9460898091CF
:10020000820886FD11C083EF9FE09F938F9383E563
:1002100099E89F938F93E0914C04F0914D040995D8
:100220000F900F900F900F908091FE0699278F707E
:100230009070892B89F082E090E19F938F9383E502
:1002400099E89F938F93E0914C04F0914D040995A8
:100250000F900F900F900F908091820882FF11C035
:100260008CE090E19F938F9383E599E89F938F9320
:10027000E0914C04F0914D0409950F900F900F9070
:100280000F908091820883FD3CC081E190E19F93B3
:100290008F9383E599E89F938F93E0914C04F091BD
:1002A0004D0409950F900F900F900F902AC00E9457
:1002B00014758093900925C00091700A063089F466
:1002C00080912804882319F01092280403C081E04B
:1002D0008093280486E00E94FC7487E00E94FC74EE
:1002E00008C0013031F40E94658900932504109202
:1002F00024041092700A05C01092240402C01092C7
:100300002504E6E0CDB7DEB70C94B98F4FB728E1EE
:1003100030E0F8948091C9008F778093C900809174
:10032000C9008F7B8093C9008091C9008F7D809325
:10033000C9005A9A52985B9A539A832F99278093AF
:10034000CD002093CC008091C80082608093C800CB
:1003500080E18093C9008091CA008F778093CA00A2
:100360008091CA008F7B8093CA008091CA008091DF
:10037000CA008F7E8093CA008091CA0088608093F3
:10038000CA008091C9008B7F8093C9008091CA0008
:1003900084608093CA008091CA0082608093CA0002
:1003A0008091C80087FF03C08091CE00F9CF809173
:1003B000C90080688093C90080916E0A8460809330
:1003C0006E0A4FBF089590910C04992341F48F3029
:1003D00031F490932A0480E580930C040895E09111
:1003E0002A04EF5FE0932A04E83121F481E080934E
:1003F00029040895E93120F089E180932A040895C1
:10040000FF27E95AF54F80830895A0E0B0E0EBE0C4
:10041000F2E80C94998F91E0D92E82E0A82EBD2CA1
:10042000E12C01E0F02E80916E0A82FDB5C0809132
:100430006F008F7D80936F00E091FB06EE2351F0FB
:10044000FF27EE0FFF1FEA53F84F8081918184361A
:1004500091055CF480910E03883C20F480910E039A
:100460008C5E01C088EC80930E038091580A682F3F
:10047000772780912B04815080932B048F3F31F498
:100480001CE7C12E82E080932B0402C0C4E2CC2E74
:1004900040E04C1508F07EC0EA2DFF27E95AF54FE1
:1004A00080818D2111F06E297F298D2D9927880F4C
:1004B000991FD82E882319F4B1E0DB2EAD0CEE0C79
:1004C000FF1C20E0E21628E0F20609F061C0A1E07E
:1004D000EA2EF12CCB018050944065E070E00E9440
:1004E000418FAB2DBB27FD01EA0FFB1FEA53F84FED
:1004F000808191819C01220F331F280F391F260F05
:10050000371F37FF02C02D5F3F4FE901D595C795D3
:10051000D595C795CB0101968C179D0714F42197AB
:1005200006C061507040C617D7070CF42196809121
:100530000E03833CD8F08D010A0F1B1FF801EA530C
:10054000F84F80819181FE01E81BF90BCF0163E038
:1005500070E00E94418FCB01880F991F860F971F73
:100560000650184FF8019183808307C0AA0FBB1F64
:10057000A650B84F11961C921E92EB2DFF27EE0F3E
:10058000FF1FEA53F84FD183C08360E070E0B3945B
:100590004F5F7FCF1092430110922904EAE0CDB75C
:1005A000DEB70C94B58F08950895002422273327D1
:1005B000442751E0BB27EE27FF27A0E1660F771FF6
:1005C000881F991F001C221F331F441F660F771FAF
:1005D000881F991F001C221F331F441F2AF4050E79
:1005E0002B1F3E1F4F1F04C0051A2B0B3E0B4F0B3A
:1005F000550FBB1FEE1F587F556047FD5250AA95FF
:10060000E9F6E695B7955795E695B7955795852FF1
:100610009B2F08952227332741E0552768E0880F54
:10062000991F221F331F880F991F221F331F1AF48F
:10063000240F351F02C0241B350B440F551F487F64
:10064000456037FD42506A9551F756954795569546
:100650004795842F0895AA2797FF04C08095909509
:100660008A1F9A1F77FF04C0609570956A1F7A1FD2
:10067000669F9001779FA001679F300D411D5A1F13
:10068000300D411D5A1F889FF001999F2E0F3F1F6B
:10069000401D511D899F300D411D5A1F300D411DB8
:1006A0005A1FCA01B901112480CF4FB720E430E0AE
:1006B000F8948091C9008F778093C9008091C90018
:1006C0008F7B8093C9008091C9008F7D8093C90082
:1006D0005A9A52985B9A539A832F99278093CD0008
:1006E0002093CC008091C80082608093C80088E18C
:1006F0008093C9008091CA008F778093CA0080914F
:10070000CA008F7B8093CA008091CA008F7D80933E
:10071000CA008091CA008F7E8093CA008091CA006F
:10072000877F8093CA008091C9008B7F8093C90026
:100730008091CA0084608093CA008091CA00826060
:100740008093CA008091C80087FF03C08091CE00CB
:10075000F9CF8091C90080688093C9004FBF089588
:100760000F931F93CF93DF93482F4F5F893108F08A
:100770008BC08091C507841720F44F5F4093C50755
:100780004150CB0183539B4268E170E00E94418F4E
:10079000A42FBB27FD01EA0FFB1FEA53F84F80810E
:1007A00091819B01281B390BC90137FF03C090952C
:1007B00081959F4F069794F480910E03883C30F406
:1007C00080910E03865F80930E0308C088EC8093AF
:1007D0000E0380916F008F7D80936F00FD01EA0F03
:1007E000FB1FEA53F84F808191819C01220F331F38
:1007F000280F391F260F371F37FF02C02D5F3F4FCD
:10080000E901D595C795D595C795CB0101968C176C
:100810009D0714F4219706C061507040C617D70792
:100820000CF4219680910E03843BD8F08D010A0FC1
:100830001B1FF801EA53F84F80819181FE01E81BEC
:10084000F90BCF0163E070E00E94418FCB01880F6C
:10085000991F860F971F0650184FF80191838083C8
:1008600007C0AA0FBB1FA650B84F11961C921E922C
:10087000E42FFF27EE0FFF1FEA53F84FD183C08309
:10088000443011F410924301DF91CF911F910F91E9
:100890000895CF93DF932091710A822F9927807F4B
:1008A0009070409709F06CC02F3109F046C08091DC
:1008B000720A809335042091740A20933704809142
:1008C000750A80933604822F99279093C7078093E7
:1008D000C607222309F054C080919406282F33279D
:1008E000220F331FF901E650F84F118210828091D8
:1008F0009506A82FBB27AA0FBB1FFD01E650F84F96
:100900001182108280919706E82FFF27EE0FFF1FBC
:10091000CF018650984FEC01198218822A53384F24
:10092000E90119821882AA53B84F11961C921E929F
:10093000EA53F84F1182108223C0C22FCF70CA3001
:10094000F8F48091720A80939D0A8091730A8093D3
:100950009C0A8091740A80939F0A8091750A809303
:100960009E0A60919C0A70919D0A8C2F0E94B08310
:1009700060919E0A70919F0A8C2F8F5F0E94B083B6
:10098000DF91CF910895CF93C82F8F3F49F4809185
:1009900038048F3F29F410923A041092390432C07F
:1009A00020913A04222339F4CF3111F485E001C0BB
:1009B00084E080933B0480913B049091390482173A
:1009C000A0F4892F8095809339048F3F19F48EEF1E
:1009D0008093390480913904C81711F40E94498426
:1009E00010923A04109239040BC0E22FFF27EF58FF
:1009F000F54FC0832F5F20933A049C0F90933904E6
:100A0000C0933804CF91089590913404933240F408
:100A1000E92FFF27E758F54F80839F5F90933404B9
:100A20000895833218F48D5F80933404089590E222
:100A3000ECE7FAE08FE19193815087FFFCCF0895B6
:100A4000CF93CFB723E031E0F8948091C9008F773E
:100A50008093C9008091C9008F7B8093C9008091E9
:100A6000C9008F7D8093C9005A9A52985B9A539A15
:100A7000832F99278093CD002093CC008091C800CC
:100A800082608093C80088E18093C9008091CA0089
:100A90008F778093CA008091CA008F7B8093CA00B1
:100AA0008091CA0080628093CA008091CA008061F0
:100AB0008093CA008091CA0088608093CA008091A8
:100AC000C90084608093C9008091CA0084608093CB
:100AD000CA008091CA0082608093CA008091C800D9
:100AE00087FF03C08091CE00F9CF8091C900806854
:100AF0008093C9008091C90080648093C9000E94DE
:100B00001785CFBFCF910895282F99278F709070A8
:100B1000892B31F4209580913304822B8093330408
:100B200008958091D301882309F44BC08091D202AB
:100B300085FD04C08091D601882381F082E98093ED
:100B4000790A83E280937A0A8091D601882309F496
:100B500085E580937B0A1092D60102C08093790AC2
:100B60008091D4018F3071F4809133040E94DF733F
:100B7000882341F081E98093790A80937A0A81E39E
:100B800080937B0A1092D3018091C80085FFFCCF2F
:100B90008091C9008F7E8093C9008091C9008E7FAB
:100BA0008093C9008091790A882311F48EEF01C0E7
:100BB0008EE78093CE00809133048093D40110920D
:100BC000330408951F920F920FB60F9211248F9342
:100BD0009F93EF93FF939091D301992309F040C025
:100BE00080913C04882361F48091790A882311F470
:100BF00083E003C0813999F481E080933C040FC005
:100C0000833099F48091790A882349F09093790A86
:100C10008091C9008E7F8093C9008EEF1EC08091A5
:100C2000C90081608093C9000EC0833261F4809155
:100C3000C9008E7F8093C9008FEF8093CE0081E042
:100C40008093D30114C080913C04E82FFF27E7581C
:100C5000F54F8F5F80933C0480818093CE0007C066
:100C600010923C048091C90080618093C900FF917B
:100C7000EF919F918F910F900FBE0F901F9018953D
:100C8000EF92FF920F931F93CF93DF937C018B0121
:100C9000EA01452B39F0F80181918F01F70109959F
:100CA0002197C9F7E6E0CDB7DEB70C94B98FEF9284
:100CB000FF920F931F93CF93DF937C018B01EA0187
:100CC000452B41F0F8010F5F1F4F8491F701099503
:100CD0002197C1F7E6E0CDB7DEB70C94B98F0F933B
:100CE0001F93CF938C01C62F161634F480E2F801BF
:100CF0000995C1501C16D4F3CF911F910F910895FF
:100D00000F931F93CF938C01C62F161634F480E3F4
:100D1000F8010995C1501C16D4F3CF911F910F9182
:100D20000895A5E3B0E0E7E9F6E80C94918F2E96DC
:100D3000EEADFFAD2E9788249924540180912D04A7
:100D4000882321F42C961FAE1EAE2C975EE4452E10
:100D5000512C4C0E5D1E6F01B60105C0153239F0E5
:100D60000894C11CD11CF60114911123B9F7A601F6
:100D7000461B570B31F02C968EAD9FAD2C970E94E1
:100D80005786112309F46AC20894C11CD11CFF24A0
:100D9000FDA6FCA64FEFE42EF9A6F6010894C11CAF
:100DA000D11C1491153721F0812F80628837B1F45E
:100DB000F0FE0AC0F20124E030E0420E531E8080B3
:100DC0009180A280B3800AC0F20142E050E0440E5C
:100DD000551E808191814C01AA24BB24103221F43C
:100DE00089A58823D1F61DC0133219F458E0F52ADD
:100DF000D4CF1A3211F01D3291F41A3259F4F201A3
:100E000082E090E0480E591EE081ECA7EE232CF61C
:100E1000E195ECA790E1F92AAFEDFA22BECF1B32A3
:100E200011F419A7BACF1E32C1F5F6010894C11CFE
:100E3000D11C14911A3279F4F20122E030E0420E12
:100E4000531E408151813FEF4F3F530714F44FEF42
:100E50005FEFE42EA2CF40E050E0812F80538A3034
:100E6000A0F4CA0133E0880F991F3A95E1F7840F87
:100E7000951F480F591F410F511D40535040F60117
:100E80000894C11CD11C1491E8CF8FEF4F3F580735
:100E900014F44FEF5FEFE42E85CF103329F4F4FC08
:100EA0007CCF90E2F92A79CF812F81538930D8F411
:100EB00040E050E0CA0123E0880F991F2A95E1F72E
:100EC000840F951F480F591F410F511D405350402B
:100ED000F6010894C11CD11C1491812F80538A30D3
:100EE00048F34CA75FCF183619F4A4E0FA2A55CF7F
:100EF0001C3619F4B1E0FB2A50CF133661F43E01E1
:100F00000894611C711CF20122E030E0420E531E75
:100F1000808189833CC1143421F0143611F01936D4
:100F200051F5143411F431E0F32AF0FE0AC0F20155
:100F300044E050E0440E551E80809180A280B38032
:100F40000CC0F20182E090E0480E591E8081918130
:100F50004C01AA2497FCA094BA2CB7FE0AC0B09406
:100F6000A09490948094811C911CA11CB11C8DE2D2
:100F700089A70AE06FC01F3411F01F3631F41F3407
:100F800011F491E0F92A08E064C0103779F4F20115
:100F9000A2E0B0E04A0E5B1E808191814C01AA2440
:100FA000BB2400E1B0E4FB2A18E753C01337C1F5B6
:100FB000F20122E030E0420E531E60807180611425
:100FC000710489F43E010894611C711C88E28983D4
:100FD0008EE6F301818385E78B838CE68C838D839A
:100FE00089E28E831F82E7FC13C08E2D992787FD2F
:100FF0009095AC0160E070E0C3010E945E8D0097A7
:1010000029F0382E3618E3140CF0C3C03E2CC1C0B2
:10101000F30101900020E9F731973E2E3618B9C050
:10102000153511F0153731F4153511F4F1E0FF2ABB
:101030000AE00FC0183519F0183709F0A0C000E118
:10104000F3FE07C081149104A104B10411F020E45F
:10105000F22A19A6EDA6E7FC02C03FEDF32289E2D1
:10106000682E712C6C0E7D1E81149104A104B104B4
:1010700021F44DA5442309F47BC0802F9927AA278A
:10108000BB278EA79FA7A8ABB9AB202E332490E037
:10109000891690E0990691E0A90690E0B90648F01B
:1010A000C501B4012EA53FA548A959A90E94548F96
:1010B00017C0AFEF8A169104A104B10449F040F0C3
:1010C000C401B1010E942D8F9B014427552708C000
:1010D000882D602F0E94218F282F332744275527E2
:1010E0002AAB3BAB4CAB5DAB0A3059F48AA9880FF5
:1010F000880F880F9AA9990F890F382D381B832FD5
:1011000010C0003139F48AA98295807F482D481B90
:10111000842F07C08AA9880F880F880F582D581B65
:10112000852F90E02EA53FA548A959A982169306C0
:10113000A406B50608F091E08AA89BA8ACA8BDA8B3
:101140008A3010F4805D04C0895A183509F48F7D07
:10115000D3018E933D01992309F099CF083041F4D2
:10116000F3FE06C0803321F080E3FD0182933F014E
:10117000CE010196382E3618F8E23F0E0BC011232F
:1011800009F46CC03E010894611C711C1983B1E024
:101190003B2E19A6032D2DA4231827FC222489A554
:1011A000882311F00F5F02C0F6FC0E5F020DEF2CDA
:1011B000FF24C70180739070892B49F48CA5801B94
:1011C000682F2C968EAD9FAD2C970E946F8689A5B7
:1011D000882331F041E050E0BE01675D7F4F0AC0D7
:1011E000E6FE0EC080E38AA71BA742E050E0BE01E6
:1011F000665D7F4F2C968EAD9FAD2C970E944086EA
:10120000C70180739070809749F48CA5801B682F6C
:101210002C968EAD9FAD2C970E948086622D2C96C9
:101220008EAD9FAD2C970E948086832D992787FDD8
:101230009095AC01B3012C968EAD9FAD2C970E947A
:101240004086E4FE89CD2CA5201B2CA7622F2C966E
:101250008EAD9FAD2C970E946F867ECDE2E1CB5C78
:101260000C94AD8F982F8091780A883A50F4809131
:10127000780AE82FFF27E257F64F93838F5F80931A
:10128000780A0895982F8091780A883A58F48091C6
:10129000780AE82FFF27E257F64F906893838F5F15
:1012A0008093780A0895982F80912E04882321F046
:1012B000892F0E9442890895892F0E9432890895BA
:1012C000883A10F48093780A089580E090E2E1E98A
:1012D000F9E091938F5F883AE0F308954FB721E8E2
:1012E00030E0F8948091C9008F778093C900809195
:1012F000C9008F7B8093C9008091C9008F7D809346
:10130000C9005A9A52985B9A539A832F99278093CF
:10131000CD002093CC008091C80082608093C800EB
:1013200088E18093C9008091CA008F778093CA00BA
:101330008091CA008F7B8093CA008091CA008F7D04
:101340008093CA008091CA008F7E8093CA008091EA
:10135000CA00877F8093CA008091C900846080930F
:10136000C9008091CA0084608093CA008091CA003D
:1013700082608093CA008091C90081608093C90017
:101380008091C80087FF03C08091CE00F9CF809183
:10139000C90080688093C9004FBF3CE7309335098E
:1013A0002DE720935A098EE88093360910924F0951
:1013B00010924E091092380930937D0920938D09BF
:1013C0001092870910928609109289091092880953
:1013D00010928B0910928A0984EF91E0909385090D
:1013E0008093840990938309809382099093810963
:1013F0008093800910927F0989E880937E0910927A
:101400008C0930933A0A2093560A10923C0A8AE8D3
:1014100080933B0A10923F0A10923E0A10923D0AB6
:101420001092410A1092420A1092430A1092440A02
:101430001092460A1092470A1092480A1092490ADE
:1014400010924D0A10924C0A10924B0A10924A0ABE
:1014500030935B0920937C0910925D098DE880939D
:101460005C098BE780938E0980E880938F09109246
:1014700090098091380990E2E1E9F9E091938F5F5A
:10148000883AE0F38DE78093390A0895CF93C82F07
:1014900080913D04803879F48C2F0E94CA75809326
:1014A000300480913004882311F1C093770A809131
:1014B00030048F5F12C08F37D1F48091700A882377
:1014C00029F48C2F80958F708093700A8EE899E0B4
:1014D00090933204809331048DEA8093300480919C
:1014E000C9008F7E8093C90082E080932F04C0934F
:1014F0003D04CF91089530912F04332331F0809132
:101500002F04815080932F04089580913004882304
:1015100081F14091300490913E04413091F4292FA3
:1015200030933E048091C90080618093C90080910E
:101530002E04882319F030932E0410C040932E04FB
:101540000DC0E0913104F09132048191F0933204A6
:10155000E0933104282F980F90933E048091C800A7
:1015600085FFFCCF2093CE00809130048150809382
:10157000300408952FB740E0F894E0E0F0E081E215
:10158000809357009491E2E0F0E08093570034910B
:10159000E4E0F0E08093570084912FBF9E3199F4EE
:1015A000363941F4893011F441E00DC08A3059F4E4
:1015B00042E009C0373939F4863011F443E003C002
:1015C000853009F444E0842F992708959FB7F89453
:1015D0008091C900877F8093C9008091C9008F7E68
:1015E0008093C9008091C9008F778093C900809152
:1015F000C9008F7B8093C9008091C9008F7D809343
:10160000C90052985A9A53985B9A9FBF08951F93A6
:10161000CF93DF93182F80912D04882309F4A7C05E
:101620008091D201181709F4A2C080912C0488235C
:1016300021F40E94BA8A80932C0482ED91E0909369
:101640004201809341018EEB90E19F938F93C0EF15
:10165000D4E1DF93CF93E0914C04F0914D040995D0
:101660000F900F900F900F90812F9927AA27BB27DB
:10167000FC01099778F5ED54FF4F20914C0430910F
:101680004D040C94C88F8AEB90E102C081EB90E18D
:101690009F938F93DF93CF93F901099527C08CEA2D
:1016A00090E1F6CF84EA90E1F3CF8CE990E19F934B
:1016B0008F93DF93CF93F901099588ED91E0909393
:1016C00042018093410112C087E990E1E1CF8BECA8
:1016D00090E1DECF81ED90E19F938F93DF93CF93E5
:1016E000E0914C04F0914D04099510E00F900F909B
:1016F0000F900F9080912C04843011F0823011F5FE
:101700000E94E68A812F8150833018F40E945F7016
:101710002CC0143019F40E94208527C0153019F40C
:101720000E94558322C0183019F40E94D3821DC034
:10173000163019F40E946E8918C01730B1F40E9457
:10174000868113C0112389F087EE90E19F938F93D8
:1017500080EF94E19F938F93E0914C04F0914D04BE
:1017600009950F900F900F900F901093D201DF9179
:10177000CF911F9108950F931F9381E080932D04C3
:101780004091D101E7E4F0E120E030E05FE48491B2
:1017900099272F5F3F4F829FB001839F700D929FCB
:1017A000700D112446275150319657FFF0CF4093CA
:1017B000D101EFE1F0E120E030E057E28491992798
:1017C0002F5F3F4F829FB001839F700D929F700DDE
:1017D000112446275150319657FFF0CF4093D10145
:1017E00080912C04882321F40E94BA8A80932C04CF
:1017F0008091D101833459F088E190E029E20FB65D
:10180000F894A895809360000FBE2093600081E952
:1018100096E890934D0480934C040E94EC0885E672
:1018200090E09F938F9388E590E09F938F931F9212
:101830001F92809102016AE00E94218F892F9927CF
:101840009F938F93809102010E94218F99279F93EC
:101850008F9382E091E19F938F9300EF14E11F93A8
:101860000F93E0914C04F0914D04099587E490E1C9
:101870009F938F931F930F93E0914C04F0914D042D
:1018800009958FE190E19F938F931F930F93E091C0
:101890004C04F0914D0409950E94EC0883EC809370
:1018A000810080916F00806280936F008DB79EB73A
:1018B00046968DBF1F910F9108958091F9068D3343
:1018C00038F08091A70887FD03C08CE38093F90668
:1018D0008091A906882331F08055853618F08FE76E
:1018E0008093A906089580912D04882309F477C078
:1018F00080913F04815080933F04882309F053C0B6
:1019000089E180933F048091F9068E3338F080910D
:10191000A70887FD03C08DE38093F90680910E032D
:10192000823820F58091D3029091D402885E934052
:1019300020F080913209843620F4109241041092F4
:1019400040048091400490914104009739F101973F
:101950009093410480934004419728F18091A70817
:1019600084FF21C08091D10284601BC080910E034E
:10197000853BC8F09091F90684E1989FC00111243D
:10198000409620914004309141042817390730F4E3
:101990002F5F3F4F30934104209340048091D10248
:1019A0008B7F8093D1029091D201963019F40E94DE
:1019B0007B8A0FC08091D501882321F081508093CC
:1019C000D501089586E98093D501943011F40E94E1
:1019D00091858091D101833411F010922D040895E6
:1019E0001F920F920FB60F9211242F933F934F9394
:1019F0005F936F937F938F939F93AF93BF93EF9377
:101A0000FF932091CE008091E0018823B1F02093D4
:101A1000C6008091E0018230B9F52F3FA9F58FEF24
:101A200094E3ACE0B0E0C297A109B109B7FFFBCFE6
:101A3000809190048093CE0027C09091D201892F8D
:101A40008150833020F4822F0E94BA701DC09430E0
:101A500021F4822F0E94848517C0953021F4822FB3
:101A60000E94C38411C0983021F4822F0E94D48236
:101A70000BC0963021F4822F0E94468A05C0973011
:101A800019F4822F0E94E381FF91EF91BF91AF91F2
:101A90009F918F917F916F915F914F913F912F9186
:101AA0000F900FBE0F901F901895FB01DC0102C034
:101AB00005900D9241505040D8F70895FC014150D7
:101AC000504030F001900616D1F73197CF010895BC
:101AD000882799270895A0E0B0E0E1E7FDE80C949D
:101AE000998F6C017B01EA01590121978FEFCF3F5C
:101AF000D80789F086010894C11CD11CC70108943D
:101B0000E11CF11CF5010995F80180832197FFEF95
:101B1000CF3FDF0779F7EAE0CDB7DEB70C94B58F9A
:101B2000CF92DF92EF92FF920F931F937C016B0194
:101B3000FB010995082FC7010196F6010995182F99
:101B4000C8011F910F91FF90EF90DF90CF90089503
:101B5000A0E0B0E0EEEAFDE80C949B8F8C017B01E5
:101B6000EA01690121978FEFCF3FD80771F0F701A4
:101B700021917F01C8010F5F1F4F622FF601099568
:101B80002197FFEFCF3FDF0791F7E8E0CDB7DEB752
:101B90000C94B78FCF92DF92EF92FF920F931F9327
:101BA0006C018B017A01FA010995812F9927682F21
:101BB000C6010196F70109951F910F91FF90EF90D3
:101BC000DF90CF9008955058BB27AA270ED0E0C0D1
:101BD000D1D030F0D6D020F031F49F3F11F41EF474
:101BE000C6C00EF4E095E7FBBCC0E92FE2D080F35D
:101BF000BA17620773078407950718F071F49EF50A
:101C0000FAC00EF4E0950B2EBA2FA02D0B01B901EE
